:020000040800F2
:100000000010002011030008130300081303000868
:100010001303000813030008130300081303000868
:10002000130300081303000813030008710F0008EE
:10003000130300081303000813030008611F0008DE
:100040001303000813030008130300081303000838
:1000500013030008130300081113000861130008BC
:10006000C113000821140008811400083119000888
:1000700061190008A1190008E1190008211A0008F7
:10008000511A0008911A000813030008130300080E
:10009000130300081303000813030008E114000809
:1000A00013030008130300081303000813030008D8
:1000B00013030008130300081303000813030008C8
:1000C00013030008130300081303000813030008B8
:1000D00013030008130300081303000813030008A8
:1000E0000116000813030008130300081303000897
:1000F000130300081303000813030008D11A0008B3
:100100001303000813030008130300081303000877
:10011000512100081303000813030008130300080B
:10012000111B0008411B0008811B0008C11B0008AF
:10013000011C000813030008130300081303000840
:100140001303000813030008130300081303000837
:10015000311C0008711C0008B11C000813030008C2
:100160001303000813030008130300081303000817
:100170001303000813030008130300081303000807
:1001800013030008130300081303000813030008F7
:1001900013030008130300081303000813030008E7
:1001A00013030008130300081303000813030008D7
:1001B00013030008130300081303000813030008C7
:1001C00013030008130300081303000813030008B7
:1001D00013030008130300081303000813030008A7
:1001E000B12D0008112F000821300008E13500086A
:1001F00072B6394880F30888384880F3098838484F
:100200004EF60851CEF20001086040F20000CCF238
:1002100000004EF63471CEF200010860BFF34F8F3C
:10022000BFF36F8F40F20000C0F2F0004EF688512D
:10023000CEF200010860BFF34F8FBFF36F8F4FF016
:100240000000E1EE100A4EF63C71CEF200010860AB
:10025000062080F31488BFF36F8F00F019F902F0C5
:100260000FF94FF055301F491B4A91423CBF41F8EE
:10027000040BFAE71C49194A91423CBF41F8040BB0
:10028000FAE71A491A4A1B4B9A423EBF51F8040B2F
:1002900042F8040BF8E700201749184A91423CBF86
:1002A00041F8040BFAE700F00BF900F0F9F8144CF0
:1002B000144DAC4203DA54F8041B8847F9E703F005
:1002C00067F9114C114DAC4203DA54F8041B88470E
:1002D000F9E700F0EDB80000001000200016002043
:1002E000000000080000002000100020043B00086F
:1002F000001600203416002038160020BCBB002059
:10030000E0010008F0010008F0010008F001000819
:100310006EE700F000F8FEE72DE9F04F2DED108AB2
:10032000C1F80CD0C3689D46BDEC108ABDE8F08FC3
:1003300000F0C6F9002383F311882846A047002067
:1003400000F0D6FC00F0ACF900F092FB00F0B8F938
:1003500000DFFEE7844641EA000313F003036DD19A
:10036000403A41D351F8043B40F8043B51F8043B78
:1003700040F8043B51F8043B40F8043B51F8043B7F
:1003800040F8043B51F8043B40F8043B51F8043B6F
:1003900040F8043B51F8043B40F8043B51F8043B5F
:1003A00040F8043B51F8043B40F8043B51F8043B4F
:1003B00040F8043B51F8043B40F8043B51F8043B3F
:1003C00040F8043B51F8043B40F8043B51F8043B2F
:1003D00040F8043B51F8043B40F8043B51F8043B1F
:1003E00040F8043B403ABDD2303211D351F8043BBF
:1003F00040F8043B51F8043B40F8043B51F8043BFF
:1004000040F8043B51F8043B40F8043B103AEDD26D
:100410000C3205D351F8043B40F8043B043AF9D2BE
:10042000043208D0D2071CBF11F8013B00F8013B91
:1004300001D30B8803806046704700BF082A13D39E
:100440008B078DD010F003038AD0C3F10403D21AB6
:10045000DB071CBF11F8013B00F8013B80D331F8EA
:10046000023B20F8023B7BE7043AD9D3013A11F86A
:10047000013B00F8013BF9D20B7803704B784370D5
:100480008B78837060467047000000000000000019
:10049000704700BF000000000000000000000000E6
:1004A000704700BF000000000000000000000000D6
:1004B000FEE700BF00000000000000000000000098
:1004C000F0B4144E144D154C154B164906F1700C32
:1004D00000279C4211D904391A4651F8040F42F8FA
:1004E000040B9442F9D8DA43144424F0030404348E
:1004F00023449D4203D943F8047B9D42FBD86645C3
:1005000005D0D6E90413D6E906451036E1E7F0BC7C
:10051000704700BF84360008BCBB0020BCBB002075
:10052000BCBB0020383B00080000000000000000B9
:10053000FEE700BF00000000000000000000000017
:10054000F8B51C4C1C4F1D4E002500F0A1F900F021
:100550004FF9C4E90C5500F08BFC00F0B1FC00F041
:10056000F7FC04F138008022154900F0C1FA154B60
:1005700001220277D968144AA0614FF6FF000140BA
:100580000A43DA60FA6842F08072FA60326810203A
:1005900042F0010220213260D87783F8221000F067
:1005A0006FF885F3118862B60848BDE8F84000F09E
:1005B000FFBA00BF481E0020F0ED00E0001000E090
:1005C0009C37000800ED00E00003FA05243700081E
:1005D00008B572B6034B0449D862D12202F028FD57
:1005E000FEE700BF481E002004370008000000009E
:1005F0002DE9F843164D00F0DBF8AA69D37F0BB163
:10060000013BD37700F0D4F8124FAB6AEC690133A9
:10061000BC42AB6219D0A668013EA660AEB94FF0ED
:1006200020092368D4F80C80E6605F60EB6100F07D
:1006300077F886F311882069C04789F3118800F0A4
:1006400057F8EC69A368002BEBD0BDE8F88300BF36
:10065000481E0020641E0020000000000000000072
:10066000044B1A6B0AB95B6B13B10348FFF7B0BFB9
:10067000704700BF481E00204437000800000000FB
:10068000044B1A6B0AB95B6B13B10348FFF7A0BFA9
:10069000704700BF481E00204C37000800000000D3
:1006A00010B5054C236B0BB9636B13B10348FFF70F
:1006B0008FFF0123636310BD481E002064370008CC
:1006C00010B5074C236B2BB9636B002B02DD0023A5
:1006D000636310BD0348FFF77BFF0023636310BD16
:1006E000481E0020743700080000000000000000D1
:1006F00010B5064C236B002B01DD636B13B104486E
:10070000FFF766FF0123636310BD00BF481E002092
:100710006C3700080000000000000000000000002E
:1007200010B5084C236B002B05DD636B002B02DD3D
:100730000023636310BD0448FFF74AFF002363638F
:1007400010BD00BF481E00207C37000800000000DC
:1007500010B5202383F31188074C236B002B01DB9A
:10076000626B1AB10548FFF733FF236B0133236334
:10077000002383F3118810BD481E00205437000861
:1007800010B5202383F31188074C236B002B01DD68
:10079000626B1AB10548FFF71BFF236B013B236314
:1007A000002383F3118810BD481E00205C37000829
:1007B000054B1A6B002A03DB5B6B002B00DD7047D7
:1007C0000248FFF705BF00BF481E0020843700081D
:1007D000044B1A6B1AB95B6B002B00DD70470248A3
:1007E000FFF7F6BE481E00208C370008000000000E
:1007F000054B4FF0FF30002103F11C025862996253
:10080000C3E90722704700BF481E00200000000017
:10081000F8B5054616461F460C46FFF7C9FF0C48BB
:100820002F61C369EE609A68944204D91B68A41AC8
:100830009A68A242FAD35A68C5E9003215605D6031
:10084000AC6099684FF0FF32091B99604262F8BDB5
:10085000481E002000000000000000000000000012
:1008600038B50446FFF7A4FF2368A5689A68616855
:1008700005482A449A600B60256800224FF0FF3338
:100880006960E260436238BD481E0020000000003D
:10089000034B0022C3E90033C3E904339A60704775
:1008A000481E0020000000000000000000000000C2
:1008B00010B50446FFF77CFF0022A168064B2277A3
:1008C0001B689A688A42FBD25A682046C4E9003203
:1008D00014605C6010BD00BF481E002000000000D6
:1008E00038B50446202383F31188FFF701FF237FE7
:1008F000072B10D8DFE803F0150F0F1B0A040F0AAF
:10090000256AFFF755FFAB680133AB60D4E90023DC
:100910001A60226853604FF0FF3323622046FFF7CE
:10092000C7FFFFF7FDFE002383F3118838BD236A5C
:1009300000221A604FF0FF3323622046FFF7B8FF12
:10094000EFE700BF00000000000000000000000012
:1009500070B50A4CA5690646FFF73AFF23682E7763
:100960001422EA771A682260012654601E7729460D
:10097000A3611846BDE87040FFF7CEBC481E0020BA
:1009800070B50D4686B00646FFF722FF6B1C14D0EB
:100990000E4C0F4AA369294601A8FFF739FF3046DC
:1009A000FFF7D6FFFFF704FF049B13B101A8FFF781
:1009B00057FFA369186A06B070BD044C3046FFF7B4
:1009C000C7FFA369186A06B070BD00BF481E0020AB
:1009D000E108000800000000000000000000000026
:1009E000F8B5144E0546B4690F46FFF7F1FEA3684B
:1009F000AA682F629A4217D9FFF7DAFE0023A1688E
:100A0000237733461B689A688A42FBD25A68626031
:100A10000120236014605C60287721462846B56178
:100A2000BDE8F840FFF778BC2846BDE8F840FFF77E
:100A30003FBF00BF481E0020000000000000000073
:100A4000084A93691168DA7F88689B6822B99842DE
:100A500034BF002001207047984294BF002001203D
:100A6000704700BF481E002000000000000000008A
:100A700070B51B4D2B68AC691A682A605560DE7F23
:100A8000AB6101221A77AEB9FFF792FEA168267713
:100A90002B461B689A688A42FBD25A68626014210E
:100AA000236014605C60E177A8692146BDE870406E
:100AB000FFF732BCFFF77CFE0023A16823772B46AB
:100AC0001B689A688A42FBD85A68A869C4E9003250
:100AD000214614605C60BDE87040FFF71DBC00BF9C
:100AE000481E002000000000000000000000000080
:100AF000F0B40B4C0B4F6569826382600026816104
:100B000000F1280200F1240145610461C761C0E9D8
:100B10000C6628616061C0E90912C262F0BC7047CE
:100B2000481E002002000114000000000000000028
:100B300070B50446FFF73CFED4E90416A3682568A7
:100B4000E06843F86C1C022103F82C1C142103F804
:100B5000291C012103F82A1C124A43F8686C002161
:100B600003F82B1C546943F8400C43F8100C43F86D
:100B7000305CA3F1AC000C4D43F83C0C43F84C5CEA
:100B800043E90611A3F14800A3F12001A3F12405D4
:100B900043E90E242061506143E9095143F81C1CCC
:100BA00070BD00BF481E0020310300080000000097
:100BB00010B52023044683F31188FFF771FD20460A
:100BC000FFF7B6FF00210446FFF70AFFFFF778FDA5
:100BD000002383F31188204610BD00BF00000000F1
:100BE0002DE9F843994604460D469046202383F3A9
:100BF0001188483D2C44184E184FFFF751FD089BB3
:100C0000716944F8203CA4F16402154BE260E36191
:100C100004F1240204F128030025124844F8249C1E
:100C2000C4E90461C4F8088044F8047CA061C4F8F5
:100C30003880C4E90C5520460C61C4E90923E362FD
:100C400029467461FFF7CCFEFFF73AFD85F3118862
:100C50002046BDE8F88300BF481E0020310300088D
:100C6000020001149437000800000000000000009A
:100C700010B52023044683F31188FFF711FDA37FED
:100C8000013BA377E36903F0FF130F2B01BFD4E906
:100C900004231A6122695361FFF712FD002383F3D5
:100CA000118810BD000000000000000000000000DE
:100CB00038B50E4B9C69636A206204F12405AB428F
:100CC00007D01A6862621846FFF7F2FD636AAB420A
:100CD000F7D1A37F23B9D4E904231A6122695361B0
:100CE0000F20BDE83840FFF733BE00BF481E00208C
:100CF00010B52023044683F31188FFF7D1FC20466A
:100D0000BDE81040FFF7D4BF000000000000000065
:100D100038B50446202383F31188FFF7C1FC237FF5
:100D20000F2B07D0094B626A9B6909201A60636226
:100D3000FFF70EFE256AFFF7C3FC002383F311883B
:100D40002046FFF795FF284638BD00BF481E00200B
:100D5000054B02469B6921B1036003201A62FFF72D
:100D60000FBE4FF0FF307047481E0020000000000B
:100D700003682BB10022026018461962FFF798BD84
:100D8000704700BF000000000000000000000000ED
:100D900069B1084B10B4024644689B690420C3E95A
:100DA0000024236053605DF8044BFFF7E9BD4FF06A
:100DB000FF307047481E00200000000000000000C7
:100DC000026890420AD010B414680460034663605D
:100DD000104611625DF8044BFFF76ABD704700BF13
:100DE00038B5036898420BD004460D461A68226055
:100DF000184654601D62FFF75BFD23689C42F5D1E5
:100E000038BD00BF0000000000000000000000002E
:100E1000014B5B6883607047001000E00000000039
:100E20000E4B0F4A5B68C168F0B48468D66F4268A5
:100E30001B1BD0E904459B1BE61845F100079342B4
:100E4000026888BF436001319342C0E90467C0E98A
:100E5000023138BF0360F0BC704700BF001000E0F3
:100E6000481E0020000000000000000000000000FC
:100E700010B50C4C86B000234FF0FF3100226846BD
:100E8000E367CDE9013303930023CDE90423009107
:100E9000FFF7BEFF6846FFF7C3FF029BE36706B09C
:100EA00010BD00BF481E0020000000000000000030
:100EB0000023C0E900008360704700BF000000000D
:100EC000034A044B02F50061C3E90021704700BFEB
:100ED000D01E0020C81E00200000000000000000FE
:100EE000F8B50E4604461546FFF762FC094AD2E9FA
:100EF00000737819013C3044714234440138084091
:100F0000214001448B4203D38F4201D81160F8BDC8
:100F10000020F8BDC81E00200000000000000000F6
:100F200070B5202304460D46164683F31188FFF75B
:100F3000B7FB324629462046FFF7D2FF0446FFF7AB
:100F4000BFFB002383F31188204670BD0000000022
:100F5000044B054A1A6003F10C000022C3E9012288
:100F6000FFF7A6BFD0260020210F000800000000D8
:100F7000064A536823F001035360EFF30983683393
:100F800083F30988002383F31188704730EF00E072
:100F9000202383F31188124B5B6813F4006302D1A2
:100FA00083F31188704710B5F1EE103AEFF309841E
:100FB0000C4B4FF08072DB6844F8083C44F84C2C32
:100FC000A4F1680383F30988FFF73AFD18B1064BD3
:100FD00044F8503C10BD054B44F8503C10BD00BFD8
:100FE00000ED00E030EF00E045030008500300088A
:100FF00008B500F0D5FB00F0FBFE00F0C9F800F0EA
:10100000DFF800F0BDF801F0DBFABDE8084000F0C1
:10101000CFB800BF0000000000000000000000008A
:10102000F8B5154682680669AA420B46816938BF41
:101030008568761AB54204461DD30AD818462A4652
:10104000FFF788F9E368A361A3685B1BA3602846E8
:10105000F8BD32461846FFF77DF9AF1B3A463044DB
:10106000E168FFF777F9A368E2685B1B3A44A26185
:10107000A3602846F8BD18462A46FFF76BF9A36916
:101080002B44A361A3685B1BA3602846F8BD00BF87
:1010900030B4029C046200250A4485600261C0E904
:1010A0000000C160C0E90511C36130BC704700BFDA
:1010B00038B504460D46FFF77BFBD4E90532934271
:1010C00011D0A268591C0132A26061611D70D4E97F
:1010D00004329A4201D3E368636120460021FFF79E
:1010E0006FFE002038BDA268002AEAD04FF0FF3022
:1010F00038BD00BF0000000000000000000000003C
:101100002DE9F04F83B006460D46144601929B46EA
:10111000C7694FF0200888F31188FFF7C1FAC4B1FE
:101120004FF00009224629463046FFF779FF8246F4
:10113000D0B1304607B1B847FFF7C2FA89F311883A
:10114000A4EB0A04554488F31188FFF7A9FA002C90
:10115000E8D1DDF804A0FFF7B3FA002383F3118888
:10116000504603B0BDE8F08F59463046FFF710FEF9
:101170000028D7D0019BA3EB040AECE70000000095
:10118000704700BF000000000000000000000000E9
:1011900000F0AEBE000000000000000000000000F3
:1011A000012200230270C0E901330C30FFF780BE3A
:1011B00000F0EEBE00000000000000000000000093
:1011C00001F046B800000000000000000000000030
:1011D0000023012202704370837043600372C0E9F0
:1011E0000333704700000000000000000000000012
:1011F00038B504460D46202383F31188FFF750FAD3
:101200002046656001F03CF802232370FFF758FA8E
:10121000002383F3118838BD0000000000000000A7
:1012200070B5202304460D46164683F31188FFF758
:1012300037FA32462946204601F0FAF80123A37016
:10124000FFF73EFA002383F3118870BD0000000011
:101250002DE9F0411F4604460E469046202383F3B5
:1012600011880125FFF71CFA424625723168204695
:1012700001F0AEF86570394604F11000FFF768FD23
:10128000054638B9FFF71CFA002383F31188284676
:10129000BDE8F081FFF78CFA6378012B05D04FF0A1
:1012A000FF3033681B1A3360ECE7204601F0B0F8DA
:1012B00000236370F5E700BF00000000000000009D
:1012C000430910B49B0000F1604404F5614403F14C
:1012D0006043090103F5614300F01F000122C9B218
:1012E00084F8001302FA00F0C3F880015DF8044BA3
:1012F00018607047000000000000000000000000BF
:1013000000F1604000F56D400901C9B201767047F7
:1013100008B5FFF71DFA104A516913680B4003F036
:101320000103536193B10D4A93680BB1D06898479C
:10133000202383F31188FFF7DBF900210748FFF72B
:101340004FFDFFF7EDF9002383F31188FFF718FA3B
:10135000BDE80840FFF71CBE003C0140702700209C
:1013600008B5FFF7F5F9104A516913680B4003F00F
:101370000203536193B10D4A93690BB1D069984749
:10138000202383F31188FFF7B3F900210848FFF702
:1013900027FDFFF7C5F9002383F31188FFF7F0F964
:1013A000BDE80840FFF7F4BD003C01407027002075
:1013B0008027002000000000000000000000000066
:1013C00008B5FFF7C5F9104A516913680B4003F0DF
:1013D0000403536193B10D4A936A0BB1D06A9847E5
:1013E000202383F31188FFF783F900210848FFF7D2
:1013F000F7FCFFF795F9002383F31188FFF7C0F995
:10140000BDE80840FFF7C4BD003C01407027002044
:1014100090270020000000000000000000000000F5
:1014200008B5FFF795F9104A516913680B4003F0AE
:101430000803536193B10D4A936B0BB1D06B98477E
:10144000202383F31188FFF753F900210848FFF7A1
:10145000C7FCFFF765F9002383F31188FFF790F9C4
:10146000BDE80840FFF794BD003C01407027002014
:10147000A027002000000000000000000000000085
:1014800008B5FFF765F9104A516913680B4003F07E
:101490001003536193B10D4A936C0BB1D06C984714
:1014A000202383F31188FFF723F900210848FFF771
:1014B00097FCFFF735F9002383F31188FFF760F9F4
:1014C000BDE80840FFF764BD003C014070270020E4
:1014D000B027002000000000000000000000000015
:1014E00010B5FFF735F93D4B5A691C68144004F4F8
:1014F00078725A61A30612D5394A936D0BB1D06D3B
:101500009847202383F31188FFF7F2F8002135482C
:10151000FFF766FCFFF704F9002383F311886006E8
:1015200012D52F4A936E0BB1D06E9847202383F3C8
:101530001188FFF7DDF800212B48FFF751FCFFF77A
:10154000EFF8002383F31188210612D5244A936F04
:101550000BB1D06F9847202383F31188FFF7C8F8A9
:1015600000212248FFF73CFCFFF7DAF8002383F361
:101570001188E20514D51A4AD2F8883013B1D2F88E
:101580008C009847202383F31188FFF7B1F80021DE
:101590001748FFF725FCFFF7C3F8002383F31188F2
:1015A000A30514D50E4AD2F8983013B1D2F89C0096
:1015B0009847202383F31188FFF79AF800210D48FC
:1015C000FFF70EFCFFF7ACF8002383F31188FFF759
:1015D000D7F8BDE81040FFF7DBBC00BF003C01407E
:1015E00070270020C0270020D0270020E0270020FF
:1015F000F02700200028002000000000000000006C
:1016000010B5FFF7A5F84B4B5A691C68144004F459
:101610007C425A61620514D5474AD2F8A83013B10A
:10162000D2F8AC009847202383F31188FFF760F8C5
:1016300000214248FFF7D4FBFFF772F8002383F341
:101640001188230514D53C4AD2F8B83013B1D2F82A
:10165000BC009847202383F31188FFF749F8002145
:101660003748FFF7BDFBFFF75BF8002383F31188D2
:10167000E00414D5304AD2F8C83013B1D2F8CC0007
:101680009847202383F31188FFF732F800212D4873
:10169000FFF7A6FBFFF744F8002383F31188A104AA
:1016A00014D5254AD2F8D83013B1D2F8DC009847C7
:1016B000202383F31188FFF71BF800212248FFF74E
:1016C0008FFBFFF72DF8002383F31188620414D5F4
:1016D000194AD2F8E83013B1D2F8EC009847202329
:1016E00083F31188FFF704F800211848FFF778FB0F
:1016F000FFF716F8002383F31188230414D50E4A4C
:10170000D2F8F83013B1D2F8FC009847202383F3C5
:101710001188FEF7EDFF00210D48FFF761FBFEF792
:10172000FFFF002383F31188FFF72AF8BDE810407C
:10173000FFF72EBC003C014070270020102800203D
:101740002028002030280020402800205028002099
:1017500060280020000000000000000000000000E1
:10176000062108B50846FFF7ABFD06210720FFF765
:10177000A7FD06210820FFF7A3FD06210920FFF79A
:101780009FFD06210A20FFF79BFD06211720FFF78A
:1017900097FD06212820BDE80840FFF791BD00BF56
:1017A000224B23481A696FEAC2526FEAD25210B52F
:1017B0001A611A69C2F308021A614FF0FF341A69FC
:1017C0005A695C6100215A6959615A691A6A62F062
:1017D00080521A621A6A02F080521A621A6A5A6AAF
:1017E0005C625A6A59625A6A1A6C42F080521A64F0
:1017F0001A6E42F080521A661A6E026842F48072C3
:1018000002601A6F02F44072B2F5407F03D04FF4C9
:1018100080321A671967064A536823F400735360CD
:1018200000F066FABDE81040FFF79ABF00380240AA
:1018300000700040000000000000000000000000F8
:10184000314B324A4FF080504FF4404118641160E0
:101850001A6842F001021A601A689207FCD599686A
:10186000294A21F003019960936813F00C03FBD11E
:101870001068254900F0F90010609360136843F484
:10188000803313600B689803FCD54B6F1E4A43F0FE
:1018900001034B67536F9907FCD51D4B53601368C9
:1018A0001A4943F0807313604B685A04FCD5164AFA
:1018B00013689B01FCD5174B174991601A68174BA9
:1018C0009A4217D0164B40F205721A600E4A93687E
:1018D00043F002039360936803F00C03082BFAD1E2
:1018E000536C43F480435364536E43F48043536614
:1018F000536E70470B4A0C4B12689A42E2D1084B68
:1019000040F205121A60E1E7003802400070004022
:1019100008544007002004E0009488381164002037
:10192000003C024000ED00E041C20F410000000019
:1019300008B5FEF70DFF084B084A196801F03D0194
:10194000996013680BB150689847FEF719FFBDE81E
:101950000840FFF71DBB00BF00600240EC260020DE
:1019600010B5FEF7F5FE094B094819688268890928
:1019700001F03D018C019C600AB1C0689047FEF700
:10198000FFFEBDE81040FFF703BB00BF0060024050
:10199000EC26002000000000000000000000000015
:1019A00010B5FEF7D5FE094B094819680269090C04
:1019B00001F03D010C049C600AB140699047FEF7BC
:1019C000DFFEBDE81040FFF7E3BA00BF0060024051
:1019D000EC260020000000000000000000000000D5
:1019E00010B5FEF7B5FE094B094819688269890DE3
:1019F00001F03D018C059C600AB1C0699047FEF77B
:101A0000BFFEBDE81040FFF7C3BA00BF0060024050
:101A1000EC26002000000000000000000000000094
:101A200008B5FEF795FE084B08485968026A01F0B0
:101A30003D01D9600AB1406A9047FEF7A1FEBDE8BA
:101A40000840FFF7A5BA00BF00600240EC26002066
:101A500010B5FEF77DFE094B09485968826A89096D
:101A600001F03D018C01DC600AB1C06A9047FEF7CD
:101A700087FEBDE81040FFF78BBA00BF0060024050
:101A8000EC26002000000000000000000000000024
:101A900010B5FEF75DFE094B09485968026B090C49
:101AA00001F03D010C04DC600AB1406B9047FEF789
:101AB00067FEBDE81040FFF76BBA00BF0060024050
:101AC000EC260020000000000000000000000000E4
:101AD00010B5FEF73DFE094B09485968826B890D28
:101AE00001F03D018C05DC600AB1C06B9047FEF748
:101AF00047FEBDE81040FFF74BBA00BF0060024050
:101B0000EC260020000000000000000000000000A3
:101B100008B5FEF71DFE084B08481968026C01F075
:101B20003D0199600AB1406C9047FEF729FEBDE87F
:101B30000840FFF72DBA00BF00640240EC260020E9
:101B400010B5FEF705FE094B09481968826C890932
:101B500001F03D018C019C600AB1C06C9047FEF71A
:101B60000FFEBDE81040FFF713BA00BF006402404B
:101B7000EC26002000000000000000000000000033
:101B800010B5FEF7E5FD094B09481968026D090C0F
:101B900001F03D010C049C600AB1406D9047FEF7D6
:101BA000EFFDBDE81040FFF7F3B900BF006402404D
:101BB000EC260020000000000000000000000000F3
:101BC00010B5FEF7C5FD094B09481968826D890DEE
:101BD00001F03D018C059C600AB1C06D9047FEF795
:101BE000CFFDBDE81040FFF7D3B900BF006402404D
:101BF000EC260020000000000000000000000000B3
:101C000008B5FEF7A5FD084B08485968026E01F0BB
:101C10003D01D9600AB1406E9047FEF7B1FDBDE8C5
:101C20000840FFF7B5B900BF00640240EC26002071
:101C300010B5FEF78DFD094B09485968826E890978
:101C400001F03D018C01DC600AB1C06E9047FEF7E7
:101C500097FDBDE81040FFF79BB900BF006402404C
:101C6000EC26002000000000000000000000000042
:101C700010B5FEF76DFD094B09485968026F090C54
:101C800001F03D010C04DC600AB1406F9047FEF7A3
:101C900077FDBDE81040FFF77BB900BF006402404C
:101CA000EC26002000000000000000000000000002
:101CB00010B5FEF74DFD094B09485968826F890D33
:101CC00001F03D018C05DC600AB1C06F9047FEF762
:101CD00057FDBDE81040FFF75BB900BF006402404C
:101CE000EC260020000000000000000000000000C2
:101CF0000E490F4A0F48002310B40B600E4C1946D2
:101D000001E052F80C0C016044F833100133102B41
:101D100002F10C02F5D10949094A5DF8044B4FF074
:101D2000FF338B60CB609360D36070476C270020DB
:101D3000C037000810600240EC260020006002401E
:101D400000640240000000000000000000000000ED
:101D5000F8B5DFF898C0477ADCF80050012404FA9F
:101D600007F62E423CD11F4C354304EBC70615F055
:101D7000FF0FCCF8005044F83720736009D01A4B9D
:101D80001C6B44F400141C631C6D44F400141C65AB
:101D90001B6D15F47F4F16D105682B6823F01F03C8
:101DA0002B602C6814F00104FBD1077A46683D23B0
:101DB000BB40212733602C606F617AB1807AFFF7D6
:101DC0007FFA2046F8BD084B1C6B44F480041C636A
:101DD0001C6D44F480041C651B6DDDE71046F8BDE6
:101DE0002046F8BDEC260020003802406C27002079
:101DF000054B002203F58071C3E90033C3E90222D9
:101E000010338B42F8D1704770270020000000008B
:101E10002DE9F04F02F00309C2F3800EC2F3C10CAA
:101E2000C2F34117C846C2F3C31200264FF0010A9D
:101E300016E0D0F800B003EA0B0343EA0803072ECC
:101E4000036044D8036A1D402C43046249083CD017
:101E50004FEA4E0E4FEA8C0CBF004FEA880801365D
:101E6000CB07F3D543680AFA06F423EA040343EAEE
:101E70000E03436003257300846805FA03F3DB4314
:101E80001C4044EA0C048460C56806F00704A40002
:101E90001D404FF00F0B3D430BFA04FBB9F1020F4D
:101EA000C56002FA04F46FEA0B05C2D1072E13D8FD
:101EB000D0F820B00BEA05052C43046204682340E7
:101EC00043EA080349080360C2D1BDE8F08F436AC2
:101ED0001D402C434462B9E7D0F824B00BEA050555
:101EE0002C434462EAE700BF00000000000000004D
:101EF00070B50F4E0F4D104C3046FFF751F90F4A99
:101F00000F4B1049F161204605F12401C6E9085143
:101F1000C6E90A23FFF744F90B490C4A0C4BE1616F
:101F2000A5F160010C3DC4E90815C4E90A2370BDA0
:101F30007028002014380008A02800201600010690
:101F40004600010600300140003C00401600010040
:101F5000460001000000000000000000000000003A
:101F600008B5FEF7F5FB202383F31188FEF7C0FBCD
:101F7000FEF73EFBFEF7D4FB002383F31188FEF748
:101F8000FFFBBDE80840FFF703B800BF00000000FA
:101F9000054B064A5A600021072299600B20082150
:101FA0001A60FFF7ADB900BF10E000E03F900200FB
:101FB000C1690A68136823F01F0330B41360136803
:101FC000DB07FCD40D7A046A496822683D23AB40E4
:101FD0000B60136823F01F031360136813F00103F1
:101FE000FBD1257A426960683D21A940016030BC7F
:101FF000D3601361536170470000000000000000CF
:1020000011F00C0F38B504462DD1216A0A68136807
:1020100023F01F0313601368DB07FCD463680D7A99
:1020200048681A683D23AB40022103606170BAB171
:10203000204690476378022B12D0237A03B938BD2B
:10204000202383F31188FEF753FB04F110000021D5
:10205000FEF78EFEFEF764FB002383F3118838BD84
:1020600000236370E9E70248FEF7B2FACDE700BF4C
:1020700074380008000000000000000000000000AC
:1020800011F00C0F2DE9F0410D46044613D1A27852
:1020900063683AB9DB68002B37D0A18C2046BDE8D5
:1020A000F04118475A6A52B1E80630D5204600215F
:1020B000BDE8F04110472548FEF78AFAE7E7E069F6
:1020C00001680A6822F01F020A600A68D207FCD47D
:1020D000077A46689D683D22BA4002203260A070AF
:1020E000FDB12046A847A378022B17D0202383F305
:1020F0001188FEF7FDFA04F10C000021FEF738FE0E
:10210000FEF70EFB002383F31188BDE8F081A906DA
:10211000FBD520460121BDE8F0411047E269636824
:102120001168DB68A269002B14BF4FF488734FF469
:10213000807313430120002504F12402A570CA60B6
:1021400048600B600B6803430B60CFE774380008EE
:10215000F8B53A4EFEF7FCFA7469E76825686368DB
:1021600040F20F131D422CD073681A696FF480730C
:102170002360BAB1ABB213F0080F0CBF00211021DD
:10218000D80748BF41F00401980748BF41F0080153
:10219000580748BF41F02001DB0548BF41F040012E
:1021A00026489047202383F31188FEF7A1FA6FF0A9
:1021B00001012348FEF7DCFDFEF7B2FA002383F3AA
:1021C000118868060ED579060CD573686FF040014A
:1021D0005A68216007EA0103E3600AB11748904793
:1021E000347AECB1EA0615D5FB0613D573681B6A81
:1021F0000BB112489847202383F31188FEF778FA31
:102200004FF0FF310E48FEF7B3FDFEF789FA0023C9
:1022100083F31188FEF7B4FABDE8F840FEF7B8BEC4
:10222000202383F31188FEF763FA21460548FEF761
:102230009FFDFEF775FA84F31188D3E7D0280020BC
:10224000DC280020E0280020000000000000000042
:1022500010B5074C2046FEF7BBFF064B064A6261ED
:10226000062103F11802C4E90613226210BD00BF63
:10227000D0280020CC370008004C004000000000AF
:102280000378012B2DE9F041044655D04569002320
:10229000A37063702046FFF78BFE434B6169994240
:1022A00063683BD041485A69814238D04049B1FB0C
:1022B000F2F2198B080438D4D3F80CE0D3F820805C
:1022C0005F8B988BE369AA602A686A68D4F818C0A3
:1022D0001B6800222A6042F21C1642F20C12B8F16E
:1022E000000F08BF1646BEF1000F14BF4FF48872EE
:1022F0004FF48072314342EA0C02012647F0400756
:1023000040F0C10024342F616861E960DC605E60E8
:102310001A601A6832431A60BDE8F0815A6925498B
:10232000B1FBF2F2198B0804C6D522F0070002F0C7
:10233000070242EA4002BFE71F4B984215D063688C
:102340001B8B03F4A053B3F5805F03D1A36943F45F
:102350002053A361D4E90723656910681968002236
:102360002B1D83608B60A28491E70346134AC069EA
:102370000621FFF7EDFC2346114A206A0621FFF7EC
:10238000E7FC104B1A6C42F400221A641A6E42F4F5
:1023900000221A66062134201B6EFEF791FFA36906
:1023A00043F00063A361CAE700100140001401403C
:1023B00080DE800200BD0105D028002081200008B9
:1023C000012000080038024000000000000000006A
:1023D00030B4036A456884691B686D68DA6044F448
:1023E0008A6459601C606DB142696FF040011160F0
:1023F000D16841F04001D1601A6842F001021A60D0
:1024000030BC7047027A002AEED0F5E700000000E9
:10241000016A0A68136823F01F0313601368DB075F
:10242000FCD4087A49683D2383400B6050687047AC
:10243000F0B4C5692B681C6824F01F041C601C687C
:10244000E407FCD444682F7A6E68656A3D24BC407A
:1024500034608069DA60002D0CBF4FF482624FF463
:10246000A362024359601A601A6842F001021A60BE
:10247000F0BC7047000000000000000000000000F9
:10248000404A414913694148F0B440F2FF142343E4
:10249000136113693E4E3F4D23F4FF7323F0010394
:1024A00013611369136B23431363136D2343136584
:1024B0006FF4A8470023126D4B604FF6FF728F60D8
:1024C000CE60354E4A610E62344E4E6206F12A5697
:1024D00006F5B0160E60402646604FF0FF31304ED4
:1024E0008160C6604FF08066426106624FF402561A
:1024F000436206602B4E2C4C6B60A960EE60012697
:102500006A612B626B622E60284D6360A160E5609A
:1025100040F6FF756561264D2362264E6362256095
:10252000C0F8043C244DC0F8081C04F58054C0F8E1
:102530000C3CC0F8142CC0F8203CC0F8243CC0F877
:10254000003C00F5E0507360B160F360726133628B
:10255000736233606B60A960EB606A612B626B62CF
:102560002B606360A160E360626123626362236049
:102570004360F0BC8160C3604261036243620360F8
:10258000FFF75EB90038024000000240000402403C
:1025900054000140000802400000565500AA0A00FD
:1025A0001585AAAAA8AAAAAA000C0240555055004F
:1025B0000001005500140240001802400000000015
:1025C000704700BF00000000000000000000000095
:1025D000434B1A69002A75DB70B5414BDA68D103A9
:1025E000FCD41A6922F480721A611A6942F40072EA
:1025F0001A611A6922F0F8021A61C20703D51A6932
:1026000042F008021A61860704D5354A136943F07F
:1026100010031361450704D5314A136943F02003C1
:102620001361040704D52E4A136943F04003136174
:10263000C10641D42A4B1A6942F002021A611A6992
:1026400042F480321A61DA68D203FCD41A6922F0AB
:1026500002021A611A6942F0004206461A61002815
:102660003AD005464FF00064013DEDB2284600F037
:1026700077F90444002DF7D1304600F071F90328B2
:1026800005D80AE00438032804F1040405D92368B6
:102690000133F7D06FF00A0070BD0028FCD023781A
:1026A000FF2BF7D1204402E02378FF2BF2D1013435
:1026B000A042F9D1002070BD094A136943F080039C
:1026C0001361B7E70749084A59605A601B69002B34
:1026D00082DA4FF0FF3070474FF00064CCE700BF64
:1026E000003C024023016745AB89EFCD00000000AC
:1026F00008B50B4601461846FDF72CFE002008BD24
:102700002DE9F043464B1F69002F83B004460E4667
:10271000154679DB424FFB68D803FCD43B6923F4B0
:1027200080733B613B6943F400733B6114F0030326
:1027300023D0A4EB030902A8C3F10408D9F80020B0
:1027400040F8042DA84528BFA84618444246314603
:10275000FDF700FE3B690199314A43F001033B61FB
:10276000C9F80010D368D903FCD4136923F001031E
:1027700044444644A5EB08051361032D23D9A5F174
:10278000040E4FEA9E0C264A06EB8C07311FA01B55
:10279000136951F8048F43F00103136140F801807D
:1027A000D368DB03FCD41369B94223F0010313613E
:1027B000EED104342EF0030E0CF1010C744406EB40
:1027C0008C0605F0030545B9154A136943F000432B
:1027D0001361002003B0BDE8F08302A8236840F82D
:1027E000043D2A463146FDF7B5FD0D4A01991369AE
:1027F00043F0010313612160D368DB03FCD4136948
:1028000023F001031361DFE70649074A59605A6064
:102810001B69002BBFF67EAF4FF0FF30DAE700BF39
:10282000003C024023016745AB89EFCD000000006A
:10283000F8B5234D234C4FF480610E464FF40077DA
:1028400028460122FFF7E4FA284601223946AE6104
:10285000FFF7DEFA284601224FF48071AF61FFF7DF
:10286000D7FA4FF48073AB61284601224FF4006120
:10287000FFF7CEFA4FF400633946AB6120460122E0
:10288000FFF7C6FA4FF00073A361204601224FF410
:102890000041FFF7BDFA4FF000433146A3612046E7
:1028A0000122FFF7B5FA4FF08063A36120460122B1
:1028B0004FF48041FFF7ACFA4FF08043A361F8BDBD
:1028C00000000240000C0240000000000000000078
:1028D00010B40E4B0E491A6892F8913043F0010380
:1028E00082F891300B68022403204FF4E13183F821
:1028F0002A4783F82E4783F82B0783F82F07C2F85F
:102900008010C3F830185DF8044B7047281600207B
:102910002C16002000000000000000000000000055
:102920000A4B0B4A1B68116893F890200120024360
:1029300083F89020C1F8380A93F89020042142F0DF
:10294000080283F86B1083F8902070472816002047
:102950002C16002000000000000000000000000015
:10296000032811D9A0F10C03032B0DD904280ED094
:1029700010280CD0431F062B0CD91138062894BF01
:102980004FF40030002070474FF4804070474FF400
:10299000803070474FF40030704700BF00000000E7
:1029A0002DE9F041202383F31188FDF7A1FE124B9E
:1029B000124FDB691B685E683B6A3D6AC6F1200600
:1029C000B342C8BF2036AE420EDDDFF834802C465D
:1029D00003E0A64204F01F0506D0795D4046FEF7ED
:1029E00067FB01340028F4D03D62FDF799FE002317
:1029F00083F31188BDE8F081D0280020F82800205A
:102A0000CC2A0020000000000000000000000000B0
:102A1000FFF7C6BF0000000000000000000000003B
:102A2000FFF7BEBF00000000000000000000000033
:102A300070B51E4C94F8F13213F0010382B002D14C
:102A4000036002B070BD1A4E1A481B4D00F0F8FA30
:102A500033681A4893F82B1740F2024200F028FA24
:102A60003368174893F82A1740F2024200F020FA20
:102A70000026144800F0E4FA05F1240105F5EA7097
:102A800033464FF4D7720096FEF702FB0E49D4F896
:102A9000E0320E484B61FEF7ABFB0C482E622A4633
:102AA000202102B0BDE87040FEF7BABB0000001064
:102AB0002C16002090380008F8280020A8380008BC
:102AC000B8380008C838000800160020D0280020B8
:102AD00010B582B002A8144640F8042D4FF47A7362
:102AE0000A4601460648FEF7B3FB019AA24204D00B
:102AF00023460449044800F0ABFA02B010BD00BF01
:102B0000D0280020DC380008B8BA002000000000FF
:102B10000148FEF7F5BA00BFCC2A002000000000F3
:102B200063498160F0B500244FF47F450460C460C0
:102B3000846144620463C463846444650466C46657
:102B4000846785800582858305858586A0F8405049
:102B5000A0F84C50A0F85850A0F8645041610162B0
:102B6000C162816341640165C16581664167C0F8E6
:102B700080102246A0F8705000F1B003A0F87C50FD
:102B8000C0F88440A0F88850C0F89040A0F8945055
:102B9000C0F8A040A0F8A450C0F88C10C0F898105D
:102BA000C0F8A81000F5B875FF2499601A601A7172
:102BB0005C710C33AB42F8D14FF47F43C0F8702105
:102BC000C0F87C21C0F88821C0F89421A0F87431A5
:102BD000A0F88031A0F88C31A0F89831C0F87811B5
:102BE000C0F88411C0F89011C0F89C1100F5D073A2
:102BF00000F548750022FF240026002799601A601E
:102C00001A715C71DA60C3E904675A769A761C76A9
:102C10002033AB42F2D100F588650022FF24996091
:102C20001A601A715C71DA601A751A611833AB4256
:102C3000F5D1204CDFF898E0DFF898C0C0F84814D0
:102C40004FF47F47C0F84024C0F85814C0F84C2413
:102C5000C0F85024C0F85C2404F59075264623463D
:102C6000A0F84474A0F854741349C0F8ACE0134AB7
:102C7000C0F89CC001E051F8042FC3F82C2318338E
:102C8000AB42F8D10E490F4A002384F8B831013322
:102C90000C2BC4F8AC2104F1200402D051F8042F0D
:102CA000F3E7094A094BC6F84C24C6F85C34F0BD7A
:102CB000F02A0020F82A0020283900088839000866
:102CC000583900088C390008A0390008A4390008D8
:102CD000903900089839000800000000000000004A
:102CE000184B98421FD003F58063984221D003F51A
:102CF0008063984219D003F5806398421BD003F596
:102D00008063984219D003F5006398420FD003F511
:102D10008063984213D00C490C4B0D4A88420CBF7B
:102D20001846104670470B4870470B4870470B48D1
:102D300070470B4870470B4870470B4870470B486B
:102D4000704700BF00000240001402401C39000818
:102D50002039000800390008083900081439000833
:102D6000043900080C390008103900081839000827
:102D7000012907D910B58C1E230658BF04F00F0097
:102D800003D410BD4FF0FF30704702460B4641F2AE
:102D9000F270034900F064F94FF0FF3010BD00BF3E
:102DA000A83900080000000000000000000000003A
:102DB0000148FFF7B5BE00BFF82A00200000000060
:102DC000064B1B6840203F21132283F80C0883F830
:102DD0000D1883F80E28FFF72BBD00BF2C1600201E
:102DE00030B40F4B0F491A6892F8913043F0210329
:102DF00082F891300B682C202D214FF416454FF4AA
:102E0000E13483F82A0783F82E0783F82B1783F819
:102E10002F17C2F88050C3F8304830BCFFF758BDB8
:102E2000281600202C1600200000000000000000E2
:102E30000B4B0C4A1B68116893F89020032042F05A
:102E4000040283F89020C1F8380A93F890203621C4
:102E500042F0080283F86B1083F89020FFF760BD02
:102E6000281600202C1600200000000000000000A2
:102E7000012908D910B58C1E230606D42411074B4E
:102E800053F8240010BD0020704702460B4641F263
:102E9000F270034900F0E4F8002010BD4C3A00083D
:102EA000A839000800000000000000000000000039
:102EB000F0B583B005460E461746FFF7D9FF3146F9
:102EC00004462846FFF754FF84B106462046FFF724
:102ED00007FF2A4603460B490B48009600F0B8F856
:102EE0002A463146204600F05BF808B103B0F0BD39
:102EF00001213A462046B14003B0BDE8F040FEF75C
:102F000087BF00BF6C3A0008582F00200000000067
:102F10000149024800F0ACB8443A0008582F00209C
:102F200008B51C4B98421ED003F5806398421ED012
:102F300003F58063984218D003F58063984218D057
:102F400003F58063984216D003F58063984214D04D
:102F500003F5806398421AD003F58063984208BF56
:102F600007200CD108BD002008BD022008BD0120AB
:102F700008BD032008BD042008BD052008BD064982
:102F800041F2F47000F06CF84FF0FF3008BD0620FD
:102F900008BD00BF00000240843A000800000000A5
:102FA0002DE9F041194B1C6882B02CB30D46174631
:102FB0008046FFF7B5FF164C05EB001654F82600C7
:102FC00040B9144A44F8267013680133136002B004
:102FD000BDE8F0814046FFF783FE54F826300193A8
:102FE000024600972B460C4941F2F57000F038F884
:102FF000012002B0BDE8F081084941F2F37000F011
:103000002FF8204602B0BDE8F08100BF5C320020FE
:103010005C30002060320020B03A0008943A00088A
:103020000149024800F024B8783A000864320020D0
:10303000704700BF0000000000000000000000001A
:103040000FB404B0704700BF000000000000000093
:103050000EB403B0704700BF000000000000000085
:103060000EB403B0704700BF000000000000000075
:10307000704700BF000000000000000000000000DA
:1030800030B5164B83B004461B68154805226946C7
:10309000FFF73EFD052802D0002003B030BD9DF8AB
:1030A00000309DF801509DF802109DF80300009A31
:1030B0006B404B409DF804104340994212BAEBD14B
:1030C00002F17843B3F5004F38BF064B4FF00100D3
:1030D00038BFD218226003B030BD00BF30160020C8
:1030E00068330020243500180000000000000000B4
:1030F00010B5044672B6FDF7B3FA0F4A606853681C
:1031000023F0805353600022930003F1604303F5E2
:1031100061430132D3F80012C3F88010082AF3D1BA
:10312000002383F31488236883F3088880470348C7
:10313000BDE81040FDF74CBA00ED00E0CC3A0008C5
:103140002DE9F04F89B008A9C948CA4CDFF83C9373
:10315000DFF82483792301F81D3D0122C823236071
:103160000646FFF7B5FC4FF400424FF000614846B9
:10317000FDF7F0F82368002701220DEB020130462D
:10318000FFF7C6FC0128054610D06FB9002009B032
:10319000BDE8F08F5246B8493046FFF7B9FC012828
:1031A000074600F02E8101272368E5E702462368E1
:1031B0000DF102013046FFF7ABFC012882460BD02F
:1031C000002FE3D008A91F2301F81C3D2A463046F2
:1031D000FFF77EFC2368CFE79DF801309DF80220C1
:1031E000DB43DBB29A4208A908D01F2301F81B3D3C
:1031F00002463046FFF76CFC2368BDE7792502469E
:1032000001F81A5D3046FFF763FC9DF801204FF48A
:103210007A73112A23600AD01AD9312A53D0442A4A
:10322000B8D0212A3CD04FF47A730127A4E707A82D
:10323000FFF726FF08A90746002874D11F2301F8CD
:103240000B3D52463046FFF743FC2368012793E7C6
:10325000002A47D0022AE6D1884B08A91F6801F846
:1032600016AD52463046FFF733FCC7F30B0708A9EB
:103270003B0A01F8153D52463046FFF729FC08A9E4
:10328000524601F8147D3046FFF722FC08A9524649
:1032900001F8135D3046FFF71BFC574623686BE7C8
:1032A00007A8FFF7EDFE08A90746002800F09F8059
:1032B000524601F8125D3046FFF70AFC0798FFF707
:1032C00017FF236858E707A8FFF7DAFE08A90746A3
:1032D000002852D11F2301F8073D52463046FFF720
:1032E000F7FBB2E708A90623654D01F8183D5246E1
:1032F0003046FFF7EDFBAF1D312301E015F8013B30
:103300008DF8093001220DF109013046FFF7E0FB8D
:10331000AF42F3D108A9792301F8193D01223046C3
:10332000FFF7D6FB3FE7524601F80C5D3046FFF74A
:10333000CFFB5246236804A93046FFF7E9FB01287A
:1033400083D1024623680DF111013046FFF7E0FBFF
:10335000012802467FF479AF9DF810309DF81100E6
:10336000D943C9B2884208A900F0D4801F2301F8CC
:103370000D3D3046FFF7ACFB67E7524601F8085DAC
:103380003046FFF7A5FB524623683B493046FFF71E
:10339000BFFB01287FF459AF98F80050DFF8E4B084
:1033A000236805F1020A524659463046FFF7B0FB42
:1033B00082457FF44AAF5FFA8AF2012A98F800301A
:1033C00008D90BF1FF32AB4412F8011F5A4583EACA
:1033D0000103F9D118F80A209A4272D008A91F23D4
:1033E00001F8093D01223046FFF772FB2DE71F234C
:1033F00001F8113D52463046FFF76AFB57462368F5
:10340000BAE6024623681F493046FFF781FB0128D0
:103410007FF4CAAE98F8001098F80120236842EAB9
:1034200001224FF6FF718A4260D05200D51C2A4615
:1034300015493046FFF76CFB85427FF406AF6B1CE5
:10344000DBB2012B98F8001009D90B480122013298
:1034500010F8017FD2B29A4281EA0701F7D308EB54
:1034600005035B788B4227D1013D00271BE000BF9D
:10347000683300203016002024B50020002004E02E
:10348000E13A000825B5002026B5002024350020AB
:103490009A78DB7843EA022318B2012BC0B232D902
:1034A000FFF796F80237BD4208EB0703F0DC08A9E6
:1034B000792301F8063D31E708A91F2301F8053DEE
:1034C0002CE707982349484505F1010202D3224B16
:1034D000984237D3FFF714F908A9792301F80A3D78
:1034E00001223046FFF7F4FA236845E601221B4922
:1034F0003046FFF70DFB012805467FF4A6AE98F88D
:1035000000100223A1E74FF40042FF21484600F0DB
:103510006FF8C7E701F80E5D30465D1CFFF7D8FA7B
:103520000799494502D30C4B99420ED308462A46C7
:103530004146FFF7DDF82A4641463046FFF7C8FA14
:10354000236819E6FCF706FFC6E72A464046FCF763
:1035500001FFF0E725B5002024B5002026B50020A6
:1035600000487047683300200000000000000000A1
:1035700008B5054B054A9B699A61FFF7E1FD0020FC
:10358000BDE80840FDF7B4BB481E0020F03A000833
:1035900010B582B0FDF72CFD0024FCF7D1FFFFF73A
:1035A0000FFCFFF71DFCFFF743FCFFF7D9FFFFF708
:1035B0003FFA084B009480224FF492610648FDF7D1
:1035C0000FFBFDF7A5FB0548FFF792FD204602B073
:1035D00010BD00BF7135000828B60020008000082B
:1035E00001490248FFF744BDE83A0008B8BA002094
:1035F000F0B4860743D0541E002A3ED0CAB2034618
:1036000002E014F1FF3438D303F8012B9D07F8D101
:10361000032C2BD9CDB245EA05250F2C45EA0545EB
:1036200016D9A4F110073F0903F1200606EB07168F
:1036300003F1100242E9045542E902551032B24248
:10364000F8D104F00F040137032C03EB07130DD955
:103650001E462246043A032A46F8045BFAD8221F83
:1036600022F003020432134404F003042CB1C9B263
:103670001C4403F8011B9C42FBD1F0BC704714466C
:103680000346C5E7383B0008BCBB0020BCBB00209C
:10369000BCBB0020383B00080000002000000020D8
:1036A00000000020383B000800C0012000C00120BD
:1036B00000C00120383B00080000000000000000AE
:1036C00000000000383B000800000010000000105F
:1036D00000000010383B000800400240004002405B
:1036E00000400240383B00080000000000000000DD
:1036F00000000000383B000800000000000000004F
:10370000000000002E2E2F43686962694F532F6F0F
:10371000732F72742F7372632F63687379732E63C0
:10372000000000003C37000838160020481E00202A
:1037300001000000310500080000000069646C65AC
:10374000000000005356233100000000535623337D
:103750000000000053562338000000005356233960
:103760000000000053562334000000005356233657
:103770000000000053562335000000005356233745
:10378000000000005356233130000000535623310F
:10379000310000006E6F6E616D6500006D61696ED5
:1037A00000164028040444080C101418001C1D00C6
:1037B0001F000000106002400860024000000B0083
:1037C000286002400860024006010C004060024090
:1037D0000860024010020D0058600240086002407C
:1037E00016030E00706002400C60024000040F00DF
:1037F000886002400C60024006051000A060024094
:103800000C60024010061100B86002400C600240DB
:1038100016072F00106402400864024000083800B8
:1038200028640240086402400609390040640240EE
:1038300008640240100A3A005864024008640240DA
:10384000160B3B00706402400C640240000C3C000C
:10385000886402400C640240060D4400A0640240EB
:103860000C640240100E4500B86402400C64024033
:10387000160F460053544D33325F554152545F4446
:103880004D415F4552524F525F484F4F4B00000031
:1038900054756E657253747564696F206F766572C6
:1038A000205553415254000074756E6572737475DF
:1038B00064696F207278000074756E657273747538
:1038C00064696F20747800005573696E67205541F4
:1038D00052542D444D41206D6F64650021212120FB
:1038E0004E4F5420414343455054454420256420C5
:1038F0006F7574206F66202564202121210000004F
:10390000504100005042000050430000504400006D
:10391000504500005047000050480000504600004D
:10392000756E6B6E6F776E0088390008183A000864
:103930001C3A0008203A0008243A0008283A0008F7
:103940002C3A0008303A0008343A0008383A0008A7
:103950003C3A0008403A00088C390008EC3900086D
:10396000F0390008F4390008F8390008FC3900087B
:10397000003A0008043A0008083A00080C3A000827
:10398000103A0008143A0008633100006931000061
:1039900064697A7A7900000074616368000000004D
:1039A000613100006132000025733A20496E766172
:1039B0006C696420627261696E5F70696E5F653AFE
:1039C000202564006F757470757450696E205B25D6
:1039D000735D20616C7265616479206173736967DE
:1039E0006E656420746F20257825640069320000BC
:1039F0006933000069340000693500006936000051
:103A000069370000693800006A3900006941000028
:103A10006942000069430000633200006333000024
:103A20006334000063350000633600006337000034
:103A30006338000063390000634100006342000006
:103A400063440000696F5F70696E7300000002409C
:103A50000004024000080240000C02400010024036
:103A60000014024000180240001C02402573206F21
:103A70006E2025732564000070696E207265706F7A
:103A800073000000756E6B6E6F776E20706F7274CE
:103A9000000000007265706F7369746F7279206E38
:103AA0006F7420696E697469616C697A656400007D
:103AB0002573256420726571206279202573207535
:103AC0007365642062792025730000006466754A7E
:103AD000756D70546F417070204641494C00000074
:103AE000310002112131440062696E617279000077
:103AF000426F6F746C6F6164657253657269616C5B
:103B000000000000000000000000000000000000B5
:103B10000000000000000000000000000000004065
:103B200000000000212A0008112A0008600200108D
:083B300008000010C8000000AD
:1080000000100020D1830008D3830008D383000828
:10801000D3830008D3830008D3830008D3830008E8
:10802000D3830008D3830008D383000811A8000875
:10803000D3830008D3830008D3830008D1D5000878
:10804000D3830008D3830008D3830008D3830008B8
:10805000D3830008D383000891B90008E1B9000870
:1080600041BA0008A1BA000801BB000821CB0008F2
:1080700051CB000891CB0008D1CB000811CC0008EF
:1080800041CC000881CC0008B1C1000881C70008BC
:10809000A1C70008C1C70008E1C7000861BB00080C
:1080A00091DB000821DB0008D383000841DB0008D6
:1080B00051DB000871DB0008C1DD0008D383000834
:1080C000D3830008D3830008D3830008D383000838
:1080D000D3830008D3830008D3830008D383000828
:1080E00081BC0008D3830008D3830008D383000831
:1080F000E1DD0008D383000801DE0008C1CC0008E0
:10810000D3830008D383000821D60008D383000856
:10811000B1DF0008D3830008D3830008D3830008AD
:1081200001CD000831CD000871CD0008B1CD0008A7
:10813000F1CD0008D3830008D383000801C80008EC
:1081400021C8000841C8000861C80008D38300089E
:1081500021CE000861CE0008A1CE0008D38300081C
:10816000D3830008D3830008D3830008D383000897
:10817000D3830008D3830008D3830008D383000887
:10818000D3830008D3830008D3830008D383000877
:10819000D3830008D3830008D3830008D383000867
:1081A000D3830008D3830008D3830008D383000857
:1081B000D3830008D3830008D3830008D383000847
:1081C000D3830008D3830008D3830008D383000837
:1081D000D3830008D3830008D3830008D383000827
:1081E000812A0108713001089140010821440108E9
:1081F000E14A01081155010831810108D19A0108AD
:10820000019C0108619F0108B1A4010801AF0108A8
:1082100011C70108A1CF0108D1F2010831FD010801
:108220005114020811210208F15B0208015F0208E3
:10823000216102081165020811710208717B0208B0
:10824000518B0208919602088198020831A5020814
:10825000A1B7020801BD0208A1D70208C1DB0208CC
:1082600031E9020891F7020801F80208511E0308DB
:1082700011230308F12B030811330308C14103083C
:10828000B147030891520308C1530308115603086C
:1082900011590308A1620308618D030821A3030893
:0882A000F1BF0308E1C103086E
:1082B00072B6394880F30888384880F3098838480E
:1082C0004EF60851CEF20001086040F20000CCF2F8
:1082D00000004EF63471CEF200010860BFF34F8FFC
:1082E000BFF36F8F40F20000C0F2F0004EF68851ED
:1082F000CEF200010860BFF34F8FBFF36F8F4FF0D6
:108300000000E1EE100A4EF63C71CEF2000108606A
:10831000062080F31488BFF36F8F01F071FB06F025
:1083200007F84FF055301F491B4A91423CBF41F8B6
:10833000040BFAE71C49194A91423CBF41F8040B6F
:10834000FAE71A491A4A1B4B9A423EBF51F8040BEE
:1083500042F8040BF8E700201749184A91423CBF45
:1083600041F8040BFAE701F063FB01F051FB144CF8
:10837000144DAC4203DA54F8041B8847F9E733F094
:1083800037FF114C114DAC4203DA54F8041B8847F7
:10839000F9E701F045BB00000010002000160020A6
:1083A000008000080000002000100020F00E0508EA
:1083B000001600207C2200208022002018B8012016
:1083C000E0810008A8820008A8820008A8820008AE
:1083D0006EE700F000F8FEE72DE9F04F2DED108A72
:1083E000C1F80CD0C3689D46BDEC108ABDE8F08F83
:1083F00001F00EFC002383F311882846A0470020DB
:1084000001F05EFF01F0F4FB01F01AFE01F000FC48
:1084100000DFFEE781F0004102E000BF83F000438F
:1084200030B54FEA41044FEA430594EA050F08BF0F
:1084300090EA020F1FBF54EA000C55EA020C7FEAD3
:10844000645C7FEA655C00F0E2804FEA5454D4EB50
:108450005555B8BF6D420CDD2C4480EA020281EA1A
:10846000030382EA000083EA010180EA020281EA52
:108470000303362D88BF30BD11F0004F4FEA0131A4
:108480004FF4801C4CEA113102D0404261EB4101B3
:1084900013F0004F4FEA03334CEA133302D0524239
:1084A00063EB430394EA050F00F0A780A4F10104F5
:1084B000D5F1200E0DDB02FA0EFC22FA05F280182F
:1084C00041F1000103FA0EF2801843FA05F3594115
:1084D0000EE0A5F120050EF1200E012A03FA0EFC94
:1084E00028BF4CF0020C43FA05F3C01851EBE371BE
:1084F00001F0004507D54FF0000EDCF1000C7EEBDB
:1085000000006EEB0101B1F5801F1BD3B1F5001F18
:108510000CD349085FEA30004FEA3C0C04F1010437
:108520004FEA445212F5800F80F09A80BCF1004F60
:1085300008BF5FEA500C50F1000041EB045141EAE2
:10854000050130BD5FEA4C0C404141EB010111F4E3
:10855000801FA4F10104E9D191F0000F04BF01468E
:108560000020B1FA81F308BF2033A3F10B03B3F16C
:1085700020020CDA0C3208DD02F1140CC2F10C02FC
:1085800001FA0CF021FA02F10CE002F11402D8BF5A
:10859000C2F1200C01FA02F120FA0CFCDCBF41EA26
:1085A0000C019040E41AA2BF01EB0451294330BDF5
:1085B0006FEA04041F3C1CDA0C340EDC04F11404D2
:1085C000C4F1200220FA04F001FA02F340EA0300A9
:1085D00021FA04F345EA030130BDC4F10C04C4F1EF
:1085E000200220FA02F001FA04F340EA03002946CF
:1085F00030BD21FA04F0294630BD94F0000F83F419
:10860000801306BF81F480110134013D4EE77FEAFB
:10861000645C18BF7FEA655C29D094EA050F08BF47
:1086200090EA020F05D054EA000C04BF1946104628
:1086300030BD91EA030F1EBF0021002030BD5FEA6C
:10864000545C05D14000494128BF41F0004130BD94
:1086500014F580043CBF01F5801130BD01F00045E8
:1086600045F0FE4141F470014FF0000030BD7FEA5B
:10867000645C1ABF194610467FEA655C1CBF0B4656
:10868000024650EA013406BF52EA033591EA030F6D
:1086900041F4002130BD00BF90F0000F04BF002165
:1086A000704730B54FF4806404F132044FF0000598
:1086B0004FF0000150E700BF90F0000F04BF002111
:1086C000704730B54FF4806404F1320410F0004577
:1086D00048BF40424FF000013EE700BF42004FEA72
:1086E000E2014FEA31014FEA02701FBF12F07F43EF
:1086F00093F07F4F81F06051704732F07F4208BFA6
:10870000704793F07F4F04BF41F40021704730B5AC
:108710004FF4607401F0004521F000411CE700BFF8
:1087200050EA010208BF704730B54FF000050AE07B
:1087300050EA010208BF704730B511F0004502D57C
:10874000404261EB41014FF4806404F132045FEA7E
:10875000915C3FF4D8AE4FF003025FEADC0C18BF27
:1087600003325FEADC0C18BF033202EBDC02C2F119
:10877000200300FA03FC20FA02F001FA03FE40EAAB
:108780000E0021FA02F11444BDE600BF70B54FF0AF
:10879000FF0C4CF4E06C1CEA11541DBF1CEA13558D
:1087A00094EA0C0F95EA0C0F00F0DEF82C4481EAF5
:1087B000030621EA4C5123EA4C5350EA013518BF15
:1087C00052EA033541F4801143F4801338D0A0FB02
:1087D00002CE4FF00005E1FB02E506F00042E0FBAF
:1087E00003E54FF00006E1FB03569CF0000F18BFB5
:1087F0004EF0010EA4F1FF04B6F5007F64F540745D
:1088000004D25FEA4E0E6D4146EB060642EAC621EF
:1088100041EA55514FEAC52040EA5E504FEACE2E5C
:10882000B4F1FD0C88BFBCF5E06F1ED8BEF1004F5F
:1088300008BF5FEA500E50F1000041EB045170BDDB
:1088400006F0004646EA010140EA020081EA03011F
:10885000B4EB5C04C2BFD4EB0C0541EA045170BD1B
:1088600041F480114FF0000E013C00F3AB8014F195
:10887000360FDEBF002001F0004170BDC4F10004DE
:10888000203C35DA0C341BDC04F11404C4F120055F
:1088900000FA05F320FA04F001FA05F240EA0200BA
:1088A00001F0004221F0004110EBD37021FA04F6F0
:1088B00042EB06015EEA430E08BF20EAD37070BDAA
:1088C000C4F10C04C4F1200500FA04F320FA05F009
:1088D00001FA04F240EA020001F0004110EBD3700B
:1088E00041F100015EEA430E08BF20EAD37070BD7B
:1088F000C4F1200500FA05F24EEA020E20FA04F354
:1089000001FA05F243EA020321FA04F001F0004102
:1089100021FA04F220EA020000EBD3705EEA430E73
:1089200008BF20EAD37070BD94F0000F0FD101F0A2
:108930000046400041EB010111F4801F08BF013CDB
:10894000F7D041EA060195F0000F18BF704703F019
:108950000046520043EB030313F4801F08BF013DA0
:10896000F7D043EA0603704794EA0C0F0CEA13555C
:1089700018BF95EA0C0F0CD050EA410618BF52EA16
:108980004306D1D181EA030101F000414FF000001C
:1089900070BD50EA410606BF1046194652EA43062A
:1089A00019D094EA0C0F02D150EA013613D195EA9E
:1089B0000C0F05D152EA03361CBF104619460AD1E6
:1089C00081EA030101F0004141F0FE4141F47001F0
:1089D0004FF0000070BD41F0FE4141F4780170BDE0
:1089E00070B54FF0FF0C4CF4E06C1CEA11541DBF45
:1089F0001CEA135594EA0C0F95EA0C0F00F0A7F847
:108A0000A4EB050481EA030E52EA03354FEA013173
:108A100000F088804FEA03334FF0805545EA131386
:108A200043EA12634FEA022245EA111545EA10654E
:108A30004FEA00260EF000419D4208BF964244F1E5
:108A4000FD0404F5407402D25B084FEA3202B61A04
:108A500065EB03055B084FEA32024FF480104FF4D8
:108A6000002CB6EB020E75EB030E22BFB61A75464C
:108A700040EA0C005B084FEA3202B6EB020E75EBDF
:108A8000030E22BFB61A754640EA5C005B084FEA47
:108A90003202B6EB020E75EB030E22BFB61A754614
:108AA00040EA9C005B084FEA3202B6EB020E75EB1F
:108AB000030E22BFB61A754640EADC0055EA060EE0
:108AC00018D04FEA051545EA16754FEA06164FEA23
:108AD000C30343EA52734FEAC2025FEA1C1CC0D1CF
:108AE00011F4801F0BD141EA00014FF000004FF05C
:108AF000004CB6E711F4801F04BF01430020B4F11D
:108B0000FD0C88BFBCF5E06F3FF6AFAEB5EB030CD4
:108B100004BFB6EB020C5FEA500C50F1000041EBD1
:108B2000045170BD0EF0004E4EEA113114EB5C049E
:108B3000C2BFD4EB0C0541EA045170BD41F4801171
:108B40004FF0000E013C90E645EA060E8DE60CEA79
:108B5000135594EA0C0F08BF95EA0C0F3FF43BAF96
:108B600094EA0C0F0AD150EA01347FF434AF95EA4D
:108B70000C0F7FF425AF104619462CE795EA0C0F31
:108B800006D152EA03353FF4FDAE1046194622E7FE
:108B900050EA410618BF52EA43067FF4C5AE50EAD8
:108BA00041047FF40DAF52EA43057FF4EBAE12E7C8
:108BB0004FF0FF3C06E000BF4FF0010C02E000BFA9
:108BC0004FF0010C4DF804CD4FEA410C7FEA6C5C8C
:108BD0004FEA430C18BF7FEA6C5C1BD001B050EA2F
:108BE000410C0CBF52EA430C91EA030F02BF90EA1A
:108BF000020F0020704710F1000F91EA030F58BFD9
:108C0000994208BF90422CBFD8176FEAE37040F03A
:108C1000010070474FEA410C7FEA6C5C02D150EAD8
:108C2000013C07D14FEA430C7FEA6C5CD6D152EA93
:108C3000033CD3D05DF8040B704700BF8446104658
:108C400062468C461946634600E000BF01B5FFF757
:108C5000B7FF002848BF10F1000F01BD4DF808ED27
:108C6000FFF7F4FF0CBF012000205DF808FB00BFF8
:108C70004DF808EDFFF7EAFF34BF012000205DF852
:108C800008FB00BF4DF808EDFFF7E0FF94BF01209F
:108C900000205DF808FB00BF4DF808EDFFF7CEFFA0
:108CA00094BF012000205DF808FB00BF4DF808EDDF
:108CB000FFF7C4FF34BF012000205DF808FB00BFB0
:108CC0004FEA410C7FEA6C5C02D150EA013C0AD1C8
:108CD0004FEA430C7FEA6C5C02D152EA033C02D1BA
:108CE0004FF0000070474FF0010070474FEA41021B
:108CF00012F5001215D211D56FF47873B3EB6252EE
:108D000012D94FEAC12343F0004343EA505311F014
:108D1000004F23FA02F018BF404270474FF00000A6
:108D2000704750EA013005D111F0004008BF6FF0E4
:108D3000004070474FF00000704700BF4FEA41020B
:108D4000B2F1E04324BFB3F5001CDCF1FE5C0DD9A9
:108D500001F0004C4FEAC0024CEA5070B2F1004FF3
:108D600040EB830008BF20F00100704711F0804FF6
:108D700021D113F13872BCBF01F00040704741F4BB
:108D800080114FEA5252C2F11802C2F1200C10FABF
:108D90000CF320FA02F018BF40F001004FEAC123A3
:108DA0004FEAD32303FA0CFC40EA0C0023FA02F347
:108DB0004FEA4303CCE77FEA625307D150EA01331D
:108DC0001EBF4FF0FE4040F44000704701F00040ED
:108DD00040F0FE4040F40000704700BF80F00040CB
:108DE00002E000BF81F0004142001FBF5FEA410383
:108DF00092EA030F7FEA226C7FEA236C6AD04FEA83
:108E00001262D2EB1363C1BFD218414048404140C7
:108E1000B8BF5B42192B88BF704710F0004F40F479
:108E2000000020F07F4018BF404211F0004F41F495
:108E3000000121F07F4118BF494292EA030F3FD061
:108E4000A2F1010241FA03FC10EB0C00C3F1200374
:108E500001FA03F100F0004302D5494260EB400003
:108E6000B0F5000F13D3B0F1807F06D340084FEA6E
:108E7000310102F10102FE2A51D2B1F1004F40EB63
:108E8000C25008BF20F0010040EA030070474900CB
:108E900040EB000010F4000FA2F10102EDD1B0FA96
:108EA00080FCACF1080CB2EB0C0200FA0CF0AABF8B
:108EB00000EBC25052421843BCBFD0401843704729
:108EC00092F0000F81F4000106BF80F4000001322F
:108ED000013BB5E74FEA41037FEA226C18BF7FEA06
:108EE000236C21D092EA030F04D092F0000F08BF48
:108EF0000846704790EA010F1CBF0020704712F02F
:108F00007F4F04D1400028BF40F00040704712F16D
:108F100000723CBF00F50000704700F0004343F0D2
:108F2000FE4040F4000070477FEA226216BF084608
:108F30007FEA23630146420206BF5FEA412390EACB
:108F4000010F40F4800070474FF0000304E000BFC1
:108F500010F0004348BF40425FEA000C08BF704772
:108F600043F0964301464FF000001CE050EA010236
:108F700008BF70474FF000030AE000BF50EA01024B
:108F800008BF704711F0004302D5404261EB410138
:108F90005FEA010C02BF84460146002043F0B6435D
:108FA00008BFA3F18053A3F50003BCFA8CF2083A82
:108FB000A3EBC25310DB01FA02FC634400FA02FC8B
:108FC000C2F12002BCF1004F20FA02F243EB020092
:108FD00008BF20F00100704702F1200201FA02FCF4
:108FE000C2F1200250EA4C0021FA02F243EB0200E7
:108FF00008BF20EADC7070477BB972B90029BEBF98
:1090000000204FF0004106E008BF00281CBF6FF0B1
:1090100000414FF0FF3000F0F3B9ADF1080C6DE9FD
:1090200004CE002909DB002B1ADB00F083F8DDF801
:1090300004E0DDE9022304B07047404261EB4101E6
:10904000002B1BDB00F076F8DDF804E0DDE90223FD
:1090500004B0404261EB4101524263EB430370476D
:10906000524263EB430300F065F8DDF804E0DDE90C
:10907000022304B0404261EB41017047524263EB6E
:10908000430300F057F8DDF804E0DDE9022304B003
:10909000524263EB4303704753B94AB9002908BFF2
:1090A00000281CBF4FF0FF314FF0FF3000F0A8B98F
:1090B000ADF1080C6DE904CE00F03CF8DDF804E0F9
:1090C000DDE9022304B0704707EE900AF5EEC07A9E
:1090D000F1EE10FA01D400F009B808B580F00040B4
:1090E00000F004F8404261EB410108BDD0B5FFF744
:1090F000F5FA00220D4B06460F46FFF747FB00F03E
:1091000081F90446FFF7C8FA0022094BFFF73EFB3E
:1091100002460B4630463946FFF780F900F072F9F7
:109120000022234610431946D0BD00BF0000F03D89
:109130000000F0412DE9F047089E04468846002BC8
:109140004BD18A42154667D9B2FA82F24AB1C2F1CE
:10915000200701FA02F320FA07F7954047EA0308CF
:1091600094404FEA154E230CB8FBFEF71FFA85FC1E
:109170000EFB178843EA084307FB0CF1994209D913
:10918000EB1807F1FF3080F01B81994240F2188103
:10919000023F2B445B1AA4B2B3FBFEF00EFB10336C
:1091A00044EA034400FB0CFCA44509D92C1900F146
:1091B000FF3380F00781A44540F2048102382C443B
:1091C00040EA0740A4EB0C0400271EB1D440002362
:1091D000C6E900433946BDE8F0878B4209D9002E25
:1091E00000F0EB800027C6E9000138463946BDE8AB
:1091F000F087B3FA83F7002F47D18B4202D3824224
:1092000000F2FA80841A61EB030301209846002ED5
:10921000E0D0C6E90048DDE702B9FFDEB2FA82F22B
:10922000002A40F08F80491B4FEA154E1FFA85F83F
:109230000127B1FBFEFC230C0EFB1C1143EA01438A
:1092400008FB0CF1994207D9EB180CF1FF3002D260
:10925000994200F2CD808446591AA3B2B1FBFEF0C8
:109260000EFB101443EA044408FB00F8A04507D99C
:109270002C1900F1FF3302D2A04500F2B680184647
:10928000A4EB080440EA0C409FE7C7F1200CBB4068
:1092900022FA0CFE4EEA030E01FA07F420FA0CF54E
:1092A00021FA0CF34FEA1E482543B3FBF8F92C0CC6
:1092B00008FB19331FFA8EFA44EA034309FB0AF448
:1092C0009C4202FA07F200FA07F10BD91EEB0303E6
:1092D00009F1FF3080F087809C4240F28480A9F140
:1092E000020973441B1BADB2B3FBF8F008FB10334B
:1092F00045EA034400FB0AFAA24508D91EEB040420
:1093000000F1FF336BD2A24569D90238744440EAB8
:109310000940A0FB0289A4EB0A044C45C2464B4617
:1093200054D351D0002E69D0B1EB0A0564EB03048D
:1093300004FA0CFCFD40FC404CEA0505C6E900546B
:10934000002747E7C2F1200320FA03F7954001FA0E
:1093500002F021FA03F34FEA154E3843010CB3FB38
:10936000FEF71FFA85F80EFB173341EA034107FBAE
:1093700008F38B4204FA02F407D9691807F1FF3C9D
:109380002FD28B422DD9023F2944CB1A81B2B3FB95
:10939000FEF00EFB103341EA034100FB08F38B4261
:1093A00007D9691800F1FF3C17D28B4215D9023852
:1093B0002944C91A40EA07473BE73746304609E7E0
:1093C0000746E7E61846FBE64145ABD2B8EB020A92
:1093D00069EB0E0201381346A4E76046E9E7184638
:1093E00095E76746D1E781467CE702382C4447E79A
:1093F000ACF1020C2B442FE7384608E73746E9E684
:10940000704700BF4A0011D212F5001211D20DD5DB
:109410006FF47873B3EB62520ED44FEAC12343F07A
:10942000004343EA505323FA02F070474FF0000024
:10943000704750EA013002D14FF0FF3070474FF0D3
:1094400000007047844641EA000313F003036DD126
:10945000403A41D351F8043B40F8043B51F8043BF7
:1094600040F8043B51F8043B40F8043B51F8043BFE
:1094700040F8043B51F8043B40F8043B51F8043BEE
:1094800040F8043B51F8043B40F8043B51F8043BDE
:1094900040F8043B51F8043B40F8043B51F8043BCE
:1094A00040F8043B51F8043B40F8043B51F8043BBE
:1094B00040F8043B51F8043B40F8043B51F8043BAE
:1094C00040F8043B51F8043B40F8043B51F8043B9E
:1094D00040F8043B403ABDD2303211D351F8043B3E
:1094E00040F8043B51F8043B40F8043B51F8043B7E
:1094F00040F8043B51F8043B40F8043B103AEDD2ED
:109500000C3205D351F8043B40F8043B043AF9D23D
:10951000043208D0D2071CBF11F8013B00F8013B10
:1095200001D30B8803806046704700BF082A13D31D
:109530008B078DD010F003038AD0C3F10403D21A35
:10954000DB071CBF11F8013B00F8013B80D331F869
:10955000023B20F8023B7BE7043AD9D3013A11F8E9
:10956000013B00F8013BF9D20B7803704B78437054
:109570008B78837060467047000000000000000098
:10958000A2EB0300704700BF02780B78012A28BFC6
:109590009A42F5D16DE9044540EA0104CDE902673C
:1095A0006FF0000C4FEA447212B380EA010414F029
:1095B000070F6AD100F0070420F0070004F003054C
:1095C00021F007014FEAC505F0E8042314F0040F69
:1095D000F1E804670CFA05F462EA040266EA04069C
:1095E0000AD063EA0403624667EA0407664603E0BA
:1095F000F0E80423F1E8046782FA4CF582EA0604F5
:10960000A4FA8CF46CBB83FA4CF583EA0705A5FA3F
:109610008CF595B950E9022351E9026782FA4CF5BD
:1096200082EA0604A4FA8CF483FA4CF583EA07056F
:10963000A5FA8CF52543DBD09CB92DBAB5FA85F493
:1096400024F0070427FA04F1DDE9026723FA04F3A2
:1096500003F0FF0001F0FF01FDE80445A0EB01006D
:10966000704724BAB4FA84F424F0070426FA04F10B
:10967000DDE9026722FA04F202F0FF0001F0FF01C7
:10968000FDE80445A0EB0100704714F0030F3CD146
:1096900010F0030428D150F8082B51F8083B82FA47
:1096A0004CF582EA0305A5FA8CF55DB950F8042C57
:1096B00051F8043C82FA4CF582EA0305A5FA8CF5D0
:1096C000002DE8D02DBAB5FA85F424F0070423FA6A
:1096D00004F122FA04F202F0FF0001F0FF01FDE8BC
:1096E0000445A0EB010070474FEAC40420F00300DA
:1096F00050F8082B21F0030151F8083B0CFA04F450
:1097000062EA040263EA0403C9E710F003041AD012
:10971000A1EB040120F00300E40750F8042B06D06D
:109720000FD28B785FFAA2F4E41A06D12BB1CB7872
:109730005FFAB2F4E41A00D11BB920465DF8104B71
:10974000704701F1040150F8042BCC0721F003010C
:1097500051F8043B48D824D222F07F4482FA4CF5D9
:1097600094EA1325A5FA8CF50AD165B951F8043BA2
:1097700084EA0204B4EB036F0ED150F8042BEBE73C
:109780004FEA132355E035F07F454DD10878FDE8C9
:109790000445C0F1000070474FEA126203F0FF0376
:1097A00047E002EA1C4482FA4CF594EA1345A5FA14
:1097B0008CF50AD165B951F8043B84EA0204B4EB94
:1097C000034F0CD150F8042BEBE74FEA134330E082
:1097D00015EA1C4528D10B884FEA124229E04FEACE
:1097E000124203EA1C4324E002F0FF0482FA4CF523
:1097F00094EA1365A5FA8CF50AD165B951F8043BD2
:1098000084EA0204B4EB032F09D150F8042BEBE7F0
:109810004FEA13630DE015F0FF0F05D10B684FEA17
:10982000122223F07F4304E04FF00000FDE80445DE
:10983000704712BA1BBA82FA4CF482EA0304A4FA03
:109840008CF5B5FA85F402FA04F203FA04F34FEA50
:109850001260FDE80445A0EB1360704700000000B3
:1098600000000000000000000000000000000000F8
:1098700000000000000000000000000000000000E8
:1098800090F800F06DE9024520F007016FF0000C40
:1098900010F0070491F820F040F049804FF00004E8
:1098A0006FF00700D1E9002391F840F000F10800C3
:1098B00082FA4CF2A4FA8CF283FA4CF3A2FA8CF3FB
:1098C0004BBBD1E9022382FA4CF200F10800A4FA62
:1098D0008CF283FA4CF3A2FA8CF3E3B9D1E90423B6
:1098E00082FA4CF200F10800A4FA8CF283FA4CF3ED
:1098F000A2FA8CF37BB9D1E9062301F1200182FAA7
:109900004CF200F10800A4FA8CF283FA4CF3A2FAAC
:109910008CF3002BC6D0002A04BF04301A4612BABA
:10992000B2FA82F2FDE8024500EBD2007047D1E9BD
:10993000002304F00305C4F100004FEAC50514F04C
:10994000040F91F840F00CFA05F562EA05021CBF1D
:1099500063EA050362464FF00004A9E70000000037
:1099600001F0FF01102A2BDB10F0070F08D010F8D0
:10997000013B013A8B422DD010F0070F42B3F6D1D4
:10998000F0B441EA012141EA014122F007047FF0ED
:1099900000070023F0E80256083C85EA010586EA44
:1099A000010685FA47F5A3FA87F586FA47F6A5FA80
:1099B00087F68EB9EED1F0BC01F0FF0102F007028C
:1099C00032B110F8013B013A83EA010313B1F8D137
:1099D0000020704701387047002D06BF3546033818
:1099E000073815F0010F07D1013015F4807F02BF51
:1099F000013015F4C03F0130F0BC0138704700BFA2
:109A0000704700BF000000000000000000000000E0
:109A1000704700BF000000000000000000000000D0
:109A2000FEE700BF00000000000000000000000092
:109A3000F0B4144E144D154C154B164906F1700C2C
:109A400000279C4211D904391A4651F8040F42F8F4
:109A5000040B9442F9D8DA43144424F00304043488
:109A600023449D4203D943F8047B9D42FBD86645BD
:109A700005D0D6E90413D6E906451036E1E7F0BC77
:109A8000704700BF5014040818B8012018B801200E
:109A900018B801206C1B0508000000000000000041
:109AA000FEE700BF00000000000000000000000012
:109AB000F8B51C4C1C4F1D4E002500F091F900F02C
:109AC0003FF9C4E90C5500F023FD00F049FE00F019
:109AD0008FFE04F138008022154900F0F1FA154B91
:109AE00001220277D968144AA0614FF6FF000140B5
:109AF0000A43DA60FA6842F08072FA603268102035
:109B000042F0010220213260D87783F8221000F061
:109B10005FF885F3118862B60848BDE8F84000F0A8
:109B20002FBB00BF902A0020F0ED00E0001000E005
:109B30005415040800ED00E00003FA05EC140408D5
:109B400008B572B6034B0449D862D12228F058FFF9
:109B5000FEE700BF902A0020D01404080000000097
:109B60002DE9F843164D00F0CBF8AA69D37F0BB16D
:109B7000013BD37700F0C4F8124FAB6AEC690133B4
:109B8000BC42AB6219D0A668013EA660AEB94FF0E8
:109B900020092368D4F80C80E6605F60EB6100F078
:109BA00067F886F311882069C04789F3118800F0AF
:109BB00047F8EC69A368002BEBD0BDE8F88300BF41
:109BC000902A0020AC2A00200000000000000000C5
:109BD000044B1A6B0AB95B6B13B10348FFF7B0BFB4
:109BE000704700BF902A0020041504080000000000
:109BF00010B5054C236B0BB9636B13B10348FFF72A
:109C00009FFF0123636310BD902A00201C150408E8
:109C100010B5074C236B2BB9636B002B02DD0023BF
:109C2000636310BD0348FFF78BFF0023636310BD20
:109C3000902A00202C1504080000000000000000FD
:109C400010B5064C236B002B01DD636B13B1044888
:109C5000FFF776FF0123636310BD00BF902A002049
:109C600024150408000000000000000000000000AF
:109C700010B5084C236B002B05DD636B002B02DD58
:109C80000023636310BD0448FFF75AFF002363639A
:109C900010BD00BF902A0020341504080000000009
:109CA00010B5202383F31188074C236B002B01DBB5
:109CB000626B1AB10548FFF743FF236B013323633F
:109CC000002383F3118810BD902A00200C1504088E
:109CD00010B5202383F31188074C236B002B01DD83
:109CE000626B1AB10548FFF72BFF236B013B23631F
:109CF000002383F3118810BD902A00201415040856
:109D0000054B1A6B002A03DB5B6B002B00DD7047F1
:109D10000248FFF715BF00BF902A00203C15040839
:109D2000044B1A6B1AB95B6B002B00DD70470248BD
:109D3000FFF706BF902A0020441504080000000029
:109D4000054B4FF0FF30002103F11C02586299626D
:109D5000C3E90722704700BF902A002000000000DE
:109D6000F8B5054616461F460C46FFF7C9FF0C48D6
:109D70002F61C369EE609A68944204D91B68A41AE3
:109D80009A68A242FAD35A68C5E9003215605D604C
:109D9000AC6099684FF0FF32091B99604262F8BDD0
:109DA000902A0020000000000000000000000000D9
:109DB00038B50446FFF7A4FF2368A5689A68616870
:109DC00005482A449A600B60256800224FF0FF3353
:109DD0006960E260436238BD902A00200000000004
:109DE000034B0022C3E90033C3E904339A60704790
:109DF000902A002000000000000000000000000089
:109E000010B50446FFF77CFF0022A168064B2277BD
:109E10001B689A688A42FBD25A682046C4E900321D
:109E200014605C6010BD00BF902A0020000000009C
:109E300038B50446202383F31188FFF701FF237F01
:109E4000072B10D8DFE803F0150F0F1B0A040F0AC9
:109E5000256AFFF755FFAB680133AB60D4E90023F7
:109E60001A60226853604FF0FF3323622046FFF7E9
:109E7000C7FFFFF7FDFE002383F3118838BD236A77
:109E800000221A604FF0FF3323622046FFF7B8FF2D
:109E9000EFE700BF0000000000000000000000002D
:109EA00070B50A4CA5690646FFF73AFF23682E777E
:109EB0001422EA771A682260012654601E77294628
:109EC000A3611846BDE87040FEF786BA902A0020CC
:109ED00070B50D4686B00646FFF722FF6B1C14D006
:109EE0000E4C0F4AA369294601A8FFF739FF3046F7
:109EF000FFF7D6FFFFF704FF049B13B101A8FFF79C
:109F000057FFA369186A06B070BD044C3046FFF7CE
:109F1000C7FFA369186A06B070BD00BF902A002071
:109F2000319E00080000000000000000000000005A
:109F3000F8B5144E0546B4690F46FFF7F1FEA36865
:109F4000AA682F629A4217D9FFF7DAFE0023A168A8
:109F5000237733461B689A688A42FBD25A6862604C
:109F60000120236014605C60287721462846B56193
:109F7000BDE8F840FEF730BA2846BDE8F840FFF7E4
:109F80003FBF00BF902A002000000000000000003A
:109F9000084A93691168DA7F88689B6822B99842F9
:109FA00034BF002001207047984294BF0020012058
:109FB000704700BF902A0020000000000000000051
:109FC00038B50F4C2368A5691A68226001215460D6
:109FD0001977A361FFF794FE0023A9682B77234626
:109FE0001B689A688A42FBD85A68A0692B606A602D
:109FF000294615605D60BDE83840FEF7EDB900BF49
:10A00000902A002000000000000000000000000076
:10A0100008B5FFF785FEFFF773FE064B1A689B69CC
:10A0200092689B689A4200D808BDBDE80840FFF7D7
:10A03000C7BF00BF902A0020000000000000000001
:10A0400070B51B4D2B68AC691A682A605560DE7FBD
:10A05000AB6101221A77AEB9FFF752FEA1682677ED
:10A060002B461B689A688A42FBD25A6862601421A8
:10A07000236014605C60E177A8692146BDE8704008
:10A08000FEF7AAB9FFF73CFE0023A16823772B4611
:10A090001B689A688A42FBD85A68A869C4E90032EA
:10A0A000214614605C60BDE87040FEF795B900BFC2
:10A0B000902A0020000000000000000000000000C6
:10A0C000F0B40B4C0B4F656982638260002681619E
:10A0D00000F1280200F1240145610461C761C0E973
:10A0E0000C6628616061C0E90912C262F0BC704769
:10A0F000902A00200200011400000000000000006F
:10A1000070B50446FFF7FCFDD4E90416A368256882
:10A11000E06843F86C1C022103F82C1C142103F89E
:10A12000291C012103F82A1C124A43F8686C0021FB
:10A1300003F82B1C546943F8400C43F8100C43F807
:10A14000305CA3F1AC000C4D43F83C0C43F84C5C84
:10A1500043E90611A3F14800A3F12001A3F124056E
:10A1600043E90E242061506143E9095143F81C1C66
:10A1700070BD00BF902A0020F1830008000000009D
:10A1800010B52023044683F31188FFF731FD2046E4
:10A19000FFF7B6FF00210446FFF7CAFEFFF738FDC0
:10A1A000002383F31188204610BD00BF000000008B
:10A1B0002DE9F843994604460D469046202383F343
:10A1C0001188483D2C44184E184FFFF711FD089B8D
:10A1D000716944F8203CA4F16402154BE260E3612C
:10A1E00004F1240204F128030025124844F8249CB9
:10A1F000C4E90461C4F8088044F8047CA061C4F890
:10A200003880C4E90C5520460C61C4E90923E36297
:10A2100029467461FFF78CFEFFF7FAFC85F311887D
:10A220002046BDE8F88300BF902A0020F183000893
:10A23000020001144C15040800000000000000009A
:10A2400010B52023044683F31188FFF7D1FCA37FC8
:10A25000013BA377E36903F0FF130F2B01BFD4E9A0
:10A2600004231A6122695361FFF7D2FC002383F3B0
:10A27000118810BD00000000000000000000000078
:10A2800038B50E4B9C69636A206204F12405AB4229
:10A2900007D01A6862621846FFF7B2FD636AAB42E4
:10A2A000F7D1A37F23B9D4E904231A61226953614A
:10A2B0000F20BDE83840FFF7F3BD00BF902A002013
:10A2C00010B52023044683F31188FFF791FC204644
:10A2D000BDE81040FFF7D4BF000000000000000000
:10A2E00038B50446202383F31188FFF781FC237FD0
:10A2F0000F2B07D0094B626A9B6909201A606362C1
:10A30000FFF7CEFD256AFFF783FC002383F3118856
:10A310002046FFF795FF284638BD00BF902A002051
:10A3200010B52023044683F31188FFF761FC637F97
:10A3300043F004036377FFF76BFC002383F311887A
:10A3400010BD00BF00000000000000000000000081
:10A3500010B52023044683F31188FFF749FC2146FA
:10A360000820FFF7B5FDFFF753FC002383F31188A6
:10A3700010BD00BF00000000000000000000000051
:10A3800038B504460D46202383F31188FFF730FCCF
:10A39000084B996A2B1B0C1BA34203D9691A08208E
:10A3A000FFF796FDFFF734FC002383F3118828465E
:10A3B00038BD00BF902A002000000000000000000F
:10A3C000054B02469B6921B1036003201A62FFF727
:10A3D0007FBD4FF0FF307047902A00200000000042
:10A3E00003682BB10022026018461962FFF708BD0E
:10A3F000704700BF000000000000000000000000E7
:10A4000038B504460D46202383F31188FFF7F0FB8F
:10A41000206820B1002329462360FFF789FDFFF75C
:10A42000F7FB002383F3118838BD00BF0000000054
:10A4300069B1084B10B4024644689B690420C3E923
:10A440000024236053605DF8044BFFF741BD4FF0DB
:10A45000FF307047902A002000000000000000003C
:10A46000026890420AD010B4146804600346636026
:10A47000104611625DF8044BFFF7C2BC704700BF85
:10A4800038B5036898420BD004460D461A6822601E
:10A49000184654601D62FFF7B3FC23689C42F5D157
:10A4A00038BD00BF000000000000000000000000F8
:10A4B000014B5B6883607047001000E00000000003
:10A4C0000E4B0F4A5B68C168F0B48468D66F42686F
:10A4D0001B1BD0E904459B1BE61845F1000793427E
:10A4E000026888BF436001319342C0E90467C0E954
:10A4F000023138BF0360F0BC704700BF001000E0BD
:10A50000902A002000000000000000000000000071
:10A5100010B50C4C86B000234FF0FF310022684686
:10A52000E367CDE9013303930023CDE904230091D0
:10A53000FFF7BEFF6846FFF7C3FF029BE36706B065
:10A5400010BD00BF902A00200000000000000000A5
:10A550000023C0E900008360704700BF00000000D6
:10A56000F8B50546364B9C69FFF7DAFBA86800286A
:10A570003DD0A26883689A4206D9037F8260062B89
:10A580003AD0072B15D043B32E462B4603E09968EB
:10A59000A268914229D31B689D42F8D173680620B6
:10A5A000C4E900631C6074602562BDE8F840FFF7F1
:10A5B00077BCD0E900131960066A01684B60334626
:10A5C00002E09968914231D31B689E42F9D17368C9
:10A5D000C0E9006318607060D6E7D0E900231A6014
:10A5E00002685360FFF70CFCCEE71E46D6E7636BAC
:10A5F000C5E902436563F8BDD0E900131960066A36
:10A60000016837464B60334602E09968914214D3A3
:10A610001B689E42F9D17B68A268C0E9007318608C
:10A620007860B06883689342A7D3ADE71E4673682D
:10A63000C0E9006318607060A6E71F46EBE700BF43
:10A64000902A002000000000000000000000000030
:10A6500010B52023044683F31188FFF7C9FA20467A
:10A66000FFF77EFFFFF7D4FA002383F3118810BDB4
:10A67000F8B51D4B05469F69202383F31188FFF72A
:10A68000B7FAEB687B63FFF74BFB2B689D4222D048
:10A69000D7E90D4664B1FFF743FB23689C4203D022
:10A6A0009B689E4238BF1E46E468002CF3D12B689D
:10A6B000596B1A68BE6018462A605560C5E90231B8
:10A6C0005D63FFF79DFBFFF7A3FCFFF7A1FA0023F3
:10A6D00083F31188F8BD0023AB60FFF799FA0023DC
:10A6E00083F31188F8BD00BF902A0020000000000D
:10A6F00038B504460D46FFF703FB216B237F294342
:10A700000A2B21630CD00B2B00D038BD236A8B435E
:10A71000FBD1002323622046BDE83840FFF770BB21
:10A72000236A1942F5D1F0E70000000000000000A4
:10A7300070B506460D46FFF7E3FA3468A6420DD021
:10A74000E3682B43E36015B123691D4203D0D4E9CC
:10A750000101FFF7CDFF2468A642F1D170BD00BF13
:10A76000034A044B02F50061C3E90021704700BFB2
:10A77000182B0020102B002000000000000000001B
:10A78000F8B50E4604461546FFF7BAFA094AD2E96B
:10A7900000737819013C3044714234440138084058
:10A7A000214001448B4203D38F4201D81160F8BD90
:10A7B0000020F8BD102B0020000000000000000069
:10A7C00070B5202304460D46164683F31188FFF723
:10A7D0000FFA324629462046FFF7D2FF0446FFF71C
:10A7E00017FA002383F31188204670BD0000000093
:10A7F000044B054A1A6003F10C000022C3E9012250
:10A80000FFF7A6BE18330020C1A700080000000013
:10A81000064A536823F001035360EFF3098368335A
:10A8200083F30988002383F31188704730EF00E039
:10A83000202383F31188124B5B6813F4006302D169
:10A8400083F31188704710B5F1EE103AEFF30984E5
:10A850000C4B4FF08072DB6844F8083C44F84C2CF9
:10A86000A4F1680383F30988FFF792FB18B1064B44
:10A8700044F8503C10BD054B44F8503C10BD00BF9F
:10A8800000ED00E030EF00E00584000810840008CF
:10A8900008B501F0C5FA02F0D3FB00F0F1F800F0C2
:10A8A00037F900F0E5F900F02BFA00F059FE00F05E
:10A8B0009FFE00F095FF00F0D3FC00F089FE03F04E
:10A8C000E7FDBDE8084000F083BF00BF00000000C6
:10A8D000F8B5154682680669AA420B46816938BFF9
:10A8E0008568761AB54204461DD30AD818462A460A
:10A8F000FEF7A8FDE368A361A3685B1BA36028467D
:10A90000F8BD32461846FEF79DFDAF1B3A4630446F
:10A91000E168FEF797FDA368E2685B1B3A44A26119
:10A92000A3602846F8BD18462A46FEF78BFDA369AA
:10A930002B44A361A3685B1BA3602846F8BD00BF3E
:10A9400030B4029C046200250A4485600261C0E9BB
:10A950000000C160C0E90511C36130BC704700BF91
:10A9600038B504460D46FFF7CBF9D4E905329342DA
:10A9700011D0A268591C0132A26061611D70D4E936
:10A9800004329A4201D3E368636120460021FFF755
:10A9900067FD002038BDA268002AEAD04FF0FF30E2
:10A9A00038BD00BF000000000000000000000000F3
:10A9B0002DE9F04F83B006460D46144601929B46A2
:10A9C000C7694FF0200888F31188FFF711F9C4B167
:10A9D0004FF00009224629463046FFF779FF8246AC
:10A9E000D0B1304607B1B847FFF712F989F31188A3
:10A9F000A4EB0A04554488F31188FFF7F9F8002CFA
:10AA0000E8D1DDF804A0FFF703F9002383F31188F0
:10AA1000504603B0BDE8F08F59463046FFF708FDB9
:10AA20000028D7D0019BA3EB040AECE7000000004C
:10AA3000C3689B0F0CD0012B08D18368C28818040F
:10AA400000F47C10104301308002704700207047F2
:10AA5000D0E9012340F6FC7000EA830040EA9270DE
:10AA6000C2F3C23202320130C3F303439040093BC8
:10AA70009840704700000000000000000000000047
:10AA800001F09EBA0000000000000000000000007D
:10AA9000002301220270C0E90133C0E9033343619E
:10AAA0001830FFF755BD00BF000000000000000097
:10AAB00038B504460D46202383F31188FFF798F834
:10AAC0002046656001F0ACFA02232370FFF7A0F87E
:10AAD000002383F3118838BD00000000000000004F
:10AAE000F8B504460D4617461E46FFF709F9032040
:10AAF0002070C4E9027625612046BDE8F84001F0E7
:10AB0000E7BA00BF000000000000000000000000E5
:10AB100001F0B6BE000000000000000000000000D0
:10AB200030B40021012400F1180200F11C0300F1EF
:10AB300020050470416000F1240400F128018261C5
:10AB4000C36100F1080200F11003C0E908548162FA
:10AB5000C0E90222C0E9043330BC704700000000A5
:10AB600038B504460D46202383F31188FFF740F8DB
:10AB7000022323702046656001F0C2FE0323237088
:10AB8000FFF746F8002383F3118838BD000000006A
:10AB90002DE9F0411F4682B004460D469046202321
:10ABA00083F31188FFF724F804F108062378042BB7
:10ABB0002946204602D001F0E3FE78B939463046F6
:10ABC000FFF736FC0028F1D00190FFF721F80023B1
:10ABD00083F31188019802B0BDE8F0812046424617
:10ABE000294601F0EDFEFFF713F8002080F31188ED
:10ABF00002B0BDE8F08100BF0000000000000000CE
:10AC00002DE9F0411F4682B004460D4690462023B0
:10AC100083F31188FEF7ECFF04F110062378042B70
:10AC20002946204602D001F003FF78B93946304664
:10AC3000FFF7FEFB0028F1D00190FEF7E9FF0023AB
:10AC400083F31188019802B0BDE8F08120464246A6
:10AC5000294601F00DFFFEF7DBFF002080F311888D
:10AC600002B0BDE8F08100BF00000000000000005D
:10AC700002F0F6BC00000000000000000000000030
:10AC80000122002302704360704700BF00000000F3
:10AC900038B504460D46202383F31188FEF7A8FF3C
:10ACA0002046656002F0ECFC02232370FEF7B0FF43
:10ACB000002383F3118838BD00000000000000006D
:10ACC00038B504460D46FFF71BF8042329462370C8
:10ACD0002046BDE8384002F013BD00BF0000000070
:10ACE00010B50446FFF70CF8022323702046BDE898
:10ACF000104002F01DBD00BF000000000000000079
:10AD000002F026BD0000000000000000000000006E
:10AD10000122002302704360704700BF0000000062
:10AD200038B504460D46202383F31188FEF760FFF3
:10AD30002046656002F03CFD02232370FEF768FFA9
:10AD4000002383F3118838BD0000000000000000DC
:10AD500038B50446202383F31188FEF749FF2046C7
:10AD600002F0EEFD0025012323706560FEF750FF21
:10AD700085F3118838BD00BF00000000000000000E
:10AD800010B52023044683F31188FEF731FF2046D7
:10AD900002F036FE03232370FEF73AFF002383F30D
:10ADA000118810BD0000000000000000000000003D
:10ADB00010B52023044683F31188FEF719FF2046BF
:10ADC00002F02EFE02232370FEF722FF002383F3FE
:10ADD000118810BD0000000000000000000000000D
:10ADE00010B52023044683F31188FEF701FF2046A7
:10ADF00002F01EFEFEF70CFF002383F3118810BD46
:10AE000010B52023044683F31188FEF7F1FE204697
:10AE100002F02EFEFEF7FCFE002383F3118810BD26
:10AE20000379052B01D001207047836A4B604FF4F2
:10AE300000730B600020704700000000000000005D
:10AE400030B5054683B009242B6801AA1868012192
:10AE500000F09EFC9DF80400FF2801D1013CF3D1D5
:10AE600003B030BD00000000000000000000000042
:10AE700030B5054683B0102401E0013C0DD02B68AD
:10AE800001AA1868012100F083FC9DF80430FF2B13
:10AE9000F3D103B030BDFFF75BFA2B6801AA186845
:10AEA000012100F075FC9DF80430FF2B4FF00100EC
:10AEB000F1D103B030BD00BF000000000000000071
:10AEC00070B5164682B005462C300C46FFF7D0FF11
:10AED000330A44F04001300E320C8DF80330002369
:10AEE000124C8DF800108DF801008DF802200DF144
:10AEF00005000DF1010281EA430190428DF80460E2
:10AF0000635C06D012F8011B81EA43019042635C46
:10AF1000F8D1590041F00101EB6A8DF8051018686D
:10AF20006A46062100F014FC02B070BD6C150408DE
:10AF3000F8B50D46C16A0446174608681E4600F07B
:10AF400097FB3A4629462046FFF7BAFF04F12C004A
:10AF5000FFF776FFE16A054632460868042100F0F3
:10AF600017FCE36A186800F09BFB2846F8BD00BF99
:10AF7000C36A70B504460D461868164600F078FBA3
:10AF8000294632462046FFF79BFF04F12C00FFF7CD
:10AF900057FFE36A0546186800F082FB284670BD3B
:10AFA00070B5C36A84B005460C461868164600F0B2
:10AFB0005FFB284621460022FFF782FF05F12C00A7
:10AFC000FFF73EFF58BB42F2107401E0013C2DD068
:10AFD000EB6A6A461868012100F0DAFB9DF8003040
:10AFE000FE2BF3D1EB6A6A461868102100F0D0FB03
:10AFF0006B4606F10C00321F53F8041B09BA40F8E7
:10B0000004198242F8D1EB6A0221186800F060FB53
:10B01000EB6A186800F044FB002004B070BDEB6AD6
:10B02000186800F03DFB012004B070BD0120F4E77A
:10B0300070B5C36A032202710546002280F83020F1
:10B0400082B0D3E9000100F0E3FAEB6A102118683E
:10B0500000F03EFB0A2401E0FFF77AF900221146D6
:10B060002846FFF785FF01284FF00A000AD0013C6F
:10B07000F2D1EB6A186800F0E3FA02232B71012089
:10B0800002B070BD01AB4FF4D57208212846FFF71E
:10B090004FFF052824D02E4E642405E0013C4FF0DC
:10B0A0000A00E6D0FFF754F9002237212846FFF7BF
:10B0B0005FFF0128F2D801AB324629212846FFF76D
:10B0C00037FF0028EAD101AB02463A212846FFF7B4
:10B0D0002FFF9DF804305B0644BF012385F8303014
:10B0E000642407E001284FF00A00C2D1013CC0D01F
:10B0F000FFF72EF9002201212846FFF739FF00282B
:10B10000F0D1EB6A9968186800F082FA4FF4007287
:10B1100010212846FFF72CFF0028AAD105F11804BA
:10B12000224609212846FFF73BFF0028A1D12046EF
:10B13000FFF77EFCA86200289BD005F108020A21D7
:10B140002846FFF72DFF002893D105232B7197E7A1
:10B15000AA01004000000000000000000000000004
:10B1600010B50368044682B0186800F081FA01E067
:10B17000FFF7EEF8236801AA1868012100F008FB28
:10B180009DF80430FF2B4FF00100F1D123681868BF
:10B1900000F086FA02B010BD0000000000000000C0
:10B1A00070B50579052D01D0012070BD0646082235
:10B1B00056F82C3F027104469968186800F028FA86
:10B1C0003046FFF7CDFF2571002070BD0000000064
:10B1D00038B50446202383F31188FEF709FD23794F
:10B1E000022B18D004232371FEF712FD002383F3F2
:10B1F0001188254655F82C3F9968186800F008FA20
:10B200002846FFF7ADFFE36A186800F019FA022339
:10B210002371002038BDFEF7FBFC002383F3118867
:10B22000002038BD00000000000000000000000009
:10B2300038B50546044655F82C3F084A18680721DA
:10B2400000F086FA2846FFF7FBFDE36A186800F075
:10B2500027FA05232371002038BD00BF9816040883
:10B26000704700BF00000000000000000000000068
:10B27000044B0360012200230271C36280F8303066
:10B28000704700BF6C1604080000000000000000BA
:10B290000223C1620371704700000000000000003B
:10B2A00010B5C36A0446186800F0CAF900220123E9
:10B2B000E262237110BD00BF00000000000000002A
:10B2C00038B5C36A0446062202710D4618689968AB
:10B2D00000F09EF9E36A186800F0CAF994F830307B
:10B2E00053B120462A461221FFF7EAFD04F12C0053
:10B2F000FFF7A6FD58B938BD20466A021221FFF7B4
:10B30000DFFD04F12C00FFF79BFD0028F3D0E36A7A
:10B31000186800F095F905232371012038BD00BF9E
:10B320000379062B01D00120704770B50D46064603
:10B3300042F2107401E0013C16D0F36A2A46186804
:10B34000012100F025FA2B78FE2BF4D1F36A2A466E
:10B3500018684FF4007100F01BFAF36A02211868B4
:10B3600000F0B6F9002070BDF36A186800F098F993
:10B37000F36A186800F064F905233371012070BD89
:10B3800070B514461D460646FFF79AFF18B935B941
:10B390003379062B0DD0012070BD013DF8D0214638
:10B3A0003046FFF7BDFF04F500740028F5D00120FA
:10B3B00070BD3046BDE87040FFF73ABF00000000A6
:10B3C0000379062B01D001207047FFF731BF00BF82
:10B3D00038B5C36A0446072202710D461868996899
:10B3E00000F016F9E36A186800F042F994F830307A
:10B3F00053B120462A461921FFF762FD04F12C00C3
:10B40000FFF71EFD58B938BD20466A021921FFF723
:10B4100057FD04F12C00FFF713FD0028F3D0E36A79
:10B42000186800F00DF905232371012038BD00BF15
:10B430000379072B01D00120704730B5C36A194A40
:10B44000044683B018680D46022100F081F9E36AD2
:10B450002A4618684FF4007100F07AF9E36A022175
:10B46000186800F035F9E36A01AA1868012100F0B4
:10B470008FF99DF8043003F01F03052B0CD0E36A0D
:10B48000186800F00DF9E36A186800F0D9F8052390
:10B490002371012003B030BD04F12C00FFF7E8FC5C
:10B4A0000020F7E7901604080000000000000000EC
:10B4B000F8B514461D460646FFF78AFF20B9074631
:10B4C0003DB93379072B0DD001273846F8BD013D32
:10B4D000F7D021463046FFF7ABFF04F50074002893
:10B4E000F5D0F1E7F36A064A1868022100F030F956
:10B4F000F36A186800F0D4F805233371E5E700BF5C
:10B500009416040800000000000000000000000085
:10B510000379072B01D001207047C36A074A10B591
:10B5200004460221186800F013F9E36A186800F075
:10B53000B7F805232371002010BD00BF941604083E
:10B54000034B00F00F0003EB0010C0E9021270473C
:10B550008034002000000000000000000000000017
:10B5600002F026BB00000000000000000000000008
:10B570000023012202704360C3600374704700BF60
:10B5800038B504460D46202383F31188FEF730FBBF
:10B590006B682046C4E9015302F02AFB0025022310
:10B5A0002370E560FEF734FB85F3118838BD00BFDA
:10B5B00010B52023044683F31188FEF719FB2046BB
:10B5C00002F0BEFBFEF724FB002383F3118810BDBD
:10B5D00001F0EEBD000000000000000000000000CF
:10B5E000704700BF000000000000000000000000E5
:10B5F00001F07EBE0000000000000000000000001E
:10B60000012200230270C0E901330C30FEF7A0BF15
:10B6100038B504460D46202383F31188FEF7E8FA77
:10B620002046656001F09CFE02232370FEF7F0FACD
:10B63000002383F3118838BD0000000000000000E3
:10B6400038B50446202383F31188FEF7D1FA20464B
:10B6500001F006FF0025012323706560FEF7D8FA8C
:10B6600085F3118838BD00BF000000000000000015
:10B6700010B52023044683F31188FEF7B9FA6268F7
:10B68000D2E9022101238B409BB25383FEF7C0FA1B
:10B69000002383F3118810BD0000000000000000AB
:10B6A00010B52023044683F31188FEF7A1FA6268DF
:10B6B000D2E9022101238B409BB21383FEF7A8FA43
:10B6C000002383F3118810BD00000000000000007B
:10B6D00038B504460D46202383F31188FEF788FA17
:10B6E000032323702946204601F0F2FE4FF0FF317C
:10B6F00004F10800FEF764FEFEF78AFA002383F3E4
:10B70000118838BD000000000000000000000000AB
:10B71000F8B51F4604460D461646202383F31188CC
:10B72000FEF766FA03203B46324629462070204643
:10B7300001F0EEFE4FF0FF3104F10800FEF740FE8D
:10B74000FEF766FA002383F31188F8BD00000000BD
:10B7500070B5202304460D46164683F31188FEF784
:10B7600047FA0323237032462946204601F0F0FEB3
:10B770004FF0FF3104F10800FEF722FEFEF748FA11
:10B78000002383F3118870BD00000000000000005A
:10B7900070B5202304460D46164683F31188FEF744
:10B7A00027FA0323237032462946204601F0F0FE93
:10B7B0004FF0FF3104F10800FEF702FEFEF728FA11
:10B7C000002383F3118870BD00000000000000001A
:10B7D00001F016BF000000000000000000000000A3
:10B7E00002F066BC00000000000000000000000045
:10B7F0000023012202704370837043600372C0E92A
:10B80000033370470000000000000000000000004B
:10B8100038B504460D46202383F31188FEF7E8F976
:10B820002046656002F05CFC02232370FEF7F0F90D
:10B83000002383F3118838BD0000000000000000E1
:10B8400038B50446202383F31188FEF7D1F920464A
:10B8500002F0EEFC00250123237065606570A57081
:10B86000FEF7D6F985F3118838BD00BF000000004F
:10B8700070B5202304460D46164683F31188FEF763
:10B88000B7F932462946204602F02AFD0123A3706B
:10B89000FEF7BEF9002383F3118870BD000000009D
:10B8A0002DE9F0411F4604460E469046202383F3BF
:10B8B00011880125FEF79CF9424625723168204621
:10B8C00002F0DEFC6570394604F11000FEF778FDE9
:10B8D000054638B9FEF79CF9002383F31188284602
:10B8E000BDE8F081FEF70CFA6378012B05D04FF02C
:10B8F000FF3033681B1A3360ECE7204602F0E0FCAF
:10B9000000236370F5E700BF0000000000000000A6
:10B91000430910B49B0000F1604404F5614403F155
:10B920006043090103F5614300F01F000122C9B221
:10B9300084F8001302FA00F0C3F880015DF8044BAC
:10B9400018607047000000000000000000000000C8
:10B950000849430910B4203300F01F0401220844B1
:10B96000A240002441F8232080F800435DF8044BF6
:10B97000704700BF00E100E0000000000000000090
:10B9800000F1604000F56D400901C9B201767047D1
:10B9900008B5FEF785F9104A516913680B4003F0AA
:10B9A0000103536193B10D4A93680BB1D068984776
:10B9B000202383F31188FEF743F900210748FEF79F
:10B9C0005FFDFEF755F9002383F31188FEF780F938
:10B9D000BDE80840FEF72CBF003C01408034002049
:10B9E00008B5FEF75DF9104A516913680B4003F082
:10B9F0000203536193B10D4A93690BB1D069984723
:10BA0000202383F31188FEF71BF900210848FEF775
:10BA100037FDFEF72DF9002383F31188FEF758F95F
:10BA2000BDE80840FEF704BF003C01408034002020
:10BA30009034002000000000000000000000000022
:10BA400008B5FEF72DF9104A516913680B4003F051
:10BA50000403536193B10D4A936A0BB1D06A9847BE
:10BA6000202383F31188FEF7EBF800210848FEF746
:10BA700007FDFEF7FDF8002383F31188FEF728F990
:10BA8000BDE80840FEF7D4BE003C014080340020F1
:10BA9000A0340020000000000000000000000000B2
:10BAA00008B5FEF7FDF8104A516913680B4003F022
:10BAB0000803536193B10D4A936B0BB1D06B984758
:10BAC000202383F31188FEF7BBF800210848FEF716
:10BAD000D7FCFEF7CDF8002383F31188FEF7F8F8C2
:10BAE000BDE80840FEF7A4BE003C014080340020C1
:10BAF000B034002000000000000000000000000042
:10BB000008B5FEF7CDF8104A516913680B4003F0F1
:10BB10001003536193B10D4A936C0BB1D06C9847ED
:10BB2000202383F31188FEF78BF800210848FEF7E5
:10BB3000A7FCFEF79DF8002383F31188FEF7C8F8F1
:10BB4000BDE80840FEF774BE003C01408034002090
:10BB5000C0340020000000000000000000000000D1
:10BB600010B5FEF79DF83D4B5A691C68144004F46B
:10BB700078725A61A30612D5394A936D0BB1D06D14
:10BB80009847202383F31188FEF75AF8002135489F
:10BB9000FEF776FCFEF76CF8002383F3118860064D
:10BBA00012D52F4A936E0BB1D06E9847202383F3A2
:10BBB0001188FEF745F800212B48FEF761FCFEF7DF
:10BBC00057F8002383F31188210612D5244A936F76
:10BBD0000BB1D06F9847202383F31188FEF730F81C
:10BBE00000212248FEF74CFCFEF742F8002383F3C5
:10BBF0001188E20514D51A4AD2F8883013B1D2F868
:10BC00008C009847202383F31188FEF719F8002150
:10BC10001748FEF735FCFEF72BF8002383F3118855
:10BC2000A30514D50E4AD2F8983013B1D2F89C006F
:10BC30009847202383F31188FEF702F800210D486E
:10BC4000FEF71EFCFEF714F8002383F31188FEF7BD
:10BC50003FF8BDE81040FEF7EBBD00BF003C0140DF
:10BC600080340020D0340020E0340020F034002064
:10BC7000003500201035002000000000000000000A
:10BC800010B5FEF70DF84B4B5A691C68144004F4CC
:10BC90007C425A61620514D5474AD2F8A83013B1E4
:10BCA000D2F8AC009847202383F31188FDF7C8FF32
:10BCB00000214248FEF7E4FBFDF7DAFF002383F39F
:10BCC0001188230514D53C4AD2F8B83013B1D2F804
:10BCD000BC009847202383F31188FDF7B1FF0021B2
:10BCE0003748FEF7CDFBFDF7C3FF002383F3118830
:10BCF000E00414D5304AD2F8C83013B1D2F8CC00E1
:10BD00009847202383F31188FDF79AFF00212D48DF
:10BD1000FEF7B6FBFDF7ACFF002383F31188A10407
:10BD200014D5254AD2F8D83013B1D2F8DC009847A0
:10BD3000202383F31188FDF783FF00212248FEF7BB
:10BD40009FFBFDF795FF002383F31188620414D550
:10BD5000194AD2F8E83013B1D2F8EC009847202302
:10BD600083F31188FDF76CFF00211848FEF788FB6C
:10BD7000FDF77EFF002383F31188230414D50E4AB8
:10BD8000D2F8F83013B1D2F8FC009847202383F39F
:10BD90001188FDF755FF00210D48FEF771FBFDF7F7
:10BDA00067FF002383F31188FDF792FFBDE8104081
:10BDB000FEF73EBD003C01408034002020350020CD
:10BDC00030350020403500205035002060350020FF
:10BDD000703500200000000000000000000000009E
:10BDE000062108B50846FFF793FD06210720FFF757
:10BDF0008FFD06210820FFF78BFD06210920FFF7A4
:10BE000087FD06210A20FFF783FD06211720FFF793
:10BE10007FFD06212820BDE80840FFF779BD00BF5F
:10BE2000284B29481A696FEAC2526FEAD25210B5FC
:10BE30001A611A69C2F308021A614FF0FF341A69D5
:10BE40005A695C6100215A6959615A691A6A62F03B
:10BE500080521A621A6A02F080521A621A6A5A6A88
:10BE60005C625A6A59625A6A1A6C42F080521A64C9
:10BE70001A6E42F080521A661A6E026842F480729C
:10BE800002601A6F02F44072B2F5407F03D04FF4A3
:10BE900080321A6719670B4B1A6F120407D41A6F96
:10BEA00042F440721A671A6F42F400421A67064A57
:10BEB000536823F40073536001F012F8BDE810409A
:10BEC000FFF78EBF00380240007000400000000005
:10BED000314B324A4FF080504FF4404118641160AA
:10BEE0001A6842F001021A601A689207FCD5996834
:10BEF000294A21F003019960936813F00C03FBD1E8
:10BF00001068254900F0F90010609360136843F44D
:10BF1000803313600B689803FCD54B6F1E4A43F0C7
:10BF200001034B67536F9907FCD51D4B5360136892
:10BF30001A4943F0807313604B685A04FCD5164AC3
:10BF400013689B01FCD5174B174991601A68174B72
:10BF50009A4217D0164B40F205721A600E4A936847
:10BF600043F002039360936803F00C03082BFAD1AB
:10BF7000536C43F480435364536E43F480435366DD
:10BF8000536E70470B4A0C4B12689A42E2D1084B31
:10BF900040F205121A60E1E70038024000700040EC
:10BFA00008544007002004E0009488381164002001
:10BFB000003C024000ED00E041C20F4100000000E3
:10BFC00070B50D4E0D4C0E4D3046FEF761FD0D4B1C
:10BFD0000D4AB2622046C6E90B53FEF759FD183DE3
:10BFE0000A4A0B4BE562A262236306211220BDE8D8
:10BFF0007040FFF78DBC00BF343300206833002051
:10C0000030170408162C02000020014000210140D6
:10C01000162C0202000000000000000000000000DA
:10C020000378012B00D070471F4B984210B504468F
:10C0300010D01E4B984222D01D48A26A436803F4D8
:10C040004003002143F48033012443605160916038
:10C05000946010BD0346174AC06A062100F070FFC5
:10C06000E36A15491A68154B91605A6C42F4807264
:10C070005A645A6E42F480725A665B6EDCE703467D
:10C080000C4AC06A062100F05BFFE36A0C491A689B
:10C090000A4B91605A6C42F400725A645A6E42F430
:10C0A00000725A665B6EC7E73433002068330020A5
:10C0B0000023014081C300084C20014000380240A9
:10C0C0004C210140000000000000000000000000C2
:10C0D0000369C2681978F0B4066B29B1012A94BFCC
:10C0E00046F4807646F48476C16A5D880C6881687F
:10C0F000E16002FB05F26260D968266027681E6A6B
:10C10000826A1869013D47F00107276046EA055534
:10C110005C69002616609E69D4609C8B1661DE8B7C
:10C120005462D3E9094341F08061966241F4807121
:10C13000D562146353634300516006D440F44070E9
:10C1400040F001009060F0BC704720F0804340F266
:10C15000033123F002030B4308439360F0BC90606B
:10C16000704700BF00000000000000000000000059
:10C1700030B4C46A2268136823F01F031360136885
:10C1800013F00103FBD1257A826A60683D21A94042
:10C19000016053609368012123F08043936030BCB9
:10C1A00091607047000000000000000000000000E7
:10C1B00038B5FDF775FD6B4A146800211160A206C1
:10C1C00000F18E8004F001042CB3674D2B6913B38A
:10C1D0002846FFF7CDFF2B699B68002B00F0B58048
:10C1E00005222A700221284698472B78052B04BF88
:10C1F00002232B7000232B61202383F31188FDF78A
:10C200001FFD4FF0FF315948FEF7EAF8FDF730FD0A
:10C21000002383F31188564A15680021AB0611608C
:10C220002ED405F001052DB3524C236913B32046DB
:10C23000FFF79EFF23699B68002B00F08280052298
:10C2400022700221204698472378052B04BF022341
:10C25000237000232361202383F31188FDF7F0FC72
:10C260004FF0FF314448FEF7BBF8FDF701FD002316
:10C2700083F31188FDF72CFDBDE83840FEF7D8BAEE
:10C280003C4CE26A1268526805F00105002ACAD0E7
:10C290002369002BEED02046FFF76AFF23699B68D5
:10C2A000002B5AD00522227001212046984723787E
:10C2B000052B04BF0223237000232361202383F373
:10C2C0001188FDF7BDFC4FF0FF312B48FEF788F8D1
:10C2D000FDF7CEFC002383F31188002DA4D1C9E71C
:10C2E000214DEA6A1268526804F00104002A3FF402
:10C2F0006BAF2B69002B8ED02846FFF739FF2B69D7
:10C300009B6833B305222A700121284698472B7871
:10C31000052B04BF02232B7000232B61202383F302
:10C320001188FDF78DFC4FF0FF311048FEF758F8EB
:10C33000FDF79EFC002383F31188002C3FF46BAFC4
:10C3400043E702222361227085E702222B612A70D3
:10C3500052E702222B612A70E0E702222361227059
:10C36000ACE700BF002001403433002048330020F8
:10C3700000210140683300207C33002000000000D1
:10C3800011F00C0F70B5044616D10369002B35D09F
:10C390008D0634D51A78002A3CD05D6875B3D0E993
:10C3A0000212012A59D95B885208540004FB031178
:10C3B0002B46BDE870401847FFF7DAFE23699B68FB
:10C3C000002B4ED00522227000212046984723786A
:10C3D000052B04BF0223237000232361202383F352
:10C3E0001188FDF72DFC04F114004FF0FF31FDF72B
:10C3F000F7FFFDF73DFC002383F3118870BDCA06EB
:10C40000FCD55B68002BF9D0D0E90212BDE8704082
:10C4100052081847FFF7ACFE23695B68C3B10422DA
:10C4200022702046D4E9021298472378042B0FD0BB
:10C43000202383F31188FDF703FC04F1140000218D
:10C44000FDF7CEFFFDF714FC002383F3118870BDC8
:10C450000222002322702361EAE72B46BDE87040E8
:10C460001847022223612270B8E700BF00000000D5
:10C47000024A536843F400035360704700230140AD
:10C48000C26A38B59368936013F00104054605D07D
:10C4900013F00C0F14BF4FF480340124D90506D5D6
:10C4A00013F4406F14BF44F4003444F00204DA0380
:10C4B00006D513F4402F14BF44F4802444F0040440
:10C4C000202383F31188FDF7BBFB05F10800002151
:10C4D000FDF7D6FF214605F11C00FEF729F9FDF70F
:10C4E000C7FB002383F3118838BD00BF00000000A4
:10C4F00038B5C36ADD68AA07044615D1EB0600D437
:10C5000038BDE36A1025DD60202383F31188FDF731
:10C5100097FB294604F12000FEF70AF9FDF7A8FB76
:10C52000002383F3118838BD5A6922F002025A6150
:10C53000202383F31188FDF783FB04F11000002111
:10C54000FDF79EFF04F118000121FEF7F1F8FDF759
:10C550008FFB002383F31188D0E700BF00000000A9
:10C5600038B5C36A1D69AA07044615D1EB0600D485
:10C5700038BDE36A10251D61202383F31188FDF780
:10C580005FFB294604F12000FEF7D2F8FDF770FBAF
:10C59000002383F3118838BD5A6922F010025A61D2
:10C5A000202383F31188FDF74BFB04F110000021D9
:10C5B000FDF766FF04F118000221FEF7B9F8FDF758
:10C5C00057FB002383F31188D0E700BF0000000071
:10C5D000C36A70B55C685C602207054614D46307C3
:10C5E00000D470BDEA6A2023946983F31188FDF7B3
:10C5F00027FB210405F12000FEF79AF8FDF738FB30
:10C60000002383F3118870BD1A68064622F00202E7
:10C61000032106F8281B20211A6081F31188FDF7F9
:10C620000FFB30460021FEF783F8FDF721FB0023C6
:10C6300083F31188D3E700BF000000000000000072
:10C64000F0B44B4D4B4B2E6CDB6A4B4F46F00076F3
:10C650002E642E6E46F000762E662C6ED3F80052B5
:10C660003D4045F00105C3F80052D3F800423C407C
:10C6700044F0010444EA0024C3F80042002947D0F2
:10C680000024C3F81C422046C3F804422546C3F8E0
:10C690000C42C3F8144203EBC00401301C28C4F858
:10C6A0004052C4F84452F6D10026012794781088ED
:10C6B00014F0010F03EBC00506F1010607FA00F0C4
:10C6C00005D0D3F804C240EA0C0CC3F804C214F03D
:10C6D000020F05D0D3F80CC240EA0C0CC3F80CC210
:10C6E000640704D5D3F814420443C3F814425468D1
:10C6F000C5F840429468C5F84442D3F81C42B142A0
:10C7000040EA040002F10C02C3F81C02CED11DE085
:10C7100003EBC0040122C3F84012C3F84412C4F86A
:10C720004012C4F84412C3F80412C3F81412C3F838
:10C730000C22C3F81C22D3F80C1282401143C3F818
:10C740000C12D3F81C020243C3F81C22D3F80012C7
:10C75000074A21F00101C3F80012136C23F00073A3
:10C760001364136E23F000731366136EF0BC7047EE
:10C77000003802409C3300200000FFFF0000000052
:10C7800008B5FDF78DFA0448FFF77AFEFDF7A0FA29
:10C79000BDE80840FEF74CB89C33002000000000C4
:10C7A00008B5FDF77DFA0448FFF7A2FEFDF790FA01
:10C7B000BDE80840FEF73CB89C33002000000000B4
:10C7C00008B5FDF76DFA0448FFF7CAFEFDF780FAD9
:10C7D000BDE80840FEF72CB89C33002000000000A4
:10C7E00008B5FDF75DFA0448FFF7F2FEFDF770FAB1
:10C7F000BDE80840FEF71CB89C3300200000000094
:10C8000008B5FDF74DFA0448FFF73AFEFDF760FA68
:10C81000BDE80840FEF70CB8CC3300200000000053
:10C8200008B5FDF73DFA0448FFF762FEFDF750FA40
:10C83000BDE80840FDF7FCBFCC330020000000003D
:10C8400008B5FDF72DFA0448FFF78AFEFDF740FA18
:10C85000BDE80840FDF7ECBFCC330020000000002D
:10C8600008B5FDF71DFA0448FFF7B2FEFDF730FAF0
:10C87000BDE80840FDF7DCBFCC330020000000001D
:10C8800038B5194D194C2846FEF74AF9184BEB629A
:10C890000B211320FFF73CF80B211420FFF738F889
:10C8A0000B211520FFF734F80B211620FFF730F885
:10C8B0002046FEF735F90F4BE3620B213F20FFF7CF
:10C8C00027F80B214020FFF723F80B214120FFF729
:10C8D0001FF80B214220FFF71BF8002211460E2003
:10C8E000BDE83840FFF7ACBE9C330020CC330020BD
:10C8F00000640040006800400000000000000000EC
:10C90000194B984210B5044623D0184B984215D0C5
:10C91000E36A01221A605A68D10707D4012108206E
:10C92000FDF7D6FAE36A5A68D207F7D5626810496C
:10C93000D2E90020D8611A60596110BD0D4B1A6C04
:10C9400042F080621A641A6E42F080621A661B6EB0
:10C95000DEE7084B1A6C42F000721A641A6E42F05D
:10C9600000721A661B6ED3E79C330020CC33002084
:10C970005B8701000038024000000000000000005A
:10C9800003291AD8DFE801F0110C0702C36A98687E
:10C99000C0F300707047C36A9868C0F3C060704706
:10C9A000C36A9868C0F380607047C36A9B6813F0DD
:10C9B000E05F14BF0120002070470020704700BFD7
:10C9C000032934D8DFE801F0232B1F02C16A01F5E7
:10C9D000D071107810B4C0F3001384064FEA4303FB
:10C9E00021D5546843EAC40343F00403D2E9024268
:10C9F00000F00F0043F0010348608C60CA605DF8EE
:10CA0000044B0B607047C16A01F5C871E1E7C16A68
:10CA10008B68C3F30163183301EB0311D9E7C16AD3
:10CA200001F5C071D5E7948843EA4453DEE77047C7
:10CA3000012911D00AD3022906D1C36A186910F05E
:10CA4000030018BF0120704700207047C36ADA68EE
:10CA50009207F3D001207047C36AD86810F0030032
:10CA600018BF0120704700BF000000000000000058
:10CA700030B400292FD1C36AD968880744D0D3F8CD
:10CA8000B001D3F8B411D3F8B841D3F8BC51146154
:10CA900020245561DC60DC68A50703D15C6944F0A3
:10CAA00002045C611379440864F30413840864F39A
:10CAB000451313719B062BD59368C00860F31C03C4
:10CAC00093601379080A61F30303090C1371107062
:10CAD000518030BC7047012920D00229F9D1C36AA6
:10CAE000D3F8C001D3F8C411D3F8C841D3F8CC515E
:10CAF0001461202455611C611C69A407D2D15C69B2
:10CB000044F010045C61CDE719698907E8D1E0E7DA
:10CB10001389400D60F30A031381D2E7C36AAEE7BD
:10CB200008B5FDF7BDF8084B084A196801F03D014A
:10CB3000996013680BB150689847FDF7C9F8BDE8D4
:10CB40000840FDF775BE00BF00600240FC330020C6
:10CB500010B5FDF7A5F8094B0948196882688909DD
:10CB600001F03D018C019C600AB1C0689047FDF75F
:10CB7000AFF8BDE81040FDF75BBE00BF00600240AB
:10CB8000FC33002000000000000000000000000056
:10CB900010B5FDF785F8094B094819680269090CB9
:10CBA00001F03D010C049C600AB140699047FDF71B
:10CBB0008FF8BDE81040FDF73BBE00BF00600240AB
:10CBC000FC33002000000000000000000000000016
:10CBD00010B5FDF765F8094B094819688269890D98
:10CBE00001F03D018C059C600AB1C0699047FDF7DA
:10CBF0006FF8BDE81040FDF71BBE00BF00600240AB
:10CC0000FC330020000000000000000000000000D5
:10CC100008B5FDF745F8084B08485968026A01F065
:10CC20003D01D9600AB1406A9047FDF751F8BDE86F
:10CC30000840FDF7FDBD00BF00600240FC3300204E
:10CC400010B5FDF72DF8094B09485968826A890922
:10CC500001F03D018C01DC600AB1C06A9047FDF72C
:10CC600037F8BDE81040FDF7E3BD00BF00600240AB
:10CC7000FC33002000000000000000000000000065
:10CC800010B5FDF70DF8094B09485968026B090CFE
:10CC900001F03D010C04DC600AB1406B9047FDF7E8
:10CCA00017F8BDE81040FDF7C3BD00BF00600240AB
:10CCB000FC33002000000000000000000000000025
:10CCC00010B5FCF7EDFF094B09485968826B890DD7
:10CCD00001F03D018C05DC600AB1C06B9047FCF7A8
:10CCE000F7FFBDE81040FDF7A3BD00BF00600240A4
:10CCF000FC330020000000000000000000000000E5
:10CD000008B5FCF7CDFF084B08481968026C01F024
:10CD10003D0199600AB1406C9047FCF7D9FFBDE82E
:10CD20000840FDF785BD00BF00640240FC330020D1
:10CD300010B5FCF7B5FF094B09481968826C8909E1
:10CD400001F03D018C019C600AB1C06C9047FCF77A
:10CD5000BFFFBDE81040FDF76BBD00BF006402409F
:10CD6000FC33002000000000000000000000000074
:10CD700010B5FCF795FF094B09481968026D090CBD
:10CD800001F03D010C049C600AB1406D9047FCF736
:10CD90009FFFBDE81040FDF74BBD00BF006402409F
:10CDA000FC33002000000000000000000000000034
:10CDB00010B5FCF775FF094B09481968826D890D9C
:10CDC00001F03D018C059C600AB1C06D9047FCF7F5
:10CDD0007FFFBDE81040FDF72BBD00BF006402409F
:10CDE000FC330020000000000000000000000000F4
:10CDF00008B5FCF755FF084B08485968026E01F06A
:10CE00003D01D9600AB1406E9047FCF761FFBDE873
:10CE10000840FDF70DBD00BF00640240FC33002058
:10CE200010B5FCF73DFF094B09485968826E890926
:10CE300001F03D018C01DC600AB1C06E9047FCF747
:10CE400047FFBDE81040FDF7F3BC00BF006402409F
:10CE5000FC33002000000000000000000000000083
:10CE600010B5FCF71DFF094B09485968026F090C02
:10CE700001F03D010C04DC600AB1406F9047FCF703
:10CE800027FFBDE81040FDF7D3BC00BF006402409F
:10CE9000FC33002000000000000000000000000043
:10CEA00010B5FCF7FDFE094B09485968826F890DE2
:10CEB00001F03D018C05DC600AB1C06F9047FCF7C2
:10CEC00007FFBDE81040FDF7B3BC00BF006402409F
:10CED000FC33002000000000000000000000000003
:10CEE0000E490F4A0F48002310B40B600E4C194630
:10CEF00001E052F80C0C016044F833100133102BA0
:10CF000002F10C02F5D10949094A5DF8044B4FF0D2
:10CF1000FF338B60CB609360D36070477C3400201C
:10CF2000AC16040810600240FC3300200060024090
:10CF3000006402400000000000000000000000004B
:10CF4000F8B5DFF898C0477ADCF80050012404FAFD
:10CF500007F62E423CD11F4C354304EBC70615F0B3
:10CF6000FF0FCCF8005044F83720736009D01A4BFB
:10CF70001C6B44F400141C631C6D44F400141C6509
:10CF80001B6D15F47F4F16D105682B6823F01F0326
:10CF90002B602C6814F00104FBD1077A46683D230E
:10CFA000BB40212733602C606F617AB1807AFEF735
:10CFB000AFFC2046F8BD084B1C6B44F480041C6396
:10CFC0001C6D44F480041C651B6DDDE71046F8BD44
:10CFD0002046F8BDFC330020003802407C3400209D
:10CFE00010B50446807AFEF7B3FC1149607A0B68ED
:10CFF0000122824023EA020313F0FF0F0B6009D1E4
:10D000000C4A116B21F400111163116D21F4001110
:10D010001165126D13F47F4F09D1064B1A6B22F480
:10D0200080021A631A6D22F480021A651B6D10BD0E
:10D030007C340020003802400000000000000000A6
:10D04000054B002203F58071C3E90033C3E90222D6
:10D0500010338B42F8D1704780340020000000006C
:10D060002DE9F04F02F00309C2F3800EC2F3C10CA8
:10D07000C2F34117C846C2F3C31200264FF0010A9B
:10D0800016E0D0F800B003EA0B0343EA0803072ECA
:10D09000036044D8036A1D402C43046249083CD015
:10D0A0004FEA4E0E4FEA8C0CBF004FEA880801365B
:10D0B000CB07F3D543680AFA06F423EA040343EAEC
:10D0C0000E03436003257300846805FA03F3DB4312
:10D0D0001C4044EA0C048460C56806F00704A40000
:10D0E0001D404FF00F0B3D430BFA04FBB9F1020F4B
:10D0F000C56002FA04F46FEA0B05C2D1072E13D8FB
:10D10000D0F820B00BEA05052C43046204682340E4
:10D1100043EA080349080360C2D1BDE8F08F436ABF
:10D120001D402C434462B9E7D0F824B00BEA050552
:10D130002C434462EAE700BF00000000000000004A
:10D1400021F0030303F1804303F59C3370B401F035
:10D1500003049D68A4000F26A640C0F3832025EA9F
:10D160000605A040012404FA01F128430D4C986003
:10D17000A368D5076FEA01004CBF0B43034012F0D0
:10D18000020F084AA360D36814BF0B430340D36067
:10D19000044B1A68114319605A6802405A6070BC07
:10D1A000704700BF003C014000000000000000008C
:10D1B00010B5124C2046FEF713FA114B2360532290
:10D1C000CA2159625A62DA6812F0100FDA6811D176
:10D1D00042F08002DA60DA685206FCD5094A002083
:10D1E00080219860D9601A611A61DA6822F08002A1
:10D1F000DA6010BD22F02002DA6010BD8035002018
:10D2000000280040FF031F00000000000000000095
:10D2100011F00C0F00D170470148FCF791BC00BF22
:10D220006417040800000000000000000000000077
:10D2300011F00C0F70B50E4604464CD163681A7895
:10D240005D6842B1F0063AD5002D37D020462B4616
:10D25000BDE870401847606A0268136823F01F0336
:10D2600013601368D907FCD4027A216A40683D2311
:10D2700093400A680360136823F01F031360136868
:10D28000DB07FCD4087A4A683D238340136035B33A
:10D29000042323702046A8472378042B1FD0202383
:10D2A00083F31188FCF7CCFC04F108000021FDF7A2
:10D2B00097F8FCF7DDFC002383F3118870BD002D87
:10D2C000FCD0042323702046A8472378042BF5D1F3
:10D2D0000323237070BD0348FCF732FCAEE7022342
:10D2E0002370DCE764170408000000000000000061
:10D2F00070B50F4E0F4D104C3046FEF781F90F4AB6
:10D300000F4B1049F161204605F12401C6E908518F
:10D31000C6E90A23FEF774F90B490C4A0C4BE1618C
:10D32000A5F160010C3DC4E90815C4E90A2370BDEC
:10D330008435002000170408B435002016000106CB
:10D340004600010600300140003C0040160001008C
:10D350004600010000000000000000000000000086
:10D360000378012B70B504462FD0C1696568A26AA5
:10D37000288AE36A060522F4F04223F4F0432E786B
:10D3800044BF42F4205243F42053C4E90A23AEB907
:10D3900022F4847223F48473C4E90A230A686B8A32
:10D3A00040F4417043F0070322F040020A60086035
:10D3B0004B600B6843F040030B6070BD42F4847215
:10D3C00043F48473C4E90A23E8E71F4B98420CD066
:10D3D0001E4B984220D0D4E90823E16910681A68EE
:10D3E00001F10C0383609360C0E70346184A006AAA
:10D3F0000A21FFF7A5FD2346164A606A0A21FFF7B6
:10D400009FFD154B5A6C42F480525A645A6E42F496
:10D4100080525A665B6EDEE703460D4A006A0A21B7
:10D42000FFF78EFD23460B4A606A0A21FFF788FD4D
:10D43000094B1A6C42F400421A641A6E42F400421C
:10D440001A661B6EC7E700BF84350020B435002084
:10D4500031D2000811D2000800380240000000005C
:10D460000378022B00D0704710B50446D0E907308E
:10D470001A68002122F040021A6019605960FFF713
:10D48000AFFD606AFFF7ACFD0D4B9C420DD00D4B1C
:10D490009C4209D10C4B1A6C22F400421A641A6E99
:10D4A00022F400421A661B6E10BD074B5A6C22F420
:10D4B00080525A645A6E22F480525A665B6E10BDD6
:10D4C00084350020B4350020003802400000000000
:10D4D000D0E9082330B412681B680A4CD0E90A501E
:10D4E000D460094C51601560DC60596018601168A7
:10D4F00041F0010111601A6842F001021A6030BC6B
:10D50000704700BFE43500206017040800000000E9
:10D5100070B4D0E90854D0E90A602D682468EB6043
:10D5200046F4806640F4806069602E60E26061606D
:10D5300020602B6843F001032B60236843F0010354
:10D54000236070BC704700BF0000000000000000B6
:10D5500070B4D0E90843C56A24681B68806A094E24
:10D56000E66045F4806561602060DA6059601D60A6
:10D57000226842F0010222601A6842F001021A6039
:10D5800070BC7047E435002000000000000000007F
:10D5900030B4D0E90843856A24681B68C06AE26039
:10D5A00045F48065074A61602560DA60596018605B
:10D5B000226842F0010222601A6842F001021A60F9
:10D5C00030BC704760170408000000000000000035
:10D5D00008B5FCF765FB202383F31188FCF730FBCB
:10D5E000FCF7BEFAFCF744FB002383F31188FCF739
:10D5F0006FFBBDE80840FDF71BB900BF000000004D
:10D60000054B064A5A600021072299600B20082129
:10D610001A60FEF7B5B900BF10E000E03F900200CD
:10D6200008B5FCF73DFB0C4B1878DA68002104289C
:10D63000116107D10220187011601161D16821F0C9
:10D64000FF01D1605B6804485B689847FCF740FBCA
:10D65000BDE80840FDF7ECB8E83500200000000008
:10D660000248034BC360FDF70BBB00BFE835002049
:10D67000000C00400000000000000000000000005E
:10D6800038B50378012B044612D0D4E90103C168F0
:10D690000568E268B3FBF5F3013B84689BB20020A8
:10D6A00021F0FF011060546093621061D16038BDB9
:10D6B0000E4B9842E9D10E4B1A6C42F008021A64E4
:10D6C0001A6E42F008021A661A6E1A6A42F00802CE
:10D6D0001A621A6A22F008021A62042132201B6AB6
:10D6E000FEF716F9034BA360CFE700BFE835002033
:10D6F0000038024000BD01050000000000000000ED
:10D700004268C36850680139D96200220121596119
:10D710005A621A6110B1DA680A43DA6085221A6027
:10D72000704700BF00000000000000000000000083
:10D73000C36800221A601A61DA6822F0FF02DA6018
:10D74000704700BF00000000000000000000000063
:10D75000F8B50D4F0D4E0E4D0E4C3846FDF7D8FA6C
:10D760000D4BFB603046FDF7D3FA4FF0804328465F
:10D77000F360FDF7CDFA094BEB602046FDF7C8FAE0
:10D78000074BE360F8BD00BFF835002010360020DD
:10D7900028360020403600200000014000040040F0
:10D7A00000400140000000000000000000000000F8
:10D7B0000378012B70B504463AD0C36800221A6082
:10D7C0005A639A635A62D4E9011288690D7D20F088
:10D7D000FF0000261E61D8604868B2FBF0F24FF6E9
:10D7E000FF70013A9A620A78D8626DB940F201205E
:10D7F000542198619960C2B113221A6203F1380270
:10D800003433C4E9042370BD4FF4817064219861FE
:10D8100099603AB131221A6203F134023833C4E913
:10D82000042370BD13221A62F6E731221A62E5E77B
:10D830003A4B984253D03A4B98423BD0394B98429E
:10D840001DD0394B984218D1384B5A6C42F4803273
:10D850005A645A6E42F480325A665A6E5A6A42F4D8
:10D8600080325A625A6A22F480325A6203211820A6
:10D870005B6AFEF74DF82E4BA360E368A3E72B4BE2
:10D880001A6C42F002021A641A6E42F002021A6620
:10D890001A6E1A6A42F002021A621A6A22F0020230
:10D8A0001A6203211D201B6AFEF732F8214BA36088
:10D8B000E36888E71D4B1A6C42F001021A641A6E85
:10D8C00042F001021A661A6E1A6A42F001021A62E6
:10D8D0001A6A22F001021A6203211C20E3E7134BAB
:10D8E0005A6C42F001025A645A6E42F001025A66C2
:10D8F0005A6E5A6A42F001025A625A6A22F00102D2
:10D900005A62032119205B6AFEF702F803211B20EB
:10D91000FDF7FEFF064BA360AFE700BFF835002020
:10D920001036002028360020403600200038024003
:10D93000007A030A00BD010500000000000000009D
:10D9400008B50378022B00D008BD2649C368002221
:10D9500088421A60DA601A6132D0234B984221D093
:10D96000224B984210D0224B9842EDD11820FDF75F
:10D97000EFFF204B5A6C22F480325A645A6E22F424
:10D9800080325A665B6E08BD1D20FDF7E1FF194B22
:10D990001A6C22F002021A641A6E22F002021A664F
:10D9A0001B6E08BD1C20FDF7D3FF124B1A6C22F032
:10D9B00001021A641A6E22F001021A661B6E08BD7B
:10D9C0001920FDF7C5FF1B20FDF7C2FF094B5A6C5C
:10D9D00022F001025A645A6E22F001025A665B6E0E
:10D9E00008BD00BFF8350020103600202836002082
:10D9F0004036002000380240000000000000000017
:10DA0000C3685A69002042F0010205215A61186179
:10DA100019607047000000000000000000000000D6
:10DA2000C36800221A60DA6822F0FF02DA607047E9
:10DA3000C268D36810B413F0FF040CD141681461BC
:10DA40000C7D886854B970B143F00603096909B1C7
:10DA500043F00103D3605DF8044B70470028F3D115
:10DA600043F00403F2E743F00203EFE70000000095
:10DA7000C268D36823F0FF03D36070470000000042
:10DA8000C36841681A69F0B5DD680E7D1540EAB2D9
:10DA9000D2431A6183B0044605F0020305F004077F
:10DAA0007EB9002F2CD00278042A24D07BB9EB0752
:10DAB00005D5636820461B6998470323237003B08C
:10DAC000F0BD53B10378042B04D0002FEFD0042312
:10DAD0002370ECE78B68E3B19847002FE7D02378F9
:10DAE000042BF4D16168CB68002BF0D02046984716
:10DAF00004232370DBE78A6842B101939047019BBE
:10DB0000002BD4D02378042BE1D1EBE7002BCED02F
:10DB1000E9E7002FCBD0E6E700000000000000009E
:10DB200008B5FCF7BDF80448FFF7AAFFFCF7D0F8EA
:10DB3000BDE80840FCF77CBEF8350020000000007E
:10DB4000FFF7EEBF00000000000000000000000032
:10DB500008B5FCF7A5F80448FFF792FFFCF7B8F802
:10DB6000BDE80840FCF764BE10360020000000004D
:10DB700008B5FCF795F80448FFF782FFFCF7A8F812
:10DB8000BDE80840FCF754BE283600200000000025
:10DB900008B5FCF785F80448FFF772FFFCF798F822
:10DBA000BDE80840FCF744BE4036002000000000FD
:10DBB00038B5084D084C2846FDF7DAFC0422074B1F
:10DBC0002A742046AB61FDF7D3FC0622044B227475
:10DBD000A36138BD5836002074360020000800408C
:10DBE00000040140000000000000000000000000F0
:10DBF0000378012B70B504464ED0836900221A6069
:10DC00005A639A63DA631A645A62D4E90115CA68DE
:10DC100060690E68B0FBF6F002F00F026C1E01386E
:10DC2000CD6A9862012ADC625D6003D0022A0CBFD3
:10DC300003220022486900F00F00012829D00228A1
:10DC400025D0C86900F00F0001281DD0022819D086
:10DC5000486A00F00F00012803D0022803D142F4E3
:10DC6000005242F48052096B1A62012521F0FF0232
:10DC700000244FF4004085215D611C61DA60586426
:10DC8000196070BD42F4007242F48072E0E742F025
:10DC9000200242F01002D4E7214B984208D0214BD9
:10DCA00098421FD0A36946F668029A61DA61ACE730
:10DCB0001D4B1A6C42F004021A641A6E42F0040200
:10DCC0001A661A6E1A6A42F004021A621A6A22F07E
:10DCD00004021A6207211E201B6AFDF719FE134B6E
:10DCE0006361DFE7104B5A6C42F002025A645A6ECD
:10DCF00042F002025A665A6E5A6A42F002025A62B0
:10DD00005A6A22F002025A6207212C205B6AFDF750
:10DD1000FFFD07212E20FDF7FBFD054B6361C1E7E9
:10DD200058360020743600200038024000BD01053E
:10DD3000007A030A0000000000000000000000005C
:10DD40008269D368D90705D443F001036FF001015C
:10DD50001161D360704700BF0000000000000000A8
:10DD6000836970B51A69DC681440E2B2D243A60731
:10DD700005461A6103D543681B6903B198476007DC
:10DD800004D56B689B690BB128469847210704D5D9
:10DD90006B681B6A0BB128469847E20604D56B688E
:10DDA0009B6A0BB128469847E30706D56B689B68CA
:10DDB0001BB12846BDE87040184770BD0000000048
:10DDC00008B5FBF76DFF0448FFF7CAFFFBF780FFBC
:10DDD000BDE80840FCF72CBD5836002000000000CC
:10DDE00008B5FBF75DFF0448FFF7BAFFFBF770FFCC
:10DDF000BDE80840FCF71CBD7436002000000000A0
:10DE0000FFF7EEBF0000000000000000000000006F
:10DE1000C1690A68136823F01F0330B413601368E4
:10DE2000DB07FCD40D7A046A496822683D23AB40C5
:10DE30000B60136823F01F031360136813F00103D2
:10DE4000FBD1257A426960683D21A940016030BC60
:10DE5000D3601361536170470000000000000000B0
:10DE600011F00C0F38B504462DD1216A0A681368E9
:10DE700023F01F0313601368DB07FCD463680D7A7B
:10DE800048681A683D23AB40022103606170BAB153
:10DE9000204690476378022B12D0237A03B938BD0D
:10DEA000202383F31188FBF7CBFE04F1100000213F
:10DEB000FCF796FAFBF7DCFE002383F3118838BDEC
:10DEC00000236370E9E70248FBF73AFECDE700BFA5
:10DED000801704080000000000000000000000009F
:10DEE00011F00C0F2DE9F0410D46044613D1A27834
:10DEF00063683AB9DB68002B37D0A18C2046BDE8B7
:10DF0000F04118475A6A52B1E80630D52046002140
:10DF1000BDE8F04110472548FBF712FEE7E7E0694E
:10DF200001680A6822F01F020A600A68D207FCD45E
:10DF3000077A46689D683D22BA4002203260A07090
:10DF4000FDB12046A847A378022B17D0202383F3E6
:10DF50001188FBF775FE04F10C000021FCF740FA74
:10DF6000FBF786FE002383F31188BDE8F081A90644
:10DF7000FBD520460121BDE8F0411047E269636806
:10DF80001168DB68A269002B14BF4FF488734FF44B
:10DF9000807313430120002504F12402A570CA6098
:10DFA00048600B600B6803430B60CFE780170408E1
:10DFB000F8B53A4EFBF774FE7469E7682568636844
:10DFC00040F20F131D422CD073681A696FF48073EE
:10DFD0002360BAB1ABB213F0080F0CBF00211021BF
:10DFE000D80748BF41F00401980748BF41F0080135
:10DFF000580748BF41F02001DB0548BF41F0400110
:10E0000026489047202383F31188FBF719FE6FF011
:10E0100001012348FCF7E4F9FBF72AFE002383F310
:10E02000118868060ED579060CD573686FF040012B
:10E030005A68216007EA0103E3600AB11748904774
:10E04000347AECB1EA0615D5FB0613D573681B6A62
:10E050000BB112489847202383F31188FBF7F0FD9A
:10E060004FF0FF310E48FCF7BBF9FBF701FE002330
:10E0700083F31188FBF72CFEBDE8F840FCF7D8BB12
:10E08000202383F31188FBF7DBFD21460548FCF7CD
:10E09000A7F9FBF7EDFD84F31188D3E79036002054
:10E0A0009C360020A0360020000000000000000088
:10E0B00010B5074C2046FDF79BFB064B064A6261F4
:10E0C000062103F11802C4E90613226210BD00BF45
:10E0D00090360020B8160408004C004000000000F4
:10E0E0000378012B2DE9F041044655D04569002302
:10E0F000A37063702046FFF78BFE434B6169994222
:10E1000063683BD041485A69814238D04049B1FBED
:10E11000F2F2198B080438D4D3F80CE0D3F820803D
:10E120005F8B988BE369AA602A686A68D4F818C084
:10E130001B6800222A6042F21C1642F20C12B8F14F
:10E14000000F08BF1646BEF1000F14BF4FF48872CF
:10E150004FF48072314342EA0C02012647F0400737
:10E1600040F0C10024342F616861E960DC605E60CA
:10E170001A601A6832431A60BDE8F0815A6925496D
:10E18000B1FBF2F2198B0804C6D522F0070002F0A9
:10E19000070242EA4002BFE71F4B984215D063686E
:10E1A0001B8B03F4A053B3F5805F03D1A36943F441
:10E1B0002053A361D4E90723656910681968002218
:10E1C0002B1D83608B60A28491E70346134AC069CC
:10E1D0000621FEF7B5FE2346114A206A0621FEF706
:10E1E000AFFE104B1A6C42F400221A641A6E42F40D
:10E1F00000221A66062134201B6EFDF789FBA369F5
:10E2000043F00063A361CAE700100140001401401D
:10E2100080DE800200BD010590360020E1DE0008AE
:10E2200061DE00080038024000000000000000002D
:10E230000278022A00D0704710B50446FFF7E8FDC7
:10E24000E069FEF7CDFE206AFEF7CAFE084B9C424D
:10E2500000D010BD3420FDF77BFB064B1A6C22F476
:10E2600000221A641A6E22F400221A661B6E10BD78
:10E27000903600200038024000000000000000003E
:10E2800030B4036A456884691B686D68DA6044F4D9
:10E290008A6459601C606DB142696FF04001116081
:10E2A000D16841F04001D1601A6842F001021A6061
:10E2B00030BC7047027A002AEED0F5E7000000007B
:10E2C000016A0A68136823F01F0313601368DB07F1
:10E2D000FCD4087A49683D2383400B60506870473E
:10E2E000F0B4C5692B681C6824F01F041C601C680E
:10E2F000E407FCD444682F7A6E68656A3D24BC400C
:10E3000034608069DA60002D0CBF4FF482624FF4F4
:10E31000A362024359601A601A6842F001021A604F
:10E32000F0BC70470000000000000000000000008A
:10E33000404A414913694148F0B440F2FF14234375
:10E34000136113693E4E3F4D23F4FF7323F0010325
:10E3500013611369136B23431363136D2343136515
:10E360006FF4A8470023126D4B604FF6FF728F6069
:10E37000CE60354E4A610E62344E4E6206F12A5628
:10E3800006F5B0160E60402646604FF0FF31304E65
:10E390008160C6604FF08066426106624FF40256AB
:10E3A000436206602B4E2C4C6B60A960EE60012628
:10E3B0006A612B626B622E60284D6360A160E5602C
:10E3C00040F6FF756561264D2362264E6362256027
:10E3D000C0F8043C244DC0F8081C04F58054C0F873
:10E3E0000C3CC0F8142CC0F8203CC0F8243CC0F809
:10E3F000003C00F5E0507360B160F360726133621D
:10E40000736233606B60A960EB606A612B626B6260
:10E410002B606360A160E3606261236263622360DA
:10E420004360F0BC8160C360426103624362036089
:10E43000FDF74EBD003802400000024000040240DB
:10E4400054000140000802400000565500AA0A008E
:10E450001585AAAAA8AAAAAA000C024055505500E0
:10E4600000010055001402400018024000000000A6
:10E4700001207047000000000000000000000000C4
:10E4800000207047000000000000000000000000B5
:10E49000704700BF00000000000000000000000006
:10E4A000024BD878203818BF0120704700000008C0
:10E4B000162303604FF0FF30704700BF00000000DC
:10E4C0000020704700000000000000000000000075
:10E4D0001846704700000000000000000000000027
:10E4E0000020704700000000000000000000000055
:10E4F00010B50022044608460421FCF761F900B17A
:10E5000010BD0C2323604FF0FF3010BD0000000051
:10E5100008B51046002158222EF0C2F94FF40052DF
:10E520004260002008BD00BF0000000000000000A5
:10E530000120704700000000000000000000000003
:10E54000D0E902239A4206D04268D154C36801330D
:10E55000C360002070476FF00100704700000000AA
:10E56000D0E903139942024604D04168C85C0133E4
:10E57000136170476FF00100704700BF000000009A
:10E5800070B5D0E90343E41A4668944228BF1446A4
:10E59000054622460846F118FAF754FF2B69234432
:10E5A0002B61204670BD00BF00000000000000008D
:10E5B00038B5D0E90243E41A05469442406828BFC2
:10E5C000144618442246FAF73DFFEB682344EB60FB
:10E5D000204638BD000000000000000000000000E0
:10E5E00010B44160044C04600021C0E902230161C1
:10E5F0005DF8044B704700BF9C1704080000000042
:10E600002DE9F04F2DED028B064691B089469246DA
:10E610004FF0000B99F8001009F1010271B12529A2
:10E6200012D033689146DB683046984799F800105D
:10E630000BF1010B09F101020029F0D1584611B08C
:10E64000BDEC028BBDE8F08F99F801102D2903BFB6
:10E6500099F8021009F1020201230023302908BFB2
:10E660005178029306BF013230272027013200245F
:10E6700007E09AF800300AF1040A12F8011B03EBD4
:10E680004004A1F13003DBB2092B154604EB8400F2
:10E69000F3D92A29EDD02E294FF000084AD001F0F5
:10E6A000DF034C2B05F1010950D0A1F14103A1F189
:10E6B0004402DBB2342A00F2D381DFE812F01E02FA
:10E6C000D101D101D101D1011E02D101D101D1016C
:10E6D000D101D101CD01D101D101D101D101D101AE
:10E6E0009701D101D1012702D101D101D101D1017D
:10E6F000D101D101D101D101D101D1014E011E02BF
:10E70000D101AA00D101D1011E02D101D101D10153
:10E71000D101D101CD01D101D101D1018800D101B7
:10E720009701D101D10127029AF800300AF1040AB9
:10E7300003EB420815F8011BA1F13003DBB2092BF2
:10E7400008EB8802F4D92A29EED0A8E72B78DBB3AE
:10E75000A3F14402342A00F28581DFE812F0A2011D
:10E760008301830183018301A2018301830183016A
:10E77000830183017E01830183018301830183017E
:10E780004801830183019F01830183018301830188
:10E79000830183018301830183018301FF00A201BF
:10E7A00083015B0083018301A20183018301830153
:10E7B000830183017E018301830183013900830189
:10E7C0004801830183019F010B46A946C0E7A94682
:10E7D000DAF800500AF1040A002D00F0A6812B7827
:10E7E0002946B8F1000F40F0BF81002B00F0CC812A
:10E7F00047F6FE782B4602E0B8F1010803D413F87F
:10E80000012F002AF8D15B1AE41A013B019320275B
:10E81000AFE0A9460AF1070A2AF0070ADAE900017F
:10E82000FAF78CFA08EE100AB5EEC08AF1EE10FA8B
:10E830000AF1080A00F16E810AAB0393019318EE06
:10E84000100AF9F74BFF08F1FF38B8F1080FCDE9CE
:10E85000040100F27381C04B53F828502846F9F7A1
:10E860001BFFBE4BCDE90601A3FB0535EB08099361
:10E870001D46FDEEC87A019BDFF8E0E2CDED087A97
:10E8800003F10B0817EE901A4246AEFB0103DB08BA
:10E8900003EB830C1846A1EB4C033033DBB202F8D8
:10E8A000013D01460028F0D10199A8EB0208084675
:10E8B000404401E012F8013F01F8013B8142F9D1E7
:10E8C000019A08982E2308F1FF3842440B700192F8
:10E8D000F9F7F2FE02460B46DDE90401F9F79EFD69
:10E8E000DDE90623F9F752FFFAF700FA019B099ACE
:10E8F0009A4903F10D080233002A08BF0546089320
:10E900004246A1FB00C3DB0803EB830E9C46A0EB51
:10E910004E033033A1FB0505DBB2ED0802F8013DE3
:10E920006046EED1A8EB0208019908F1020001440B
:10E930000846089901E012F8013F01F8013B8142C5
:10E94000F9D1089B039D43449846A8EB050808F1BC
:10E95000FF33A4EB080401930BE0A94610ADDAF8ED
:10E96000003005F8183D0023013C0AF1040A019328
:10E970002027002C6ADB029B002B7BD16342002CFA
:10E9800077D0297832682D29D26877D0984601E06F
:10E990003368DA6839463046904718F10108F7D1F4
:10E9A000019A002A4346A344FFF634AE1C46DDF824
:10E9B0000480336815F8011BDB6808F1FF38304626
:10E9C0009847B8F1FF3FF4D1019B0BF1010B5B4479
:10E9D0009B46002C3FF41EAE254633683946DB6863
:10E9E00030469847013DF8D1A34413E6A9464FF0BD
:10E9F0000A0C5AF8042B0DF1330100E00146B2FB7A
:10EA0000FCF50CFB152202F13003392BC8BF02F1D3
:10EA10003703DBB201F8013C481E2A46002DEDD138
:10EA20000DF133050AAAA5EB00080392404401E06A
:10EA300011F8013B02F8013B8142F9D1A4EB080433
:10EA400008F1FF33002C0193039D94DA019B002B06
:10EA5000FFF6E0AD0024AAE7A9464FF0080CC8E78E
:10EA60000B46A94610AD013C05F8183D0023019363
:10EA70007FE71C46019B002B99DAAAE7302F85D14E
:10EA8000304602939047019B3268013B0193029B01
:10EA9000D2680BF1010B013598467BE74FF0100C63
:10EAA000A7E70AF10402DAF800109246002962DBB7
:10EAB0000AAD039505F10B02DFF8A0801046A8FB14
:10EAC00001C3DB0803EB830E9C46A1EB4E033033FE
:10EAD000DBB2614600F8013D0029F0D1121A2A4448
:10EAE00001E010F8013F05F8013BAA42F9D1039D6E
:10EAF000521B531EA41A01933BE75246192B52F89E
:10EB0000041BA94688BF9246D0D8CCE7A9464FF04F
:10EB1000100C6EE72D238DF828300DF12903019399
:10EB20000AABB1EE488A039389E60D490D46B8F168
:10EB3000000F3FF45DAE08F1FF385BE69FED047B0C
:10EB4000084D09958DED067B93E600BFAFF300807D
:10EB50000000000065CDCD41B8170408CDCCCCCC69
:10EB6000B017040800E1F505002BE4D14FF0FF33A6
:10EB700001932027FDE62D238DF828300AAB49426A
:10EB80000DF12905039395E74FF0FF3301932027FB
:10EB9000F1E600BF000000000000000000000000DF
:10EBA0000EB400B582B003AA52F8041B0192FFF71D
:10EBB00027FD02B05DF804EB03B0704700000000D1
:10EBC0000CB430B5054687B00C46B1B14A1E01A859
:10EBD00000232946FFF704FD0BAB1A4601A80A994A
:10EBE0000093FFF70DFD049BA34201D20022EA54DB
:10EBF00007B0BDE8304002B070470146234601A887
:10EC00002246FFF7EDFC0BAB01A81A460A990093C8
:10EC1000FFF7F6FC07B0BDE8304002B0704700BF18
:10EC200000291CDD421E10B40020541812F8011FE8
:10EC30000823484010F0800F4FEA400018BF80F0D2
:10EC4000D80003F1FF3314BF00F0FE00C0B213F090
:10EC5000FF03EFD1A242E9D15DF8044B70470020D9
:10EC6000704700BF0000000000000000000000002E
:10EC700091B110B4094C01444FF0FF3210F8013B40
:10EC80005340DBB2884254F8233083EA1222F5D194
:10EC9000D0435DF8044B704708467047DC17040802
:10ECA000C94382B110B4094C024410F8013B4B40F7
:10ECB000DBB2904254F8233083EA1121F5D1C843E6
:10ECC0005DF8044B7047C843704700BFDC17040869
:10ECD0002DE9F041984604460E4617461EF010FEF8
:10ECE0000546FBF70DF8E36833B1FBF709F8E36875
:10ECF00013B12046FBF75CF8FBF702F8E36813B1A9
:10ED00002046FBF755F843463A4631462046FBF786
:10ED100027F80DB1BDE8F081BDE8F0411EF010BE4E
:10ED2000002070470000000000000000000000000C
:10ED3000434B1A69002A75DB70B5414BDA68D10381
:10ED4000FCD41A6922F480721A611A6942F40072C2
:10ED50001A611A6922F0F8021A61C20703D51A690A
:10ED600042F008021A61860704D5354A136943F058
:10ED700010031361450704D5314A136943F020039A
:10ED80001361040704D52E4A136943F0400313614D
:10ED9000C10641D42A4B1A6942F002021A611A696B
:10EDA00042F480321A61DA68D203FCD41A6922F084
:10EDB00002021A611A6942F0004206461A610028EE
:10EDC0003AD005464FF00064013DEDB228461AF0F6
:10EDD00027FF0444002DF7D130461AF021FF032805
:10EDE00005D80AE00438032804F1040405D923688F
:10EDF0000133F7D06FF00A0070BD0028FCD02378F3
:10EE0000FF2BF7D1204402E02378FF2BF2D101340D
:10EE1000A042F9D1002070BD094A136943F0800374
:10EE20001361B7E70749084A59605A601B69002B0C
:10EE300082DA4FF0FF3070474FF00064CCE700BF3C
:10EE4000003C024023016745AB89EFCD0000000084
:10EE500000293BD02DE9F843074689464FF00008CA
:10EE600008F1010616F0FF0612D034464FF0006597
:10EE7000013CE4B220461AF0D3FE0544002CF7D141
:10EE8000AF4209D3B04608F1010616F0FF06ECD1F7
:10EE90004FF00065AF42F5D24046FFF749FF98B901
:10EEA0004FF000673EB1013EF6B230461AF0B8FEB0
:10EEB0000744002EF7D140461AF0B2FE814502D930
:10EEC000A9EB0009CAE70020BDE8F88300207047DD
:10EED00008B50B4601461846FAF7B4FA002008BDFB
:10EEE0002DE9F043464B1F69002F83B004460E46C0
:10EEF000154679DB424FFB68D803FCD43B6923F409
:10EF000080733B613B6943F400733B6114F003037E
:10EF100023D0A4EB030902A8C3F10408D9F8002008
:10EF200040F8042DA84528BFA8461844424631465B
:10EF3000FAF788FA3B690199314A43F001033B61D2
:10EF4000C9F80010D368D903FCD4136923F0010376
:10EF500044444644A5EB08051361032D23D9A5F1CC
:10EF6000040E4FEA9E0C264A06EB8C07311FA01BAD
:10EF7000136951F8048F43F00103136140F80180D5
:10EF8000D368DB03FCD41369B94223F00103136196
:10EF9000EED104342EF0030E0CF1010C744406EB98
:10EFA0008C0605F0030545B9154A136943F0004383
:10EFB0001361002003B0BDE8F08302A8236840F885
:10EFC000043D2A463146FAF73DFA0D4A0199136984
:10EFD00043F0010313612160D368DB03FCD41369A0
:10EFE00023F001031361DFE70649074A59605A60BD
:10EFF0001B69002BBFF67EAF4FF0FF30DAE700BF92
:10F00000003C024023016745AB89EFCD00000000C2
:10F01000214BDA68D00605D52049CA691020024381
:10F02000CA61D8601C4BDA68910606D51B49CA69CB
:10F03000202042F00802CA61D860174BDA685206F5
:10F0400006D51649CA69402042F00402CA61D86058
:10F05000114BDA68100606D51049CA69802042F0C3
:10F060000202CA61D8600C4BDA68D10507D50B499A
:10F07000CA694FF4807042F00102CA61D860064B41
:10F08000DA68920706D50549CA69022042F02002D3
:10F09000CA61D860704700BF003C0240B83600200B
:10F0A000054B5A69D20705D50449054A99600020E5
:10F0B0009A60704701207047003C02403B2A1908C3
:10F0C0007F6E5D4C000000000000000000000000AA
:10F0D000034A536943F0010353610020704700BFA6
:10F0E000003C0240000000000000000000000000A2
:10F0F00008B50B4B0B4A0021D961D368D903FCD466
:10F10000D368DB0744BF0123D360064BD86810F4F3
:10F11000F97000D108BDFFF77BFF012008BD00BFDB
:10F12000B8360020003C0240000000000000000053
:10F13000044A137843F0020313704CF25030FFF787
:10F14000D7BF00BF143C02400000000000000000D8
:10F1500070B52D4D2B7E012B48D003680446DE0789
:10F160004FF00100287612D4990721D45A072BD4E6
:10F170001B0709D5254B227D197801F0F301197081
:10F1800019780A431A70002000232B7670BDD4E949
:10F19000013683424CF250302AD0FFF7A9FF18BB4A
:10F1A0001B4A236811880E43B6B299071680DDD535
:10F1B0004CF250302669FFF79BFF10B9154BF6B2A1
:10F1C0001E7023685A07D3D54CF25030267EFFF7C5
:10F1D0008FFF38B90D4A137826F01F0603F01F037E
:10F1E0001E4316702368C3E72368BDE7022070BD85
:10F1F000FFF77EFF0028F7D1054923680A8822EA35
:10F2000006060E80B0E700BFB8360020143C02406E
:10F21000163C0240153C02400000000000000000C7
:10F220000C4B0D4A1B8883600F2101601378DBB201
:10F23000CC2B04D01378552B14BFAA235523074A8F
:10F240000361536923F01F030376137D03F00C035E
:10F2500043617047163C0240153C0240003C0240AE
:10F2600010B558B907480479053C18BF0124FFF7C9
:10F2700007F908B144F00404204610BD01242046DB
:10F2800010BD00BF3088002000000000000000001A
:10F29000FFF7E6BF000000000000000000000000D3
:10F2A000D8B970B5104E1D463379052B01D0032017
:10F2B00070BD0C4630461146FCF702F858B915B936
:10F2C0000DE0013D0BD021463046FCF729F804F54E
:10F2D00000740028F5D0012070BD0420704702485A
:10F2E000BDE87040FCF76CB83088002000000000DA
:10F2F00000BBF8B5144D1E462B79052B01D0032019
:10F30000F8BD28460C461746FFF7BAF8A0B93946AB
:10F310002846FCF75DF858B916B90FE0013E0DD04C
:10F3200021462846FCF784F804F500740028F5D03F
:10F330000120F8BD042070470220F8BD0248BDE856
:10F34000F840FCF7E5B800BF30880020000000005E
:10F3500020B900290CBF002004207047042070470A
:10F3600030B40468DCB125781F2D0BD93A2D16D0A6
:10F37000234602E03A2A08D00B465A781F2A03F1A6
:10F380000101F7D8002030BC70470134A14206D1FA
:10F39000302D04D10233036030BC002070474FF0A1
:10F3A000FF3030BC704700BF0000000000000000CC
:10F3B000D8B110B5036882B004462BB11A781AB1DF
:10F3C0008088DA88904204D0092000230B6002B0C4
:10F3D00010BD58780191FFF75BFF10F00100019913
:10F3E000F2D123680B6002B010BD002309200B602E
:10F3F000704700BF00000000000000000000000097
:10F4000000232DE9F04BD0F800808B76826B002A28
:10F4100075D098F80020042A0D46064671D0C26CBB
:10F42000013200F0A280D8F80C201088D0B11C4620
:10F4300002270FE0FF288ABF9A762346631C1F2B02
:10F4400005EB03020ED89076D8F80C20D05B5C1C3C
:10F45000023740B140F2523103F0FAF82B19020A98
:10F460000028E7D100242B1900229A76AC7EF66B97
:10F47000002106F10B0C32464FF02E0812F8013B2A
:10F48000202B1CD0052BA2EB060708BFE523092F74
:10F4900000F0B9806818437384B9A3F1410EBEF13E
:10F4A000190F0AD8082F96F80CE08CBF10270827F0
:10F4B0001EEA070F1CBF2033DBB2837601316245A1
:10F4C000DCD1681824B98476337B002B08BF28462A
:10F4D00000214173F37A2B73F08B727F337F696065
:10F4E00042EA002243EA02232B60318BF27DB37D96
:10F4F00042EA012243EA02231A0C6B812A81BDE809
:10F50000F08BD8F8107097F8232082B31C461E4663
:10F510004FF0400810E0731C91761F2B05EB03029F
:10F5200004F1010403F1010608F102081FD89076E6
:10F5300097F823309C421DD218F01F0F08BF08F126
:10F54000020807EB080317F80820587840F25231F8
:10F5500042EA002003F07CF8FF2805EB06024FEAA0
:10F560001021D8D818B13346D7E71C467FE73F2390
:10F57000AB760126AB1900229A766A733B792B731E
:10F58000DB063DD4F96B97F83B000B0E0A02002115
:10F5900041EA030940EA02084FEA092343EA1863F3
:10F5A00097F83A00002141EA03094FEA082240EAAD
:10F5B00002084FEA092343EA186397F8390000214B
:10F5C0004FEA082241EA030C40EA020B4FEA0C29F9
:10F5D00097F8380049EA1B694FEA0B28002148EAEE
:10F5E000000249EA0103C5E900237A7B3B7B43EA39
:10F5F00002236B81FA7BBB7B43EA02232B817EE7EC
:10F6000000220023EFE768180CB980F81A8080F810
:10F610000D8001313EE700BF000000000000000047
:10F6200038B5851C0088A0B1002403F051F8C3B29E
:10F6300003EB540303EBC4339AB2030A03EB520304
:10F6400035F8020B03EBC2339CB20028EDD1204603
:10F6500038BD0446204638BD000000000000000010
:10F660000A44013811F8013B00F8013F9142F9D1F9
:10F67000704700BF00000000000000000000000014
:10F6800070B500F138060446426B407831460123DC
:10F69000FFF72EFE60B9616BA36A226AE070CB1A95
:10F6A0009342054602D2A378022B03D0284670BDB0
:10F6B000012070BD0A44607831460123FFF718FE2F
:10F6C000284670BD0000000000000000000000009F
:10F6D000F8B5C37805460E465BBBEA69B31E023A2D
:10F6E000934224D26E892A6B03FB062605F1380764
:10F6F0006E633B4605F50E71002203F8012B8B4229
:10F70000FBD16889044670B1002403E068890134A4
:10F71000A04208D90123321939466878FFF7E8FD7D
:10F720000028F3D06889201A18BF0120F8BD0026F0
:10F73000DCE7FFF7A5FF0028CFD00120F8BD00BF10
:10F7400070B5C37805465BB92B78032B0FD0002228
:10F7500068781146FFF7FCFD003018BF012070BD2E
:10F76000FFF78EFF0028FAD12B78032BEFD12B79EE
:10F77000012BECD105F138010B4605F50E72002482
:10F7800003F8014B9A42FBD1D5E90530060A85F80A
:10F79000200285F82162060C000E6A6A85F8226252
:10F7A00085F823021E0A180C85F824321B0E85F8F2
:10F7B000256285F826025526AA2085F8273252238D
:10F7C000013285F8366285F837026126412085F8D6
:10F7D000383085F83930722385F83B0085F81E02F1
:10F7E00085F81C3285F81D326A6385F83A6085F821
:10F7F0001F6201236878FFF77BFD2C71A7E700BF2C
:10F8000038B5C37804460D4613B1FFF739FF70B918
:10F810002A46012304F138016078FFF741FD0028F2
:10F8200018BF4FF0FF3565630CBF0020012038BDC5
:10F830002DE9F0478E1E06F007044FF00108016B1A
:10F8400008FA04F401EB1631074615469946E4B26E
:10F85000C6F3C8067B6B994201F1010A03D0384612
:10F86000FFF7CEFF48BBBA1992F838100C4214BF0C
:10F87000012300234B4581EA04014FEA440413D0DD
:10F88000013D82F8381087F8038010D014F0FF048F
:10F89000ECD10136B6F5007F07EB06024FF001040C
:10F8A00008D092F83810E1E70220BDE8F08728463A
:10F8B000BDE8F08751460026CCE70120F5E700BF00
:10F8C000012914D9F8B50568EB698B420DD92B785D
:10F8D000013B0C46032B08D8DFE803F031240B0270
:10F8E000D0E9042352EA030150D10120F8BD0120E0
:10F8F0007047A96A6B6B01EBD411994203D028467B
:10F90000FFF77EFFC0B9A10001F4FE7138356B1816
:10F91000685C5A885C7844EA022440EA042020F0BB
:10F920007040F8BDA96A6B6B01EB1421994223D09A
:10F930002846FFF765FFF8B14FF0FF30F8BDAB6A1E
:10F94000686B01EB510703EB5721814243D1C7F3A9
:10F95000080201372A4403EB5721814292F83860AC
:10F9600041D1C7F308073D44E30795F8380046EA5C
:10F9700000203ED50009F8BD610001F4FF71383563
:10F980006B18685C5C7840EA0420F8BDC679816831
:10F99000022EA4EB01012FD0032E3DD0C369002B12
:10F9A0003ED1A96A6B6B01EBD411994204D0284671
:10F9B000FFF726FF0028BFD1A30003F4FE733835FC
:10F9C000EA18E85C5188537843EA012340EA0320AF
:10F9D00020F00040F8BD2846FFF712FF0028ABD109
:10F9E000AB6A686BB3E72846FFF70AFF0028B8D078
:10F9F000A2E7C0F30B00F8BD12F1FF3643F1FF3769
:10FA0000720A688942EAC752B2FBF0F291423FF6AD
:10FA10006CAF05D0601CF8BD83698B42BED9F9E795
:10FA20006FF00040F8BD00BF0000000000000000C3
:10FA3000F8B506683378042B14BF4FF400124FF06A
:10FA400080528A4225D9CA060C4622D181680463B5
:10FA5000054609BB022B02D9F36AC171DBB93389B0
:10FA6000B3EB541F15D9F36AAB6369638BB1C4F36D
:10FA70000802383603EB54241644C5E90E4600202C
:10FA8000F8BDF369023B8A1E9A421BD30023C5E9E5
:10FA90000D130220F8BD194677897F02BC4207D2B8
:10FAA000EFE70128F5D9F3698342F2D9A742E9D8F3
:10FAB0002846FFF705FF431C0146A4EB0704F0D1DD
:10FAC0000120F8BD7389306B02FB0303AB63CCE705
:10FAD0004FF0FF330022994270B50446C270436371
:10FAE00020D194F8371294F836324AF6552243EA78
:10FAF0000123934214D194F838602449A6F1EB0312
:10FB000004F1390204F1430593B912F8013B11F8ED
:10FB1000010FAA42A3EB0003F6D14BB9012070BD3F
:10FB2000032070BDFFF76CFE0028DAD0042070BD02
:10FB3000E92E05D0A36B164A03F0FF1393420DD1B3
:10FB400094F86E30462B0BD194F86F30412B07D1CF
:10FB500094F87030542B03D1002070BD022070BD8A
:10FB600094F88A300B4904F18B02463B8F34002B0A
:10FB7000F4D112F8013B11F8010FA242A3EB0003EC
:10FB8000F5D1002B14BF0220002070BD6C1C0408AE
:10FB9000EB009000781C040800000000000000004A
:10FBA0002DE9F04F002385B00B600F461546FFF797
:10FBB000D7FB061EC0F2C880864B53F82640002CA7
:10FBC00000F0EF803C60237805F0FE057BB16078A3
:10FBD000FFF75EFBC7070AD4002D00F0B38010F0DA
:10FBE000040000F0B2800A2005B0BDE8F08FF0B24A
:10FBF000002360702370FFF733FBC60700F1A88075
:10FC00000DB14507EFD400212046FFF761FF022820
:10FC100000F0A280042800F0CF80012800F2BD800F
:10FC20000026012894F8432000F0C88094F844305E
:10FC300042EA0322B2F5007F40F0AF8094F84F20F3
:10FC400094F84E3053EA022309D1B4F85E1094F8C8
:10FC50005D3094F85C2043EA012342EA032394F8E0
:10FC600048202362511E0129A27000F2968094F868
:10FC7000451088B26081002800F08F80481E08423D
:10FC800040F08B8094F84A0094F8495045EA0025EA
:10FC90002807258140F0818094F84C7094F84B003F
:10FCA00050EA072009D1B4F85AC094F8597094F872
:10FCB000580047EA0C2740EA072094F847C094F818
:10FCC000467057EA0C2C68D003FB02FE0CEB1517AC
:10FCD0007744B84261D3404AC01BB0FBF1F1481EE3
:10FCE00090425AD84FF6F57841450CEB0600374460
:10FCF00001F1020200F24B8140F6F57C6145E261C0
:10FD0000C4E90960276300F23A81002D45D002EB77
:10FD10004201704402F0010202EB5102E062012153
:10FD200002F2FF12B3EB522F37D34FF0FF33C4E987
:10FD3000053380222271294A2170138801339BB236
:10FD40001380E380002000E00B2005B0BDE8F08FB9
:10FD5000032005B0BDE8F08F6D46294604F5007319
:10FD600004F5107613F8062C42B11F8813F8010C25
:10FD700013F8022C40EA072042EA00221033B34273
:10FD800041F8042BEED105F1100755F8046B66B964
:10FD90000320BD42F9D104280ED00D2005B0BDE8E6
:10FDA000F08F0C2005B0BDE8F08F31462046FFF7FC
:10FDB0008FFE0128EDD834E70120C6E704F14303A4
:10FDC00004F17701002AE8D18B4209D013F8012F02
:10FDD000F8E700BFD8360020F4FFFF0FDC36002024
:10FDE00094F8A12094F8A03043EA0223B3F5807F71
:10FDF000D3D194F8A430092BCFD1D4F8841094F83F
:10FE000083000B0E0A02002141EA030840EA0207C0
:10FE10004FEA082343EA176394F88200002141EA7D
:10FE200003083A0240EA02074FEA082394F88100E7
:10FE300043EA17633A02002140EA020941EA030A51
:10FE400094F880004FEA0A284FEA092748EA19681F
:10FE5000002147EA000212EB060A48EA010343F1D7
:10FE6000000BBBF1010F08BFBAF1000F95D2B4F837
:10FE70008E5094F88D0094F88C1040EA052094F888
:10FE8000A650A57041EA0021012D216285D194F888
:10FE9000A5108D40A9B2618100293FF47EAFB4F86E
:10FEA000967094F8951094F8940041EA0721754FE4
:10FEB00040EA0120B8423FF670AFB4F8928094F85F
:10FEC00091C094F8901094F88970B4F88AE0666252
:10FED0004CEA082C41EA0C21ADB2314400FB05FC90
:10FEE00011EB0C0847EA0E2E4FF0000394F88870CF
:10FEF000216343F1000947EA0E27CB453E4408BF82
:10FF0000C24500F10207A662E761FFF446AFB4F80C
:10FF10009A6094F8992094F8983042EA062243EACD
:10FF200002239A1E9042E362636B8CBF02FB0511B1
:10FF300000218B4205D02046FFF762FC00287FF4A9
:10FF40003BAF04F14E0304F24E2103E0203399420B
:10FF50003FF423AF13F8162C812AF7D11D8813F82C
:10FF6000010C13F8022C40EA052042EA0022022A82
:10FF7000ECD14FF0FF33C4E905330421DBE6002D5B
:10FF80003FF40BAF7044E06252000221C8E694F8DF
:10FF900063C094F86210E26151EA0C21C4E909607F
:10FFA00027637FF4FAAE002D7FF4F7AEB4F8665005
:10FFB00094F8650094F86410920040EA052002F27B
:10FFC000FF1241EA0021B3EB522FE162FFF4E5AEEC
:10FFD00094F8691094F8683043EA01234FF0FF3237
:10FFE0008021012BC4E90522217101D00321A2E661
:10FFF000636B711C994204D02046FFF701FC002876
:020000040801F1
:10000000F4D194F8372294F8363243EA02234AF6C0
:100010005522002193422171E8D1608F94F8392054
:1000200094F83830184942EA002243EA02238B420E
:10003000DCD1B4F81E0294F81D2294F81C3201F1B0
:10004000FF5101F5005142EA0022203143EA022328
:100050008B42CBD1B4F8226294F82102B4F8265234
:1000600094F8251294F8202294F8243240EA0620CD
:1000700041EA052142EA002243EA0123C4E90532AC
:10008000B4E700BFFDFFFF7F525261410000000056
:100090002DE9F84304460078431E0D461646032B0F
:1000A00000F29A80DFE803F03D240202A16A636B4C
:1000B00001EBD511994267D1AD0005F4FE7504F14D
:1000C0003801042801EB050306D05A88120426F0F3
:1000D000704602F0704216434E55300A320C012130
:1000E000360E58709A70DE70E1700020BDE8F8831B
:1000F000A16A636B01EB1521994203D02046FFF7FB
:100100007FFB60B96D0004F1380305F4FF755A19DF
:100110005E55C6F30721012351700020E370BDE84E
:10012000F883A16A636B05EB550701EB57219942F0
:1001300031D107F10108EB07C7F308074FEA58214F
:1001400004F138092DD519F8073003F00F0343EAFD
:10015000061309F80730A26A636B114499424FF005
:100160000102E27004D02046FFF74AFB0028D6D1F6
:10017000C8F30808C844C6F30716012388F80060CE
:10018000E3700020BDE8F8832046FFF739FB002824
:10019000C5D1207890E72046FFF732FB0028C8D071
:1001A000BDE709F80760A26A636B114499424FF0FA
:1001B0000102E2700AD1C8F30808C844C6F303225A
:1001C00098F8003023F00F061643D6E72046FFF7D5
:1001D00017FB0028A3D1EEE70220A0E700000000F3
:1001E00001295CD92DE9F8430568EB698B420C467F
:1001F000074646D99146002A3AD1A04603E0B046C8
:100200008E4234464DD221463846FFF759FB06460A
:10021000002846D0012834D0411C47D02B78042B2D
:100220000AD0012C2DD9EB699C422AD2002221460A
:100230002846FFF72DFF28BBD5E906318A1E9342D9
:1002400005D22A79013342F00102AB612A710134EF
:10025000B442D5D02B78042BD1D1A4EB080241466F
:1002600000232846FFF7E4FA60B9E969B046C7E71A
:100270002A78042A02D1C279022ABED0B9F1010F2C
:1002800002D80220BDE8F8834B45FAD94FF0FF327F
:1002900049462846FFF7FCFE0028AED0F2E70220D0
:1002A00070472B78042B03D00020EBE70120E9E70F
:1002B000B9F1000F14D0FB79B3B9BC680BE021464B
:1002C0003846FFF7FDFA631C01281C46D9D9421CA9
:1002D000ECD08342E8D1A145F1D10223FB71E3E7E1
:1002E00087F807904846CDE7032BDDD1BB684B4527
:1002F000DAD8BA6913444B45EFD2D5E700000000C5
:10030000F8B50C460968E1B1064615461F460AE0F5
:10031000DCF81CC0634512D2FFF7BAFE80B9216831
:100320000139216069B16A1A531C0129D6F800C04D
:100330008CBF02323A46012B19466046E8D80220AB
:10034000F8BD0020F8BD00BF000000000000000064
:10035000836970B506468568E3B1012D006805F133
:10036000010415D9C269954212D21D4408E0A54284
:1003700010D0012C30680BD9C269A24208D91C46A2
:100380002246611EFFF784FE631C0028EFD070BD7B
:10039000022070BD0020F07170BD00BF00000000A1
:1003A0002DE9F84F074688460668002958D1756937
:1003B000002D4DD0F369AB4298BF0125B369002BE6
:1003C0004AD03278D6F81CC0042A634675D0454519
:1003D00058D02C4606E0012850D0013068D0AC42FD
:1003E0003AD0F36901349C42384602D3012D33D907
:1003F00002242146FFF764FA0028ECD1012C3DD9F4
:10040000F3699C423AD24FF0FF3221463046FFF763
:100410003FFE88BBB8F1000F0BD0B8F1010F2DD90A
:10042000F36998452AD2414622463046FFF730FE0E
:1004300010BBD6E90623023B9A423379746198BF18
:1004400002F1FF3243F0010398BFB261337104E05F
:10045000B3690125002BB4D100242046BDE8F88FF4
:10046000FFF72EFA0128044608D9421C20D0F36970
:100470008342F2D84546A1E7012819D0012420463D
:10048000BDE8F88F6C1C644528BF0224214638461D
:10049000FFF716FA0128F1D0431C09D000286AD0D2
:1004A0007269F369012A94D99A4238BF154690E7D8
:1004B0004FF0FF342046BDE8F88FA5F10209ACF1FA
:1004C0000203994528BF4FF000094C464FF0010A3E
:1004D000D6E90C1301EB1431994206D03046FFF7F0
:1004E0008FF90028E4D1D6F81CC0C4F3C80B06EB82
:1004F0000B0204F007030AFA03F392F83800DBB2A8
:10050000ACF1020E621C724503EA000117D361BB15
:10051000033204F10204A0D801231A4621463046D2
:10052000FFF786F90228A9D00128C1D0B8F1000F41
:1005300026D10223FB7100283FF47BAF9EE75B00CE
:100540000029E5D04A4587D013F0FF0301D01446B7
:10055000D8E70BF1010BBBF5007F06EB0B0339D09D
:1005600093F8380014460123CCE7B9F1000F3FF4AB
:1005700073AF0024ACE7002C7FF440AFF36928E7A9
:10058000FB79022B1BD008F10103A342FA690FD0BB
:100590000AB90123FB614246234607F11C01384694
:1005A000FFF7AEFE00287FF467AF0123FB6140E751
:1005B00072B10132FA6100283FF43BAF5EE76B1C79
:1005C000A342B8D0BB680322EB1ABB61FA71DAE729
:1005D0000222EFE714467BE7000000000000000065
:1005E000826B22B3F0B50568046B2E78042E14BF1D
:1005F0004FF400164FF080562034A64283B00346D5
:1006000012D9C4F308070E463FB9416B0132826329
:1006100079B92A89B2EB541F40D938353D440020BE
:10062000DD631C6303B0F0BD042003B0F0BD042003
:1006300070476A89013A12EA5422EED10090FFF71E
:100640003FF901280246009B2ED9411C2AD0E969B6
:10065000814217D816B3596B00931846FFF7A0FED6
:1006600020B3012820D0431C1CD00146019028460D
:10067000FFF72EF8B0B9009B019AD97941F0040137
:10068000D971E9695A630239023A8A423BBF6989E2
:10069000286B002202FB01029A63BEE700229A63E4
:1006A0000420C2E70120C0E70220BEE70720BCE724
:1006B0002DE9F04104460068A16B436B076999423C
:1006C0005AD1E16B0B78852B03D002252846BDE873
:1006D000F08120223846FEF7C3FF7E78013676018E
:1006E000A6F16003B3F5007FEFD800212046FFF7A5
:1006F00077FF04280546E8D00028E7D12068A16BE1
:10070000436B994240D1E16B0B78C02BDDD12022A5
:10071000B818FEF7A5FF97F823302E4A2C33A2FB1A
:100720000323DB08B6EB431FCFD34FF0400803E0B1
:1007300008F1200846452DD900212046FFF750FF3B
:1007400004280546C1D00028C0D12068A36B426BA5
:100750009342194603D0FFF753F8002838D1E16BD4
:100760000B78C12BB1D1B8F19F0FE1D8202207EB54
:100770000800FEF775FFDBE7FFF742F805460028A3
:100780009FD02846BDE8F081FFF73AF805460028DB
:10079000B9D09BE7B8F1A00F98D878780021013044
:1007A00040010B4602E0022B08BF0423FA5C02EB77
:1007B000C13292B2013302EB5101984289B2F2D8B0
:1007C000FA78BB7843EA02238B423FF47FAF7CE7A1
:1007D00005467BE78988888800000000000000004B
:1007E0002DE9F0418846002104460568FFF720F90D
:1007F0000746E8B90646A16B6B6B994203D02846C1
:10080000FEF7FEFF98B92A78E36B042A1B7817D00D
:10081000E52B03D0B3FA83F35B097BB10136464580
:1008200009D001212046FFF7DBFE0028E3D0074670
:10083000042F08BF07273846BDE8F0811E46F0E7C1
:10084000DB43C3F3C013E8E7000000000000000032
:100850002DE9F84303681D696E7804460022701C78
:100860004001134602E0022B08BF0423E95C01EBC0
:10087000C23189B2013301EB5202984292B2F2D8EE
:10088000130AAA70EB70E16C2046FFF7D1F881469D
:1008900048BB07464FF0010804E0FFF7A1FE2035F2
:1008A0000137C0B92068A36B426B9342194602D04E
:1008B000FEF7A6FF78B92946E06B2022FEF7D0FEAE
:1008C0002368BE424FF00001204683F80380E4D144
:1008D0004846BDE8F883022828BF02205FFA80F965
:1008E0004846BDE8F883022828BF4FF002095FFAA6
:1008F00089F9EDE7000000000000000000000000A2
:10090000C16C4B1C2DE9F04104460568066B2AD1E9
:100910004FF0E50801270BE083F80080EF70236BB0
:10092000B3424FF0000120461AD2FFF759FE00BB38
:10093000A36B6A6B93422846194602D0FEF760FF0C
:10094000B8B92A78E36B042AE6D11A7802F07F025C
:100950001A70EF70236BB3424FF000012046E4D3CE
:100960000020BDE8F081FFF763F80028D0D0BDE893
:10097000F081042808BF0220BDE8F08100000000DB
:100980002DE9F047FF26044607683546042011E0AC
:10099000CA7AE52B02F03F02A27105D02E2B03D0BC
:1009A00022F02000082823D1FF2500212046FFF750
:1009B00017FEC8B9A16B002957D07B6B8B4203D0BF
:1009C0003846FEF71DFF78B9E16B0B78002B51D04C
:1009D0003A78042ADCD1852BE7D1236BE3642046E7
:1009E000FFF766FE002847D00023A363BDE8F08729
:1009F0000F2A47D15A0635D5226B4E7BE26403F0AD
:100A0000BF054B7BB342CFD1CA7E8B7E53EA022314
:100A1000CAD10A782B48D7F80C8022F04002013A5C
:100A200002EB420C012302EB8C0200F10C0E9C46FF
:100A30004FF6FF7909E01F2AB6D828F812309C46F5
:100A40000132864531D010F8013F01EB030ACB5C3F
:100A50009AF801A043EA0A23BCF1000FEBD14B4501
:100A6000EFD0A1E7AB429FD1CBE70028BCD100205B
:100A7000BDE8F0870420B7E73B691B7903F03F032B
:100A8000A371B3E76DB901F10B0011F8012BEB0174
:100A900043EA550552FA85F58142EDB2F5D1B542EA
:100AA000E5D04FF0FF33E364E1E70B785B0605D553
:100AB0001F2A3FF679AF002328F81230013DEDB22E
:100AC00073E700BF5C1C0408000000000000000089
:100AD0002DE9F04F002187B005460768FEF7A8FF13
:100AE000814600284CD13B78042B00F0BB804FF0AE
:100AF000FF334FF0FF0BEB649846DA460CE00F2B08
:100B000042D0C5F84C804FF0FF0A00212846FFF77D
:100B100067FD002840F09C80A96B7B6B994205D053
:100B20003846FEF76DFE002840F09280EC6B267888
:100B3000002E00F0D680E27AE52E02F03F03AB7182
:100B4000DFD01207DBD40F2B1ED0BAF1000F6DD00F
:100B500095F84B30DB07D4D42046294610F80B3BE0
:100B600011F8402F01349B1A002BCAD114F8013B15
:100B700011F8012F8442A3EB0203F5D1002BC0D161
:100B8000484607B0BDE8F08F95F84B305806BCD406
:100B9000710662D52B6B94F80DB0EB6406F0BF06BE
:100BA000637B5B455BD1E27EA37E53EA022356D191
:100BB0002378F968594A049103F03F03013B03EBA2
:100BC000430003EB80030121CDE900B7CDE9029595
:100BD000049F0596254692461C460B4611E01F2CA5
:100BE0001DD801F075FD834637F8140001F070FD43
:100BF000834514D133464C46494A524577D01AF8BA
:100C0000011F6E5C681804F10109407846EA00266D
:100C10003046002BE3D14FF6FF729642ECD0DDE96F
:100C200000B7DDE902954FF0FF0A6EE704F10B0013
:100C3000214611F8012B4FEACA1343EA5A0A52FA25
:100C40008AFA81425FFA8AFAF3D1D34580D197E7D5
:100C50008146484607B0BDE8F08FB245A0D04FF0BE
:100C6000FF0A52E7F868FEF7DBFC80462846FFF7EC
:100C700087FE0028ECD13B6993F82360202EF5D83D
:100C800093F8251093F8242042EA01229045EDD1F3
:100C900016B306F1FF3A5FFA8AFA0AF1010A06462C
:100CA000402400E03B69E10608BF02341A191B5DCD
:100CB000507843EA002001F00BFDFB68834633F8CF
:100CC000160001F005FD834506F1010604F102045A
:100CD000CCD15645E6D17600FB689B5B002BC5D195
:100CE0004EE74FF00409484607B0BDE8F08F9C4638
:100CF00023462C46DDE900B72278059E5206DDE941
:100D0000029507D5BCF1000F04D0049A32F81330D5
:100D1000002BA4D1013E5FFA86FAF6E65C1C0408BB
:100D2000681C040800000000000000000000000033
:100D30002DE9F04FD0F800B087B007460D4611F806
:100D4000013B2F2BFAD05C2BF8D00021B960F96160
:100D500028781F2840F28C8103915B4680B21F28BF
:100D6000D3F80C8046D92F282CD05C282AD0A8F1A3
:100D700002092E4601240FE029F8020F16F8010F90
:100D80001F2804F1010340F252812F281CD05C2857
:100D90001AD0212B12D01C4640F2523101F080FCB7
:100DA00060B17F28E8D8222808D0CC4A2A2303E063
:100DB00012F8013F002BDFD09842F9D1062007B08E
:100DC000BDE8F08F002401232B441A782F2A1D46FA
:100DD00003F10103F9D05C2AF7D05CB14FF00009B0
:100DE00008EB440232F8023D202B01D02E2B05D116
:100DF000013CF7D10023A8F80030DFE7039B28F877
:100E0000143008EB440207F1400307F14B002021A6
:100E100003F8011B8342FBD1A8F10203002600E086
:100E2000013633F8020F2028FAD02E28F8D00EB160
:100E300049F00309134633F8022D2E2A01D0013C54
:100E4000F9D100239A460822013668B320287AD0C7
:100E50002E2800F0CC8093421CD2A64200F0C9801C
:100E60007F2800F2E8802B2800F0FA80DFF874C2B7
:100E70002C21814200F0F4801CF8011F0029F8D1D8
:100E8000A0F1410189B2192900F21C814AF0020A3D
:100E9000C0B2E8E00B2A00F00A81A64200F0AB8065
:100EA00049F0030940F2A78097F84030E52B04BFD2
:100EB000052387F84030082A04BF4FEA8A0A5FFA00
:100EC0008AFA0AF00C030C2B00F09D800AF0030A4A
:100ED000BAF1030F00F0978019F0020F08D1BAF1B0
:100EE000010F08BF49F01009042B08BF49F0080999
:100EF00087F84B903846FFF7EBFD97F84B3000280A
:100F000040F08D805A073FF55AAFBB79DB0640F1C0
:100F1000CA809BF8001004291AD03A6B0BF13803F1
:100F2000C2F3080213440329D87E9A7E42EA0022C3
:100F300005D1597D1B7D43EA012342EA0342BA6091
:100F40003B6828780AE749F0030938F816007BE780
:100F50003B69F879FA6CDBF81040B968396223F024
:100F6000FF030343C7E90932E18E94F8352094F872
:100F7000343042EA012243EA0223BB6094F8213074
:100F800003F00203FB71E36B94F83B001A0E1B02A3
:100F900001920093DDE9002300210B4302431B0271
:100FA00043EA126394F83A00002141EA030912026D
:100FB00040EA02084FEA092343EA186394F839002B
:100FC000002141EA03094FEA082240EA02084FEAF9
:100FD000092994F8380049EA186900214FEA0828DD
:100FE00048EA000249EA0103C7E90423A8E7A64248
:100FF000A9D10B2A5BD04FEA8A0A5FFA8AFA264601
:101000000B220823A1E749F0020987F84B903846E4
:10101000FFF75EFD97F84B3000283FF473AF0428CC
:101020007FF4CDAE13F0040F08BF0520C7E61D44C2
:101030004FF00409D4E640F25231CDE9043201F018
:1010400007FB10F0800F49F0020EDDE9043218D0E2
:1010500000F07F002249085CF14600287FF403AFCE
:1010600049F003095F20F918013381F840006CE76B
:101070008023384687F84B3007B0BDE8F04FFEF7C5
:10108000D7BCFF28E8D9511E8B4208D2F9184FEA85
:10109000102CF146013381F840C0C0B2E3E749F0BB
:1010A0000309134651E7052007B0BDE8F08F97F814
:1010B0004030E52B49F003097FF403AF052387F89F
:1010C0004030FEE6A0F1610189B2192997BF2038AE
:1010D000C0B2C0B24AF0010AC5E700BF811C0408D3
:1010E000DC1B04088D1C0408000000000000000048
:1010F0002DE9F04F90F84B3013F0A0089BB040F072
:101100001181D0F800B0DBF80C301A88002A00F00A
:10111000E38133F8022F08F10108002AF9D19BF886
:101120000030042B044677D000F14005294606A87C
:101130000C22FEF795FA9DF82330DE0740F1FE8081
:10114000402384F84B300B2206A928464FF00109B2
:10115000BC4FFEF785FA4B460DF11706072203F048
:101160000F0000F13001392988BF00F137011B0958
:1011700002F1FF3206F80119F1D11AA911447E20BB
:1011800001F8580C002A00F0088194F8401020293A
:1011900008D0294603E011F8010F202802D00133BE
:1011A0009A42F8D1591E29441AA81044072A03F17B
:1011B000010396BF10F8580C20200132072B01F8CC
:1011C000010FF1D92046FFF783FC002840F0AF80E3
:1011D00009F10109B9F1640F00F0F9810B2206A9A8
:1011E0002846DBF80C60FEF73BFAB9F1050F40F238
:1011F0009780023E4B4636F8022F002AACD01021D1
:1012000002F0010000EB4303D80348BF7B400139E3
:101210004FEA5202F4D1EEE78B4D08F10E03A5FB25
:101220000323DD08A91CFFF7DBFA0646002873D16B
:1012300005F10063216BE2790133A1EB4313E36411
:10124000530714D502F0FB03032BE37100F0B781C1
:101250004FF0FF33626B04F11C012046FFF750F89A
:10126000002840F0A581A368002B40F03D81DBE918
:101270000308002208F14001434603F8012B8B428A
:10128000FBD14FF0000A8522C02388F8002088F89F
:101290002030D6465546D346012240214C1C6FF0E3
:1012A0003E0308F8013008F804B05FFA8AF408EB4E
:1012B00001030194023115E030F815200EF1010907
:1012C000D4B2170A002A00F005815FFA89FE0FFAEE
:1012D0008EF500EB450C0231DF70CF069C7003F1F8
:1012E000020306D000EB450C002AE5D11746144650
:1012F000F1E7BCF800300AF1010A002BCED1019BC6
:1013000088F823E0023388F80130FEF789F9030AF0
:1013100088F8240088F8253030461BB0BDE8F08FEF
:101320004B4619E7062630461BB0BDE8F08F04286F
:101330000646F1D19DF8233084F84B309B072ED41C
:1013400001212046FFF74CFA06460028E4D1A16BA4
:10135000DBF83430994205D05846FEF751FA06467C
:101360000028D9D1E36B002103F1200203F8011B0F
:101370009342FBD12946E06B0B22FEF771F994F8FA
:101380004B30E16B002603F01803012230460B734B
:101390008BF803201BB0BDE8F08F134602E72B4A01
:1013A00008F10C03A2FB03239B08591C20461F468F
:1013B0000193FFF715FA06460028ADD1002FC6D0DD
:1013C000216B2046A1EB4711FEF732FB06460028B1
:1013D000A2D10246294604F14B00D30111F8016B5A
:1013E00043EA520356FA83F38142DAB2F5D1DFF8C9
:1013F00060A002920395A16BDBF83430994205D0CE
:101400005846FEF7FDF9002840F0D2809DF8049080
:10141000E16B029EDBF80CE04E7309F1FF32002510
:1014200002EB42004FF00F060D732B4602EB8002D9
:101430008D762846CD76CE7201254FF6FF784FF097
:10144000FF0C20E021100100898888884FECC44EF1
:101450005C1C04083EF812304B551D0A01327D70A9
:10146000002B40F0AA800C2E21D81AF80630CD1897
:1014700001F803C0023085F801C04FF6FF730C2855
:101480000ED81AF80050434501EB050700F101069C
:10149000E0D130460C2801F805C087F801C0F0D92A
:1014A0004FF6FF70834202D03EF812300BB949F07C
:1014B0004009012381F80090204600218BF8033079
:1014C000FFF78EF8002873D1019B013B019392D165
:1014D000039D3CE71446FEE69BF80030042B904643
:1014E00004467FF421AE97E6D4E909158DF81F1064
:1014F00021F0FF012268236A0B900D900A9106A843
:101500002946199506920893FEF792FA00284FD1C2
:1015100006A8FFF7CDF800284AD1D4E90423BBF888
:101520000A50DBF810104FF40070E0FB052317465B
:101530009846C4E90478150A100C81F8395081F8EE
:10154000382081F83C3081F83A00150E180A1A0C40
:101550001B0E81F83B5081F83D0081F83E2081F858
:101560003F30D4E90412DBF81030080A83F8290070
:1015700083F8281083F82C20100A0F0C0D0E110C84
:10158000120E83F82D0083F82A7083F82B5083F80D
:101590002E1083F82F20E379DBF8102043F00103AD
:1015A00006A882F82130FFF753F900283FF45FAE18
:1015B000064630461BB0BDE8F08F30465FE7204658
:1015C000FEF7C6FE00283FF443AE0646F1E70726C5
:1015D000A2E600BF000000000000000000000000C4
:1015E00010B584B004AB019043F8041D1846009177
:1015F0001446FDF7B5FE002816DB0D4A52F82030E0
:101600000BB100211970019B0BB10021197042F838
:10161000203014B9204604B010BD002201A968464C
:10162000FEF7BEFA04B010BD0B2004B010BD00BF21
:10163000D83600200000000000000000000000007C
:101640002DE9F04FD1B0019168B302F03F06044696
:10165000174602A9324601A8FEF7A2FA054628B1AC
:1016600000232360284651B0BDE8F08FDDE9011367
:1016700003A828AAC3E9030214A81493FFF758FB90
:1016800007F01C03A0B99DF99B20002AC0F2CF806F
:101690009DF856208BB112F0110F16D17B0740F147
:1016A0001F810825DCE70925284651B0BDE8F08FE9
:1016B0000BB104280DD00546D2E7D30607D4B907ED
:1016C00040F1AE80D30740F1AB800725C8E7042581
:1016D000C6E714A8FFF70CFD46F008060028EAD17B
:1016E000029B1978042900F01E81239AD07E977EF0
:1016F000032947EA002705D1507D117D41EA0021E9
:1017000047EA014700214A204FF0A10C5074917321
:10171000D17382F810C0239A2020D072239A917638
:10172000D1761878032801D11175517523990022BB
:1017300001200A774A778A77CA77D870002F00F09D
:10174000648114A83946D3F83480FEF749FD002897
:10175000B1D1029B5A6B904507F1FF3740F065818C
:101760005F61197846F04006239A0429C4E9128281
:101770005FD0D77E907E032940EA072005D1577DB0
:10178000117D41EA072140EA0140A060D08B517FE2
:10179000127F41EA002142EA01220021C4E904212A
:1017A00000200021DA88A280C4E90E0104F1500A69
:1017B0000021236084F8306084F83110616452465F
:1017C00004F5147002F8011B8242FBD1B1067FF5CB
:1017D00049AFD4E9046756EA07023FF443AFB3F8D0
:1017E0000A80A1684FF000094FEA4828B94508BFB0
:1017F000B045C4E90E670AD37AE0421C6ED0B6EB5E
:10180000080667EB0907B94508BFB04570D2204606
:10181000FEF756F801280146EFD8022521641FE79C
:10182000029B3807D3F8348019789DD59AE70625AE
:1018300016E718999DF857C027981A69169F2762CE
:1018400021F0FF0141EA0C01C4E90910D78E92F89A
:10185000350092F8341040EA072041EA0021A160E7
:10186000D16B92F83B004FEA11694FEA0128002141
:1018700041EA090B40EA080A4FEA0B2992F83A00BC
:1018800049EA1A69002141EA090B4FEA0A2840EAAD
:10189000080A4FEA0B2992F8390049EA1A6900212F
:1018A00041EA090B4FEA0A2840EA080A4FEA0B29E5
:1018B00049EA1A694FEA0A2892F838A04FF0000B5B
:1018C0004BEA09014AEA0800C4E9040192F8212020
:1018D000002102F00202E271E16161E701259DE76A
:1018E000029B380719783FF5FDAED3F834803BE70B
:1018F000002340F2FF1202EA060803EA070958EA49
:10190000090321643FF4AEAE029BDA690239023A60
:10191000914206D25A89186B01FB0202002A40F05C
:101920008B8002259CE61A692360D18E92F835706F
:1019300092F8343047EA012743EA0727A760D36BC0
:1019400092F83B80190E4FF00009180249EA010B8A
:1019500048EA000A4FEA0B2192F83A8041EA1A61FC
:101960004FF0000949EA010B4FEA0A2048EA000A51
:101970004FEA0B2192F8398041EA1A614FF00009D1
:1019800049EA010B4FEA0A2048EA000A4FEA0B2B0A
:1019900092F838804BEA1A6B4FF000094FEA0A2A96
:1019A0004BEA09014AEA0800C4E9040192F821302F
:1019B000002103F00203E371E161931C203203F87C
:1019C000011B9342FBD1029B1A69002102F12603FD
:1019D000403203F8011B9342FBD1029A1369202085
:1019E000187113694FF0A10C4A20D87219725972FC
:1019F00083F80AC01369012283F8212014A8FEF796
:101A000027FF024620B92FB9029BD3F83480A8E6FD
:101A1000054625E639462046FEF7E2FB029B013FDC
:101A20005F610028F0D005461AE618464146FDF7EA
:101A3000E7FE029B5F61F4E7710A41EAC7510A447D
:101A40006264587851460123FDF72AFC00283FF4D0
:101A500009AE012504E600BF000000000000000000
:101A60002DE9F04F1E4687B000238946336005A953
:101A700015460446FDF79CFC804600285ED194F88C
:101A80003180B8F1000F59D194F83030DA0740F1C5
:101A90009D80D4E90E23D4E90401801A4FF0000B95
:101AA00061EB0301594508BFA84238BF0546002D28
:101AB00044D0CDE9002304F15007CDF80C80DDE9D6
:101AC00000AB40F2FF10002152465B460B40024043
:101AD0001046194650EA010349D105995346B1F819
:101AE0000AC0580A0CF1FF3C40EACB501CEA000A3D
:101AF00060D0206CCB690238023B984280F0918024
:101B00004A890B6B02FB0030002800F08A805FEAF4
:101B100055280AEB000B15D00AEB0803934288BF47
:101B2000A2EB0A08487843465A464946FDF7B8FBF7
:101B300000284ED04FF0010884F83180404607B0AD
:101B4000BDE8F08F626C5A450BD094F9303048787C
:101B5000002B4ADB01235A463946FDF7A1FB00283A
:101B6000E8D1D4E90E23CDE90023C4F844B0009BAA
:101B7000C3F30802C2F50078A84528BFA846B918E3
:101B800048464246FDF76CFDD4E90E23316812EB5E
:101B9000080A43F1000B52465B464144B5EB080589
:101BA0003160CDE90023C144C4E90E2387D1DDF8BB
:101BB0000C80C3E7DDE90023134311D1A06801289D
:101BC0002FD9431CB6D00599206493E74FF007083E
:101BD000B4E794F93030002B16DB4FEA4828D3E7FE
:101BE000216C2046FDF76CFEE9E701233946FDF73D
:101BF0007FFB00289ED194F83030059A03F07F03D4
:101C000084F830305078A5E7606CA0EB0B004045BD
:101C1000E3D209EB40204FF400723946FDF720FD76
:101C2000DBE74FF0020884F8318087E7000000000E
:101C30002DE9F04F984685B000238A46C8F8003059
:101C400003A916460446FDF7B3FB074600286DD1ED
:101C500094F83170002F69D194F830309A0740F130
:101C6000C280039A1278042A03D0A26BF24200D3F6
:101C7000D643002E00F0A08004F15003D4E90E01F9
:101C8000CDE9003740F2FF12002300EA020B01EA1F
:101C9000030C5A46634613435AD1DDF80CC0BCF816
:101CA0000A90430A09F1FF3943EAC15319EA0309CB
:101CB00012D150EA010340F09E80A068002800F095
:101CC000A280012800F0C380431C2CD0A3682064AC
:101CD000DDF80CC003B9A06094F93030002B70DB44
:101CE000276CDCF81C30023F023B9F4280F0AF8043
:101CF000BCF80A30DCF8301003FB0717002F00F0A7
:101D0000A680750A4F4415D009EB05029A4288BF98
:101D1000A3EB09059CF801002B463A465146FDF716
:101D2000E7FA002861D0012784F83170384605B001
:101D3000BDE8F08FD4E90E12636CBB420846114631
:101D400005D0D4E90423994208BF904263D3676465
:101D5000C0F30800C0F50075009BB54228BF3546AA
:101D600018442A465146FDF77BFC94F8303063F066
:101D70007F0384F83030D4E90E01D4E9042310EB5A
:101D8000050B41F1000CD8F80070634508BF5A45B7
:101D90002F44584661463CBF5A466346761BC8F8F6
:101DA0000070AA44C4E90E01C4E90423002E7FF4A4
:101DB00069AF019F94F8303043F0400384F830302D
:101DC000B4E79CF80100626C00990123FDF790FADA
:101DD0000028A8D194F83030DDF80CC003F07F0360
:101DE00084F830307CE70727A0E7616CC91BA94263
:101DF0001FD36D02BFE7216C2046FEF7D1FA002801
:101E00007FF45FAFD5E701462046FEF7C9FA002808
:101E10007FF457AFCDE79CF80100009901233A46C3
:101E2000FDF73EFA00287FF47EAFD4E90E2310467A
:101E30008DE70AEB41214FF400720098FDF710FC8A
:101E400094F8303003F07F0384F83030D1E7022774
:101E500084F831706AE700BF000000000000000055
:101E6000F0B5CFB069460446FDF7A2FA0346002854
:101E700043D194F8302051063FD51306009D00F160
:101E8000D2802B78042B3BD0A16C6B6B994205D090
:101E90002846FDF7B5FC034678BB009DE36CDA7A73
:101EA00042F02002DA72A26821689A76C2F3072013
:101EB000D8760978032903D1120C110A1A755975BD
:101EC00022691A77110A100C120E5977987700219F
:101ED000DA774A20A126012258769975D975997426
:101EE000D9741E762846EA70FDF72AFC94F8302053
:101EF00022F04002034684F8302018464FB0F0BD6F
:101F0000E379032B00F0A1804FF0FF33226C04F142
:101F10001C012046FEF7F4F903460028EDD1D4E970
:101F2000092500998DF84F2001A8C86022F0FF0212
:101F300026A80861179319931692236A22681493AE
:101F4000294612A825951292FDF772FD0346002836
:101F5000D3D112A8FEF7ACFB03460028CDD1009ADE
:101F60001069017941F020010171E179106941F0B6
:101F7000010180F82110A0681169070A060C050EFE
:101F800081F8357081F8366081F8340081F8375077
:101F9000D4E9045011692E0A81F8396081F838506B
:101FA00081F83C004FEA154C2F0E060A050C000E76
:101FB00081F83AC081F83B7081F83D6081F83E506D
:101FC00081F83F00D4E9045011692E0A4FEA154CFC
:101FD00081F8296081F8285081F82C002F0E060A1C
:101FE000050C000E81F82AC081F82B7081F82D6055
:101FF00081F82E5081F82F0011694A20A1250B731A
:102000004B73C8738D7311694B75126912A81374E1
:1020100053749374D374FEF71BFC034600287FF4BB
:102020006CAF009860E76878626C012304F150019E
:10203000FDF75EF938B994F83030009D03F07F0366
:1020400084F830301DE7012357E72046FEF780F97A
:10205000034600283FF458AF4FE700BF00000000E0
:1020600010B582B00446FFF7FBFE08B102B010BD08
:1020700001A92046FDF79CF90028F7D1206002B0A5
:1020800010BD00BF000000000000000000000000C4
:102090002DE9F04F85B003A9904699460446FDF717
:1020A00087F90546002840F0018194F83150002D51
:1020B00040F0FC8003990B78042B00F0078100238B
:1020C0004B454FF0FF3208BF42453CBF9046994612
:1020D000D4E904234B4508BF424505D294F83000AB
:1020E00080075CBF9046994600230022D4E90E6722
:1020F000C4E90E2358EA090300F0D8804B894FEA5F
:10210000432B56EA070300F0D58016F1FF3647F15E
:10211000FF3718F1FF3049F1FF315A460023F6F737
:10212000BBFF5A46CDE90001002330463946F6F799
:10213000B3FFDDE900238B4208BF8242C0F0BA80C2
:102140000BF1FF3326EA030632463B46C4E90E2371
:10215000B8EB060269EB0703D4F840A09046994615
:10216000BAF1000F71D000224A4508BFC34549D2D9
:102170005346CDE90089DA46934625E0D4E90423A5
:10218000BB4208BFB24205D2C4E904674CF0400C20
:1021900084F830C0FEF704F90346002800F0CF8031
:1021A0005A1C00F0B880012B40F2BC80039AD2691F
:1021B0009A4240F2B780DDE90012934508BF8A4594
:1021C0002364D4E90E671AD216EB0A0847EB0B0911
:1021D00046464F46DDE9008994F830C0B8EB0A085E
:1021E00069EB0B091CF0020F19462046C4E90E6783
:1021F000CDE90089C2D1FDF763FB0346D0E79A46DB
:1022000088469146002340F2FF1216EB080602EAC8
:10221000080003EA090147EB090750EA0103C4E992
:102220000E6700F09280039AD369AAF1020A023B7A
:102230009A4577D25389126B0AFB0323002B71D086
:102240004FEA582A4AEAC95A9A44D4E90401B946DD
:10225000B046494540F2FF124FF0000308BF404529
:1022600006EA020607EA030742464B4607D294F8FD
:102270003010C4E9042341F0400184F8301056EADC
:10228000070313D0626C524510D094F93030039993
:10229000002B487804F1500638DB314601235246C2
:1022A000FCF7FEFF002836D1C4F844A0284605B04C
:1022B000BDE8F08FD4F808A0BAF1000F16D00022C4
:1022C000002316461F46C4F840A049E74FF0FF33ED
:1022D000226C04F11C012046FEF712F8002837D1C9
:1022E00003990B78042B3FF4F3AEE8E65146204601
:1022F000FEF756F80128824614D0B0F1FF3F0AD00D
:10230000D4E90E23A06016461F46DCE701233146C0
:10231000FCF7EEFF50B10125284684F8315005B096
:10232000BDE8F08F022584F83150BFE794F83030D3
:10233000039A03F07F0384F830305078ADE7D4E996
:102340000E23824616461F467FE74FF0000A7CE7C1
:102350000546ABE7000000000000000000000000A0
:102360002DE9F04BBCB0019100283CD0044600227E
:1023700002A901A8FDF714FC20B1002323603CB0A2
:10238000BDE8F08B029B236003A914AAC3E90312E2
:1023900020460199FEF7CCFC48BB94F94B30002B4A
:1023A00029DBA379DB0624D5029B1978042924D0E4
:1023B000E06BC57E827E032942EA052205D1457D78
:1023C000017D41EA052142EA0142A260DB88A38047
:1023D00000212046FDF72CFB04280AD00028CCD190
:1023E0003CB0BDE8F08B09203CB0BDE8F08B042880
:1023F000C3D10520C1E7029BE8E72169E579E06CDC
:102400001A69A668266221F0FF012943C4E9091070
:10241000D58E92F8350092F8341040EA052041EA52
:102420000021A160D56B92F83B60290E002747EA96
:10243000010C280246EA000B4FEA0C2192F83A60A0
:1024400041EA1B61002747EA010C4FEA0B2046EAEC
:10245000000B4FEA0C2192F8396041EA1B6100271A
:102460004FEA0B2047EA010946EA00084FEA092C27
:1024700092F838604CEA186C4FEA082B00274BEAB8
:1024800006004CEA0701C4E9040192F8212002F099
:102490000202E2719AE700BF0000000000000000A5
:1024A00070B5BAB00D4669460446FCF781FFB0B975
:1024B000BDB1009B01A912AAC3E903122046FEF791
:1024C0005FFA10F0FB060AD129462046FCF798FF78
:1024D00031462046FEF784F8042808BF00203AB0B1
:1024E00070BD01462046FDF7A3FA3AB070BD00BFAB
:1024F0002DE9F04BF2B003A90190022201A8FDF7EB
:102500004FFB10B172B0BDE8F08B039B0199229391
:1025100011A84AAAC3E9030222A8FEF709FC002871
:10252000F0D19DF9D330002B05DB9DF88E30DA0712
:1025300003D50720E6E70620E4E7039A0492117822
:10254000042903F0100321D03198C57E847E03292D
:1025500044EA052468D073B13692389436A8002135
:10256000FDF766FA0028CDD136A8FEF709FA002853
:10257000DFD00428C6D122A8FEF7C2F90028C1D1B5
:10258000002C58D10398FDF7DBF8BBE71169CC6B41
:10259000C88E270E2602002591F83B4045EA070920
:1025A00044EA06084FEA092747EA186791F83A40D3
:1025B000002545EA07094FEA082644EA06084FEADB
:1025C000092747EA186791F83940002545EA0709C5
:1025D0004FEA082644EA06084FEA092C91F83540EC
:1025E00091F834504CEA186C4FEA082B91F8388077
:1025F00091F821104FF0000944EA00204BEA080648
:102600004CEA090745EA002401F00201CDE9086718
:1026100006948DF81710002BADD036923894CDE982
:102620003A678DF8DF1099E7457D017D41EA052184
:1026300044EA01448FE70246214604A8FDF7D0FD95
:1026400000289FD05EE700BF0000000000000000EF
:102650007F2805D940F25233994202D000207047BA
:10266000704710B40A490023C72203E0802B0CD026
:1026700031F8022F90429CB203F10103F6D104F12C
:10268000800080B25DF8044B70470020FAE700BF7D
:10269000441F0408000000000000000000000000CB
:1026A0007F2804D940F25233994201D0002070476C
:1026B000FF28FBD800F10040024B803833F81000AF
:1026C000704700BF441F0408000000000000000025
:1026D00070B4264A264BB0F5805F41F67D513CBF71
:1026E0001346612104330DE081420ED833F8022CE9
:1026F000D4B26518A8424FEA122208DB04337AB13B
:1027000033F8041C1E460029EED170BC7047082A1D
:10271000FBD8DFE802F00E12181B1E2124270A0046
:1027200006EB440336F81410DCE7A0F5E35080B262
:10273000EBE7411A33F81100E7E7411A01F0010312
:10274000C01A80B2E1E7103880B2DEE7203880B2EC
:10275000DBE7303880B2D8E71A3880B2D5E70830E6
:1027600080B2D2E7503880B2CFE700BF941C040893
:10277000881E0408000000000000000000000000A7
:10278000014B1860704700BF0416002000000000D5
:10279000034A044B0449116001221A70704700BFBC
:1027A0000416002000160020FFC99A3B000000001C
:1027B000174B1B6810B50446C3F86C02A8B99FED0F
:1027C000150A15480DF03CFE144A43F250531268A6
:1027D000D35C13B1124807F06BFA124B1249186818
:1027E0002246BDE8104024F013B9D3F8E8010CF0FC
:1027F000B7F807EE904AF8EEE77A9FED0C7A0648B4
:1028000027EE800A80EE070A0DF01AFEDCE700BF13
:102810006C1800200000C07FE83D002060180020F8
:10282000C03E0020E43D0020442004080000704227
:102830002DE9F0411B4D1C4A2B68116841F2F474DC
:1028400086B01C598C422ADD184914600646184689
:102850000F680CF0FDF9804623F06AFA224614490D
:1028600000904346384624F0D3F82C6804F5BF5452
:102870001034D4F8803F1A6803925A6804929B6817
:102880000593204604F0A4F903ABD4F8842F0093F9
:102890000146032330460DF0BBFE064B336406B001
:1028A000BDE8F08160180020D4390020E43D00200C
:1028B000B0200408000080BF0000000000000000FD
:1028C0000844013890FBF1F301FB1300704700BF8F
:1028D000F8B50646084414461D46421E204692FBA3
:1028E000F1F301FB1322294625F072FB324607461D
:1028F0002946204625F06CFB381A18BF0120F8BD88
:1029000070B5154601F118040E462246896D284619
:102910000023FFF7DDFF38BB01232246B16D2846B7
:10292000FFF7D6FFA0B9B16D022322462846FFF774
:10293000CFFF00B970BD2A462046022125F048FB92
:10294000002814BF05200420BDE8704001F060BAE3
:102950002A460121204625F03BFB002814BF032016
:10296000022001F055FADEE72A460021204625F034
:102970002FFB003018BF012001F04AFACCE700BF5E
:1029800038B50E4B1B688B420D4B0CD01B784BB1EE
:1029900005460C460DF05CFF0A4B1B6893F84C3063
:1029A000DB0703D438BD00221A7038BD2246294601
:1029B0000548BDE83840FFF7A3BF00BF041600205C
:1029C000001600206C180020E03D002000000000F0
:1029D00030B51D4D1D4B2C681B681D4A04F5BF54B6
:1029E0008BB01060D3F86C02FFF7E2FED4F8903F92
:1029F0002D681A6807925A68089210349B680993E8
:102A0000204604F0E5F81349134B049307AACDE9D7
:102A1000022103230193D4F8843F009305F5FE655A
:102A200003462A460D490E480DF032FE0D490E4868
:102A300024F0D6F80D490E4824F0D2F80D490E487E
:102A400024F0C6F80BB030BD601800206C180020D0
:102A5000E43D002031280108812901086C20040888
:102A6000E83D0020B12701087C20040881270108E7
:102A700080200408912701089C2004080000000021
:102A800038B50E4C0E49204625F002FA201D0D499E
:102A900025F0FEF904F108000B4925F0F9F9D4E915
:102AA00000250A4BA4681A60C3E901541A46084974
:102AB0000848BDE838400DF02BBC00BFD43D0020D5
:102AC000E0360020DC370020D8380020C83D002048
:102AD000D8390020E83D0020000000000000000080
:102AE00010B5084C0848D4F8F81924F089FF94F878
:102AF000D43903B910BD044A04490548BDE8104063
:102B000007F096B9B02E0010843E002070CB040868
:102B1000C03E002000000000000000000000000097
:102B200070B506684068F5F7C7FD044630460D46A7
:102B3000F5F7C2FD02460B4620462946F5F750FF41
:102B4000F6F7FCF800EE100A70BD00BF00000000B0
:102B500090F820301BB1012B03D0002070470120DA
:102B600070470068B0FA80F040097047000000002C
:102B700090F82030022B09D0012B01D000207047A3
:102B800000680028D4BF0020012070470120704752
:102B900090F82000A0F10100B0FA80F040097047E1
:102BA000C069704700000000000000000000000045
:102BB00000687047000000000000000000000000F6
:102BC000F0B40FA5D5E9004500220B4E0B49026079
:102BD000002786600026C0E904674260826180F8B1
:102BE0002020C26180F82120C0E904450A60F0BCC1
:102BF000704700BFAFF300800000C07F903E002010
:102C0000003CDD9BFFFFFFFF000000000000000014
:102C100090F82000A0F10300B0FA80F0400970475E
:102C20002DE9F84F06461A4892469B460BF0F0FFF6
:102C300000BBD6E90445174911A7D7E90067BAEBED
:102C4000040209686BEB0503964201F54E5177EBE0
:102C50000303D1E900890BDB0BA3D3E90023BAEB13
:102C600008046BEB0905A242AB41ACBF0120002078
:102C7000BDE8F88F0020BDE8F88F00BFAFF30080FB
:102C8000FF61113200000000FF79030A000000001C
:102C9000B02E0010601800200000000000000000AE
:102CA0000368016002684360002A0EDDD0ED007AFF
:102CB000DFED076AF8EEE77A86EEA77A80ED027A12
:102CC00003B1704703480CF0C3BA034B83607047ED
:102CD000ABC22248B02E00100000C07F00000000F0
:102CE00010B50446FFF7DCFF236894F8202033B1C9
:102CF0000C4B2168B3F9643099420CDB03239A42F0
:102D000084F8203009D0084B1868BDE8104000F660
:102D1000180028F015B8012A00D910BD022384F844
:102D20002030F0E7386B0010601800200000000031
:102D30002DE9F04F644E87B083460F4622F0D0FF56
:102D400034688046894604F6F81A002F42D05F4D59
:102D5000D5F8D839012B06D094F8183A012B1BD09E
:102D600007B0BDE8F08F336803F60823D3E90023EA
:102D7000D5F8F859002D5ED19FED550A4FF47A73BE
:102D800003FB0B7300EE903AF8EEE00A06F0C0FE8B
:102D900094F8183A012BE3D1306800F6586004F03B
:102DA0000FFC306842464B4605A900F6586004F017
:102DB00027FC484BFDEEC07AB3F9641017EE900A79
:102DC000013924F055FD01465046FFF769FF07B071
:102DD000BDE8F08F404B3D4D5A6843F6784350466E
:102DE000EA5042460B46FFF71BFF70B1DAE90423B5
:102DF000B8EB020269EB0303CDE9002313432DD1A5
:102E00004FF0FF315046FFF76BFFD4F8103A3249CC
:102E10000133C4F8103AD4F8143A0133C4F8143A20
:102E2000CAE9048943F678424B68A95843F67C42C4
:102E30005B1AAB508CE7B8EB020069EB0301F6F7C5
:102E40009DF807EE905ADFED256AF8EEE77A86EEF8
:102E5000A77A07EE900A87EE870A8FE7204909686C
:102E6000D1F8E80106F02CFCFDEEC07A1D48DFF831
:102E700078E017EE901A80FB01C00844C917C1EB37
:102E8000202C6046C117DDE90023CDE9000101993E
:102E90004FEA4C000EFB01010391ACFB0E01CDE9A2
:102EA00000010198039908440190DDE90001F6F75B
:102EB000A3F847F230518842D4BF01464FF0FF31AA
:102EC0005046FFF70DFFA0E760180020B02E00105D
:102ED0000000C07F386B0010001000E0809FD54BD1
:102EE0006C180020B7600BB60098D05800000000A6
:102EF0008069704700000000000000000000000032
:102F0000002110B5C1610368044633B1FFF7C8FE64
:102F1000044B0549186823F07BFD002384F820301A
:102F200010BD00BF803E002000210408000000000A
:102F3000002280F82120FFF7E3BF00BF000000005F
:102F4000184991F8F212C90616D590F8201070B5FC
:102F500041B990F8211081B127F022FFBDE87040FF
:102F600027F00EBF0129F7D10F4C0168246879B909
:102F700090F8211019B10BE070470B490C6841F231
:102F8000E4250121002680F82010665180F82110E8
:102F900004F6586004F054FC27F002FFBDE87040CE
:102FA00027F0EEBE386B0010601800200000000013
:102FB000024B1B68D3F8100A704700BF601800204E
:102FC0002DE91848104B114C1B6803F60823D3E970
:102FD0000023D4F8F84994B1801A61EB0301F5F7A6
:102FE000CDFF07EE904ADFED0A6AF8EEE77A86EE4B
:102FF000A77A07EE900A87EE870ABDE818889FED4A
:10300000050ABDE8188800BF60180020B02E001027
:10301000809FD54B0000C07F000000000000000032
:10302000094B0A4A1B78106003B1704710B5084C71
:1030300008492268084800F0B3FB2268074908489D
:10304000BDE8104000F0ACBB40490120803E0020AC
:1030500060180020E0200408C1300108F0200408B6
:10306000312D0108000000000000000000000000F9
:1030700010B5054C20460DF00BFC04F11800BDE81E
:1030800010400DF005BC00BF503E002000000000C5
:1030900010B4019C0848D4ED027A0068019327EE31
:1030A000800A1346FDEEC07A00F5FE6017EE902A06
:1030B0005DF8044B0EF044BA6018002000000000D8
:1030C00091B91A4B93F8D42972B1194A106830B5E6
:1030D000D0F8102AD3F8F83947F22E54013BA34216
:1030E00083B002D903B030BD7047124C124BD4EDFF
:1030F000007A93ED747A114C114B00F6F81577EEC7
:10310000877A95ED027A009167EE877A02F00102E4
:10311000FDEEE77A5100114400F5FE6017EE902AAB
:1031200004EBC1010EF00CFA03B030BDB02E00105C
:103130006018002008560010386B0010503E002028
:10314000E12A01080000000000000000000000006B
:103150002DE9F04FC04DC14E2B68C14C1868336843
:10316000D4F800B0DFF86CA38FB009931EF018F804
:103170002B680D90D3F80C021B680C9308F038FAFA
:1031800029680A9042F25D70D1F80C321AF80000FA
:103190000B9324F05DFB2968074691F8C505C0F341
:1031A000801024F055FB2968804691F81002C0F386
:1031B000800024F04DFBAB4981460868F5F78EFA94
:1031C0000A9A0B9B0092CDE9060101930D9A0C9B84
:1031D00002975846CDE90389A34923F019FC2A68D0
:1031E000D2F80C32002B00F0D181099F32689F4940
:1031F000206843F2044C07F5BF5743F208431037E9
:10320000D35852F80C2023F003FC7B78002B40F0BD
:10321000B08142F2687142F2647342F260725AF80D
:1032200001105AF802205AF80330206800919049A2
:10323000DFF8A4B223F0ECFB2B68D4F80080D3F8BD
:103240000C9241F2F1731AF8030024F001FB4A4694
:1032500003468849404623F0DBFB5BF8040BF5F797
:103260003DFA8046DBF80000D4F800B08946F5F757
:1032700035FA4246CDE900014B4658467E4923F0D7
:10328000C7FB099B21680B9141F2F072985C24F016
:10329000DFFA804604F04CF924F0DAFA3368D3F808
:1032A000C42E09928146D3F8C82E0A9203F65860BC
:1032B00004F07EF92B68834693F84C0000F001007F
:1032C00024F0C6FA0A9A0B990192099A0390009287
:1032D0004B4642460846CDF808B0684923F098FBB3
:1032E00041F2F0721AF80230002B40F029812B686D
:1032F000D4F8008093F8C408002840F00881604D9D
:1033000095F8C40212F01CFD5E490246404623F0C7
:103310007FFB95F8E802D4F8008012F011FD814699
:1033200095F8EB0208F0F4FAD5F8743200934A46A7
:1033300003465549404623F06BFB7B78E3B195F893
:10334000C502276812F0FCFC50490246384623F0BB
:103350005FFB95F8E902276812F0F2FC804695F8C9
:10336000EC0208F0D5FA4A4B4A491B6D00934246DD
:103370000346384623F04CFB95F844032768DFF8F2
:103380005C8112F0DDFC814695F8450308F0C0FA37
:103390004A4603464049384623F03AFB95F8F40282
:1033A000D4F800903D4F12F0CBFC3D490246484610
:1033B00023F02EFB95F8F502D4F8009012F0C0FC33
:1033C00038490246484623F023FB3068D8F80030DD
:1033D000354943F6544243F63C458258206823F071
:1033E00017FB324B31681B6843F6644043F65C427E
:1033F0001B688A580958009120682D4923F008FB62
:1034000032682C4943F6444043F64C43D358125893
:10341000206823F0FDFA316820684D59264E43F6A6
:10342000744343F66C42CB588A58019543F67C4569
:10343000495900912149224D23F0EAFA3A6820685F
:10344000204923F0E5FA204B20681A681F4923F031
:10345000DFFA1F4B206843E06C1800206018002042
:10346000A83E0020085600101021040888210408F6
:10347000D8210408F82104081C2204083C2204086E
:10348000386B0010E4220408002304082C230408ED
:10349000E83D0020482304087423040848720020F3
:1034A00094230408AC230408C82304080816002049
:1034B000F823040824240408B43E00204C24040803
:1034C0000887002088240408C8AB0020A42404082E
:1034D000B8760020B02E0010A84600104C720020D4
:1034E0001A682F4923F094FA326820682D4923F096
:1034F0008FFA20682A682C4923F08AFA0023C8F83A
:10350000003033603B602B600FB0BDE8F08F12F0ED
:1035100017FC2B688146D3F8300908F091F94A4628
:1035200003462249404623F073FA214B214A1B6887
:1035300012682149206823F06BFAD4F80080DEE697
:103540001E4B03F63C731868F5F7C8F81B4BD4F80C
:1035500000A003F64C73804618688946F5F7BEF85C
:103560004246CDE900014B465046154923F050FA3A
:10357000BDE632681349206843F20C4C43F2104315
:10358000D35852F80C2023F043FA42E6D2F818320E
:103590000D49D2F81422206823F03AFA25E600BF3C
:1035A000C0240408D8240408F8240408B02204081D
:1035B00074A5002078A50020C8220408A8460010A1
:1035C00098220408B02104087421040800000000B7
:1035D000074B196842F2AC5001F658610A180023F3
:1035E0000B5053609360D36013615361FFF7B0BD1C
:1035F0006018002000000000000000000000000033
:103600002DE9F043224B234A1D68DFF89C80DFF848
:103610009C90D8F8004042F25D7383B0D05C24F0F7
:1036200017F91D490246204623F0F2F91B4B186892
:10363000F5F754F81A4B064618680F46F5F74EF89A
:103640003B46CDE9000105F5BF573246D8F80000EA
:10365000144905F5C05523F0DBF910370435002473
:103660000DE055F8040BD8F80060F5F737F822465E
:10367000CDE9000130464946013423F0C9F9384606
:1036800003F0A6FAA042ECDC03B0BDE8F08300BF73
:1036900060180020B02E001080250408E4550010AA
:1036A000F455001098220408A83E00208C25040838
:1036B00038B5044600F517503022FF21083029F0B4
:1036C000EFF8302504F517502A460021383029F04C
:1036D000E7F804F518502A4628300021BDE83840A4
:1036E00029F0DEB80000000000000000000000002B
:1036F000F8B50446002603F0F3FE002704F688120E
:1037000004F51863C3E90067002104F5196311602B
:1037100004F51455C3E9006704F6981003F030FA75
:103720003C220021C5E90667C5E9086705F170007C
:1037300029F0B6F83C22002105F1340029F0B0F858
:1037400004F5165304F517522C330432002143F8C4
:10375000041B9A42FBD10AA7D7E9006742F2305214
:1037600004F51453C3E90A672046A15003F080FE14
:103770002046FFF79DFF2046F8BD00BFAFF3008055
:10378000003CDD9BFF79030A000000000000000000
:1037900001F66A1100EB81014868704700000000E3
:1037A00038B50546084814461AF0BAF943F288328B
:1037B00043F28C31A358581CA05004EB830343F20E
:1037C000C8325D509C5038BDBC2504080000000084
:1037D0002DE9F04F9B4B2DED028B93F8D43985B03A
:1037E000044643B1984A994B99499A48012C08BF1D
:1037F0001A4606F01DFB984D95F8F232003418BFBA
:103800000124C3F34003A34204D005B0BDEC028BF6
:10381000BDE8F08F914A924B166806F52062146855
:103820009C42F2D0DFF85C8222F05AFAD8F800907D
:10383000D9F83039032BCDE9000106F6586770D06E
:1038400007F51963D3E90001DDE90023121A63EBE0
:10385000010310461946A8220023F5F7CDFBF5F722
:103860008DFB07EE104A07EE900AC7EE877A7D4A75
:103870007B4B92ED007AD5ED746A37EE267A77EEBF
:10388000C77A17EE902A9A4200F0B980764BF5EE8F
:10389000C07AF1EE10FA93ED007A06D577EE877ACA
:1038A000F5EEC07AF1EE10FAF8D4B4EEE77AF1EE64
:1038B00010FA06D877EEC77AF4EEC77AF1EE10FA6E
:1038C000F8DAD8F8003093F8B825D20703F61802D2
:1038D00092ED007A48BFF1EE677A77EE277A06F527
:1038E000BF56C6ED007AD3F83039002B62D0012BD9
:1038F00000F09180032B88D101E003F0C9FF384626
:1039000003F056FED8F80020434203F00303D2F838
:10391000882900F0030058BF584290423846ECD145
:1039200073E742F2185A42F2205257F80A300392D3
:1039300007EB020B009AD31A08EE103ADBE90001FC
:10394000F5F71CFB18EE101A039A0023B950CBF8B8
:103950000430DDE90023BA44CAE9002399F8C535EB
:1039600007EE900AB8EE488A1807C8EE278A38D4BE
:10397000D5EDCF7AF4EEE87AF1EE10FA3FF745AFE5
:10398000D5EDD07AF4EEE87AF1EE10FA3FF53DAFDE
:10399000D8F8003093F8C525110743D4D3F8403840
:1039A000082B7FF44DAF314AD2F8C0300133C2F852
:1039B000C03045E7384603F073FF00287FF425AF99
:1039C000384603F065FFD8F80030D3F84038082BAC
:1039D0007FF41BAF254AD2F8C0300133C2F8C030A3
:1039E00013E718EE900AF4F779FEDFF89CC0024660
:1039F0000B46DCF800001E4923F00AF8B8E71D4A20
:103A00001D4941F688101FF053F8174BDFED1B7A64
:103A100093ED007A49E7384603F042FF00283FF46F
:103A2000F4AECDE718EE900AF4F758FEDFF858C070
:103A30000B4602461249DCF8000022F0E9FFD8F8F4
:103A40000030ABE7B02E00104CA704084C2504084A
:103A5000FC370408C03E0020386B001060180020BE
:103A60000000C07F08560010E038001094160120B6
:103A70005C2504086C250408782504080000000073
:103A8000502504086C180020A83E0020000000000B
:103A90002DE9F84F5F499DF828C011F80C10002956
:103AA00040F0928000EBCC0505F517510831D1E9C3
:103AB00000AB05F51754DFF860E1BBF1FF3F04F1FF
:103AC000380408BFBAF1FF3FD4E900671EF80CC004
:103AD00009D0B2EB0A0863EB0B0916EB080647EBBB
:103AE0000907C4E90067C1E90023DFF830E141F2CA
:103AF000F0730CF2C54C1EF803A000EBCC0CDCE913
:103B00000089BAF1000F31D14046494600234000F8
:103B100041EB01010322F5F76FFA864277EB0103CF
:103B200021DB4B4642469B00900043EA987118EB1C
:103B3000000849EB0109B8F1000F79F100033EDB01
:103B40004FEA980141EA89724FEAA90352EA030158
:103B50003FD105F51855C5E90A6700220023C4E9DD
:103B600000234FF0010A5046BDE8F88F90F808A0F6
:103B7000BAF1000FC8D042F26072C36B5EF8022047
:103B80000133934229D0404649460023400041EB8F
:103B900001010322F5F730FA864277EB010335DBAA
:103BA000494640468900820041EA987318EB0208B2
:103BB00049EB0309B8F1000F79F10003C0DA18F1FD
:103BC000030849F10009BBE74FF0010A5046BDE880
:103BD000F88FB242BB41C0DBBBE742F25473032211
:103BE0005EF803004B464FEAE07B00FB03F308FB63
:103BF0000B33A0FB08011944400041EB01010023F5
:103C0000F5F7FAF9864277EB0103A6DA4FF0000ADE
:103C1000A9E700BF042604080C260408B02E0010F3
:103C200090F89A39002B72D12DE9F04F83B00446F9
:103C30000D4622F055F804F518660B460246C6E913
:103C40000023694991F8F212C90950D1674F6849B8
:103C500008680AF0CDFF04EB850142F2AC5204F58E
:103C600014588B5801338B5008F12808D6E90023EB
:103C7000D8E900010FF2681BDBE900AB101A63EB17
:103C8000010182457BEB0101C0F29080C8E900236D
:103C90002946204603F0BCFE3B68D3F8E8319A1E63
:103CA000012A40F28980012B204614BF4FF00408FE
:103CB0004FF0020803F07CFC90FBF8F303FB1808BC
:103CC000204603F0DDFDDFF8449142F66C4359F8DD
:103CD000033003FB0808B8F1000F1DD099F8D43960
:103CE00023BB237A002B4AD103B0BDE8F08F0095A7
:103CF0002046FFF7CDFE0028F6D03C4F2846396815
:103D000004F036FA0028EFD0D6E900239FE73949BE
:103D10004FF4C0501EF024BFD6E9000104F519632A
:103D2000C3E9000199F8D439002BDAD03248414672
:103D3000861E23F065FE314A99F8D43912F805A0A1
:103D4000BAF1000F0CBF642275223270002B3DD1F6
:103D50003B6893F8C5355B06C3D5BAF1000F99F8F7
:103D6000D4390CBF752264223270002BB9D0244B99
:103D7000244A53F82510244806F05AF8B1E72046A3
:103D800003F06EFD0028AFD042F23053E718E3583D
:103D9000002BA9DD3E46002456F8043F4146284644
:103DA00098473B680134A342F6DC9DE7204603F0C8
:103DB0007FFDD6E9002369E7204603F061FD8046D8
:103DC000DFF84890B8F1000F88D1A5E70C4B0E48FA
:103DD00053F82510324606F02BF8B9E7AFF3008010
:103DE000007A030A00000000386B00106C180020F5
:103DF00060180020D82504089A3E0020B425040845
:103E00009C250408983E0020C03E0020B02E0010E3
:103E100070B5164B93F8F232DB0905461FD0144CEF
:103E2000144922680B6814489A42466800DD0A600B
:103E3000124B18680132294600F658602260FFF7DD
:103E4000EFFE22680C4B0E495B680E48013A226077
:103E50000A689B1B9342036088BF0B6070BD0A4BCE
:103E6000196804F085F90028D9D170BD386B0010AD
:103E7000B83E0020AC3E0020001000E0601800209A
:103E8000B43E0020B03E00206C180020000000006E
:103E9000704700BF000000000000000000000000AC
:103EA00010B40648064C0749074A00232360036004
:103EB0000B6013605DF8044B704700BF4872002030
:103EC000B43E00204C720020088700200000000053
:103ED000444BD0F80C221B68D3F80C12914205D148
:103EE000D3F8E811D0F8E821914210D03E4B3F487A
:103EF000196810B53E4C0AF0ABFD206800F658601A
:103F0000FFF7D6FB2368012283F8E82710BD93F85A
:103F1000C52590F8C5154A405206E7D493ED727A4C
:103F2000D0ED727AB4EE677AF1EE10FADED1D3F802
:103F30001412D0F814229142D8D1D3F81812D0F824
:103F400018229142D2D1D3F8BC22D0F8BC124A40F8
:103F500032F07F42CAD193F8C41890F8C428914235
:103F6000C4D1D3F83019D0F830299142BED190F89D
:103F7000EA1293F8EA224A409107B7D403F61801EF
:103F800000F6180291ED007AD2ED007AB4EE677A6D
:103F9000F1EE10FAAAD193F8B82590F8B8154A4076
:103FA000D207A3D493EDCD7AD0EDCD7AB4EE677A73
:103FB000F1EE10FA9AD193EDCE7AD0EDCE7AB4EE3E
:103FC000677AF1EE10FA91D1D3F88829D0F88839C0
:103FD0009A428BD1064B1B6893F8E82783F8E827B1
:103FE000704700BF6C180020A83E0020B02E0010C3
:103FF0006018002000000000000000000000000029
:1040000010B5094C20680AF023FE0146074823F04A
:104010002FFF236810B193F8E80700B900200022B1
:1040200083F8E82710BD00BF60180020943E0020F0
:1040300008B50C4B0C491A680C4B0860110C9970B0
:104040001A800B4805F06CFF0A490B4822F0C0FDAE
:104050000A490B4822F0BCFD0A490B48BDE808405C
:1040600022F0B6BD18250408A83E0020983E002086
:10407000C03E0020513101081C250408013601080A
:1040800028250408D13501083C250408000000005B
:1040900008B5044805F06CFE0348BDE8084023F06D
:1040A000DFBE00BFC03E0020943E002000000000A4
:1040B0002DE9F047C36D3A493A4AD1ED007ADFF86D
:1040C000F490394E03F65451054603F556602DED34
:1040D000028B02EB810102EB800291ED018AD2F8A2
:1040E00004A003F2822309EB830338EE678AD3ED41
:1040F000017A5046F0EE408A38EE278A26F028FCF6
:10410000471E4FEA470826F04BFE08EB0704E40081
:1041100004F54874022834441ED04FF000092046AC
:104120000CF09EFE48B9474406EBC7061F49D6F877
:104130002C2341F283701EF013FD85ED0E8A38EEBC
:10414000680ABDEC028BC5E9004905F13C0118483D
:10415000BDE8F04702F04CBF99F8CD35DB0901D13D
:104160009946DCE7D9F8980100EBD0700AEB6000C3
:1041700026F0EEFB013800EB40004FEAC00A0AF5DA
:104180004879B14448460CF06BFE0028C7D1B244D0
:104190000649DAF82C2341F283701EF0E1FCBEE7F9
:1041A00074650010B02E00105872002028270408F3
:1041B000A0460010386B0010000000000000000056
:1041C0002DE9F047DFF86C80DFF86C90DFF86CA029
:1041D0000646051F071D55F8044F6CB194F90530CC
:1041E000B26D2261C3B120460CF082FE98F8CE3841
:1041F00013B148460CF07CFEBD42ECD10B4B0C4A8F
:104200001B68934206D0304600EE103ABDE8F047F6
:10421000FFF74EBFBDE8F087E268514642F2343006
:104220001EF09EFC01232375DDE700BF78650010BA
:104230000000C07F386B0010F8720020C42604080C
:104240002DE9F04FDFF89090DFF89080DFF890A034
:1042500083B00646051F071D55F8044F2CB3D8F848
:104260000020D9F8F839B2F95C20B3EB420F0BDD2E
:10427000E368DFF870B001931A46DBF800309A4229
:1042800018D0019BCBF80030237D2BB1B36D226990
:1042900000219A42217508D020460CF011FE9AF8B0
:1042A000CE3813B10A480CF00BFEBD42D4D103B096
:1042B000BDE8F08F26F074FD0028E2D0FEF778FE0E
:1042C000019B0449024641F29D701EF049FCD8E76B
:1042D000F8720020E0260408B02E00106C180020B0
:1042E000386B0010203F002000000000000000009C
:1042F00070B50646044600F59C65204668340BF010
:1043000027FCA542F9D1002386F8E034304670BD81
:10431000024B93F8CC0500F001007047386B001099
:1043200070B4144DD5F80432052B1ADDD5F80012FF
:1043300006260024D5F808220139204600290B461C
:1043400001DA9B18FDD455F823300130B0421C44EB
:1043500001F1FF31F2DB042CD4BF0020012070BC3E
:104360007047D5F80462D5F80012002EE1DC002079
:1043700070BC7047283F00200000000000000000D3
:10438000014B1860704700BF34410020000000005E
:10439000012811D008B50AD3022800D108BD024671
:1043A000064941F2DC701EF083FB012008BD044B7E
:1043B0001B68D3F8900108BD704700BF08270408A8
:1043C0006C18002000000000000000000000000049
:1043D00010B52DED028B044626F0E2FCFFF7D8FF66
:1043E00007EE900A2046B8EEE78A26F089F9084BD6
:1043F000DFED087A1B68D3F8E831032B28EE278A13
:1044000018BF30EE000A88EE000ABDEC028B10BD2A
:104410006C1800200000C8420000000000000000EE
:10442000094B10B500244FF4007218462146C3F81A
:10443000004228F035FA8022C0F80442C0F8082271
:10444000C0F8004210BD00BF283F0020000000005F
:104450002DE9F04F2DED028B551E47F22E539D4254
:1044600087B000F2D680CE4F97F8CC359B0740F14D
:10447000D080DFF85C8398F8E0370C46CDE9032064
:10448000002B00F0CB80D8F8D01991B3DFF84CA303
:10449000DFF83893C34E01E029462DB38B6C4D6D88
:1044A000A342F9D1D8F8D0298A4204D129E18B421C
:1044B00000F03E811A46536D002BF8D1D1ED147AED
:1044C0009AED007AD9F80000009167EE277A203142
:1044D000FDEEE77A00F5FE6017EE902A33460DF008
:1044E0002FF82946002DD9D198F8E037002B00F09D
:1044F0009080D7F89831002B40F38B80DFF8D08282
:10450000DFF8BCB2CDF8148045460026A046D5F8A9
:104510003C33434575D1A44B1868584500F0F480EE
:1045200007EE900AF5EEC07AF1EE10FA40F2EC8058
:10453000D5F83893D94500F02D81DFF8A0A2D5ED4C
:10454000D17A9AED007A994B67EE277AD3F8002258
:10455000D3F80812F5EEC07AF1EE10FA4CBF012044
:10456000002043F82200D3F800220132C3F80022D1
:10457000D3F800228A4204BF0022C3F80022D3F8F5
:104580000422F5EEC07A0132F1EE10FAC3F80422EB
:1045900000F12C81864A1368C5F858330133136043
:1045A000049B05F54074002B00F0E18000EE109AAA
:1045B00005F552717F4802F01BFDD5F84833984548
:1045C00000F0BC80059BD3F8D029002A00F0608160
:1045D000A24200F0058113464FF47A7906E0B9F162
:1045E000010900F04281A34200F0FA805B6D002BCC
:1045F000F5D1C5F8543300E01A46536D002BFBD1BA
:104600005465D7F898310136B34205F168053FF794
:104610007EAF07B0BDEC028BBDE8F08FDFF8ACA138
:10462000654ADAF80030654D51682A6803F5715320
:104630001960D2F8E80105F043F8B0EE408A26F0A0
:10464000AFFB002800F0F780B6EE000A28EE008AE3
:10465000BDEEC88AB8EEC88ADAF8009043F2C865A1
:1046600009EB0503D3ED007AF5EE407AF1EE10FA8E
:1046700000F0D680B4EEE78AF1EE10FA00F1C280C5
:1046800043F2C4614E4B58F80110994252D04D4943
:10469000D1ED007A17EE901A99424BD0D7F89831A5
:1046A000002B40F3F38017EE90BA059409F540769D
:1046B00000254C46C4F85C53304600EE10BAFFF7B4
:1046C000F7FCD7F898210135AA4204F1680406F1F5
:1046D0006806EFDC059CDAF80030012189F8E01764
:1046E0009946354BD8F8D0195B6809F571500068C8
:1046F0001B1A43F6444049F8003000297FF4C6AE47
:10470000F2E6C8F8D059D9E6F3F7E8FF039B009327
:1047100002460B4641F2D2702B491EF021FAD7F81F
:1047200098310136B34205F168053FF7F0AE70E706
:104730005565C3E6002389F8E037D2E79AED007AA1
:10474000D5EDD47A214B009467EE277A204A186879
:10475000144BFDEEE77A02F54871682417EE902AB3
:1047600000F5FE6004FB06110CF0EAFE49E7174B6A
:104770000094174A1868174BFDEEE77A02F542726B
:10478000682101FB062100F5FE6017EE902A0CF06F
:10479000D7FE0BE710494FF4D1501EF0E1F930E796
:1047A000386B0010C141010870650010283F0020DF
:1047B000243F0020A0460010001000E06C180020EC
:1047C0000000C07F786500104426040860180020AF
:1047D000B02E00104142010868260408B0380010CD
:1047E0002F4942F233301EF0BBF90AE717EE900A68
:1047F000F3F774FF2B4C02460B4620682A4922F03F
:1048000007F9FEE617EE900AF3F768FF02460B463B
:1048100041F2917025491EF0A3F9DAF800902FE7D4
:10482000234941F290701EF09BF9DAF800904D4454
:10483000D5ED007A1EE72B68D3F8E80104F040FFBD
:104840002B68D3ED647AF8EEE77AC0EE277A17EE9C
:10485000900AF3F743FF10A3D3E90023F4F7C0F85D
:10486000F4F76CFA08EE100AF6E6124941F2E3702A
:104870001EF01EF9059BD3F8D029C5F85493002AE1
:104880007FF4BBAE059BC3F8D049BAE64B4624E79C
:10489000C5F85423F6E700BF9A9999999999F13F81
:1048A000A0260408344100207426040828260408A1
:1048B00018260408902604080000000000000000EC
:1048C000D0F8243AD3F89031002B10DD70B5084DA4
:1048D0000646002428460CF0F3FAD6F8243AD3F81A
:1048E00090310134A34205F12005F3DC70BD70471F
:1048F000F87300200000000000000000000000002D
:1049000010B50446406B28B1837E01335BB2012BA6
:1049100083760CDDA06B28B1837E01335BB2012B63
:10492000837600DD10BDBDE810400CF0C9BA0CF074
:10493000C7FAEFE7000000000000000000000000E0
:10494000D0F8243AD3F89031002B10DD70B5084D23
:104950000646002428460CF0CBFAD6F8243AD3F8C1
:1049600090310134A34205F12005F3DC70BD70479E
:10497000F8730020000000000000000000000000AC
:104980002DE9F0410F4F3E68D6F8243AD3F8903124
:10499000002B80460EDD0C4D002428460CF0A8FAB2
:1049A000D6F8243AD3F890310134A34205F120051A
:1049B000F3DC3E68D8F8101006F61800BDE8F041A8
:1049C00026F096B860180020F87300200000000060
:1049D00010B50446406B002384F8303010B1427E9D
:1049E000B2B14376A06B18B1437E43B10023437646
:1049F000E36B0C481969BDE8104026F079B8837E56
:104A0000013B5BB2002B8376F2DC0CF071FAEFE72E
:104A1000837E013B5BB2002B8376E3DC0CF068FA0B
:104A2000E0E700BFC83600100000000000000000F2
:104A3000F0B5044683B01648164DFEF7B9F80646A1
:104A400025F07EFE10EE100AF3F748FE2B68324682
:104A5000CDE900011846104921F0DAFF30462D68F3
:104A600007F0C6FC10EE100AF3F738FE064604F510
:104A70005B5004300F460068F3F730FE3246CDE954
:104A800000013B462846054921F0C2FF03B0F0BDB6
:104A9000A83800105C410020742804088C28040801
:104AA00008B5FFF7F5F9BDE8084005F031BA00BFD9
:104AB00010B5094C237803B110BD084B186800F6F7
:104AC000F810FEF745F80028F6D10146012014F051
:104AD00017FF0123237010BD9841002060180020AB
:104AE00008B504480BF024F803490448BDE8084021
:104AF00022F0AEBC384100202C750010604100202F
:104B0000F0B52DED028B012083B0384E14F0D8FEA5
:104B100033680A2894BF0446002403F6F810FEF711
:104B200017F880B1324D95F8CC355B0702D49CB1B3
:104B3000611C09E01AF074FCDFED2E7AB4EEE70A8E
:104B4000F1EE10FAF3DD0021012003B0BDEC028B81
:104B5000BDE8F04014F0D4BEB5F9D6352649274A51
:104B600091ED002AD2ED000ADFED251A9FED250A0E
:104B700001EE103A244BB8EEC11A01251C611D70DC
:104B800024F04EFAB5EEC00AF1EE10FAB0EE408A0B
:104B90002ADD3768D7F8243AD3F89031002B0CDDA2
:104BA0001A4D28460CF08CF9D7F8243AD3F89031F6
:104BB0000134A34205F12005F3DC9FED150AF7EE61
:104BC000000A28EE000A22F05BFE10EE100AF4F74D
:104BD0007BFA34680F49009402460F4B04F5FE60DF
:104BE0000CF0AEFC0121AFE72946ADE760180020CC
:104BF000386B00100000B4426C6600104473001063
:104C000000000000000020C238410020F87300209E
:104C100000007A44C82E001041490108000000003D
:104C200070B5194C194D2060FFF7AAFB206800F001
:104C3000EFFB1749174821F0CBFF2A6816491748A0
:104C400021F0BEFF266821F073F815490246304670
:104C500021F0DEFDFFF75CFB88B12A68114912489C
:104C6000FEF79EFD114BD3ED007AF5EEC07AF1EE22
:104C700010FA03DDBDE87040FFF742BF70BD206849
:104C80000B4921F0C5FDE8E75C41002060180020D9
:104C9000A14A010810280408314A01082028040804
:104CA0002C28040868280408C14C0108447300102B
:104CB0004028040800000000000000000000000080
:104CC0002DE9F04FBE4ABF4BBF4C15785A682DED09
:104CD000048B43F638438DB0E250002D40F03D8107
:104CE00043F2F073E3588B4240F23781D4F8F8A9CD
:104CF000BAF1000F00F03181BAF1FF3F00F0B68148
:104D0000DFF80C8308F50766D6ED007AD8F8A871AD
:104D1000F5EE407AF1EE10FA8B4640F04581BA4547
:104D200006DD5246A94941F292701DF019FF012596
:104D3000BBF1000F00F07481D8F8DC359B4500F022
:104D40001181FFF7E5FA002800F0F680002D40F011
:104D5000F38043F2EC73E35C002B40F0ED8094F8B9
:104D60009839002B00F0C6811AF05AFB984807F0DA
:104D700027FF984807F044FF504607F039FBD8F862
:104D8000982104F55253002A83ED0C0A40F3D48095
:104D9000DFF880929FED909ADFED909A03950027BF
:104DA00007E0D8F898310137BB4209F1200940F3F8
:104DB000C280D9F814309B45F3D1D9F80430884A21
:104DC00093F9181092ED000A8648874E07F048FDC7
:104DD0008648B0EE408AFDF7CBFE3368002800F02D
:104DE0005881D3F8A80106F0D3FE07EE900A50468A
:104DF000F8EEE78A25F05CFC68EE888AF4EEC08A5B
:104E0000F1EE10FA00F3DD81794D7A4B286893EDCD
:104E1000000A00F55650383038EE400A0AF0F0FA31
:104E2000754A764B82ED008A18EE102A9A4200F0FD
:104E30004F81B5EEC08AF1EE10FA00F14F81B4EE69
:104E4000C98AF1EE10FAACD46D4BD9ED077AD3EDE7
:104E5000008A99F80030BA010492A21828EE298A33
:104E600068EEA78A0592002B40F089813368B3F978
:104E70005C20BAEB420F0BDDD9F80420614ED268FA
:104E8000069211463268914200F0B581069B33606C
:104E900020F046FF049EA319CDE9060193F83020C7
:104EA000002A7FF47EAFD9F804C02A680492DCE9B6
:104EB0000412FDEEE87ACDE90812D9F808209A63C9
:104EC000DDE9060117EE902A801841EBE271DFF868
:104ED00048E1049AC3F834C0764402F5FE6E4FF000
:104EE000010283F83020CDE90A010246C3F83C9064
:104EF0000B46DDE9080182428B4180F26E814FF062
:104F000001038CF8193038EE288A3146FDEEC87A54
:104F1000DDE9065617EE902AAD18059BDFF8FCC0B8
:104F2000019346EBE27670462A463346CDF800C040
:104F30000CF096FB35E7039D524628465946FFF78D
:104F400087FABBF1000F08D143F638421D4BA15838
:104F50005B6843F63C425B1AA3500DB0BDEC048B7A
:104F6000BDE8F08F98F83F3C102B3FF4EAAE1E4EA0
:104F7000DFED257A3368254893ED897A93F8371C5D
:104F800087EE278A12F02CFA3268194B07EE900A46
:104F9000F8EEE77A92ED730A186867EE887A27EEE2
:104FA000800A09F0F5FFCCE61EF062F9D6ED007A32
:104FB000B4EEE70AF1EE10FA7FF7B1AEB1E600BF4A
:104FC00040490120001000E0B02E001048270408DE
:104FD000F43A0010E4380010CDCC4C3D00007A4487
:104FE000606300104C3800106C180020A8380010C6
:104FF0006018002098650010686300100000C07FF2
:10500000B03800105841002000F07F4568270408A0
:10501000386B0010C8360010C82E0010D1490108A6
:10502000FEF7EEFF60BB98F8C0359B077FF584AEB6
:10503000D4F8F829B8F9F0399A420DDBB8F9EC390F
:10504000764E07EE903A96ED007AF8EEE77AB4EEF7
:10505000E77AF1EE10FA51D5714B72481B6803F5EF
:105060005D5300229A6122F023F965E66E4940F211
:1050700055100DB0BDEC048BBDE8F04F1DF070BDB8
:10508000674B186880F8E0B780F898B90AF0E0F844
:10509000C9E7D3F8AC0106F07BFD07EE900A504655
:1050A000F8EEE78A25F004FB68EE888AF4EEC08A01
:1050B000F1EE10FA7FF7A8AE18EE100AF3F70EFB28
:1050C00002460B4642F2353058491DF049FD9BE639
:1050D000574941F28E701DF043FD62E618EE100A4A
:1050E000F3F7FCFA02460B4641F28F7051491DF06E
:1050F00037FD56E6504825F023FE35E61AF090F9C4
:10510000B8F9EE3907EE903AF8EEE77AB4EEE70A2E
:10511000F1EE10FAA0DCD6ED060AD8EDB07AF4EE86
:10512000E70AF1EE10FA97D4444F3B6803F5206389
:10513000D3ED007AF4EEE70AF1EE10FA8CDCDFF83A
:10514000E09016ED1E0A3748D9F80060B7EE001A55
:1051500022F016FA43F258723B68164486ED000AB4
:10516000D3F840380B2B7FF4E7ADD9F80030344941
:105170002C4813441B684B6422F072FADCE5286863
:105180000090FDEEE88A114600F5FE6018EE902AC8
:105190002C4B0CF0D5F9F8EEE88A2B4B2868CDF8AB
:1051A000009038EE888AA3F6E811FDEEC87A049BD9
:1051B00000F5FE60194417EE902A244B0CF0C0F95C
:1051C000EFE518EE100AF3F789FA02460B4641F2B2
:1051D000A6701F491DF0C4FC16E6059B1D490193EE
:1051E00070460091DDE90A2305990CF039FA286828
:1051F00000F5FE6E87E6D3F8AC31002B3FF446AEE7
:10520000032B3FF443AEFDF7D3FE069B1249024643
:1052100042F232301DF0A4FC38E600BF6C6600108C
:105220006018002060410020382704087027040817
:10523000B8270408CC270408C83600106C180020D2
:1052400094160120C1480108B038001081490108B6
:105250009027040801490108EC2704080000000019
:105260000BF046BE0000000000000000000000003F
:105270000BF026BE0000000000000000000000004F
:10528000022900D070472DE9F04F544BD3F8F8595C
:105290002DED028B47F22E52691E914285B004D942
:1052A00005B0BDEC028BBDE8F08F03F5236B4C4FCE
:1052B000DFF85091DFF850A1002303934FF030083E
:1052C000039EA8F13004D9F8003007EE906A03F588
:1052D000585292ED0D0AB8EEE78A38EE000A10EE49
:1052E000102A52456CD0B5EEC00AF1EE10FADBED93
:1052F000007A06D530EE270AB5EEC00AF1EE10FAB4
:10530000F8D4B4EEE70AF1EE10FA06DB30EE670AE5
:10531000F4EEC07AF1EE10FAF8D93249324A03F6C7
:10532000F813009321443B462846FDF7B1FED9F817
:10533000003003F5585292ED0E0A38EE000A10EED6
:10534000102A52452FD0B5EEC00AF1EE10FADBED6F
:10535000007A09D530EE270AB5EEC00AF1EE10FA50
:10536000F8D401E030EE670AF4EEC07AF1EE10FAFC
:10537000F8D91E491E4A03F6F813009321443B4610
:1053800028461834FDF784FEA04506F5B4769AD178
:10539000039B08F13008B433B8F1900F07F1100700
:1053A00003938DD17CE7134A134941F688101DF011
:1053B0007FFBDBED007AD9F800309FED100AD3E7D0
:1053C0000F4A0D4941F688101DF072FBDBED007AA3
:1053D000D9F800309FED090A93E700BFB02E001006
:1053E00098760020A0410020715201080042002060
:1053F00061520108D828040878250408000000003C
:10540000D0280408601800200000C07F00000000C1
:10541000054B1B6893F82C3703B97047034B0449BD
:105420001A680448FEF7BCB96C1800206018002008
:10543000A4280408815201080000000000000000B8
:105440002DE9F0412D4C2DED028B236893F82C377C
:1054500084B023B904B0BDEC028BBDE8F08119F033
:10546000DFFF274B10EE105A9D42F3D02168254FE5
:105470002548D7F8008001F6F422102301F6B42164
:1054800023F0BEFE43F2346621681F483C68B044F6
:1054900001F6743288ED000A102301F6343100EE73
:1054A000105A23F0ADFE3B6843F2386214441E44A8
:1054B00084ED000A1344D3ED008A96ED008AB4EE21
:1054C000E88AF1EE10FAC5DB2846F3F707F904463F
:1054D00018EE900A0D46F3F701F9CDE9020118EE36
:1054E000100AF3F7FBF82246CDE900012B460749E5
:1054F00041F2A9701DF0DCFAACE700BF6C18002087
:105500000000C07F60180020AC280408B028040800
:1055100038B5114D114C28460BF0BAF905F11800B9
:105520000BF0B6F905F130000BF0B2F905F14800C7
:105530000BF0AEF920460BF0ABF904F118000BF0BC
:10554000A7F904F130000BF0A3F904F14800BDE81D
:1055500038400BF09DB900BFA04100200042002060
:1055600038B501222DED068B0446022101F088FAA0
:105570002046002201219FED550ADFED558ADFED1F
:10558000559A01F075FC172501221146B0EE680A04
:10559000204601F06DFC78EEA98A0022B0EE680A80
:1055A0000121204601F064FC013D78EEA98AEBD18F
:1055B0009FED49AA9FED479A38EE8A8A0122B0EE04
:1055C000480A1146204601F053FC38EE0A8A2A4662
:1055D000B0EE480A0121204601F04AFC38EE298A43
:1055E000242501221146B0EE480A204601F040FC75
:1055F00038EE098A0022B0EE480A0121204601F067
:1056000037FC013D38EE098AEBD1294601229FED96
:10561000330A9FED309A204601F02AFC152501221D
:105620001146B0EE480A204601F022FC38EE098A05
:105630000022B0EE480A0121204601F019FC013D8C
:1056400038EE098AEBD1DFED249ADFED228A38EEBD
:10565000298A0122B0EE480A1146204601F008FCD2
:1056600038EE298A2A46B0EE480A0121204601F088
:10567000FFFB38EE098A212501221146B0EE480AC7
:10568000204601F0F5FB38EE288A0022B0EE480AE9
:105690000121204601F0ECFB013D38EE288AEBD1D8
:1056A0000122B0EE480A1146204601F0E1FB2A46ED
:1056B00029469FED0B0A204601F0DAFBBDEC068B74
:1056C0000123257084F86C3F38BD00BFC969BE3F17
:1056D00057CF8E40C9693E4057CF0E410000BC43B2
:1056E0000000344400000000000000000000000042
:1056F00070B5012205462DED028B0221B0EE408AE5
:1057000001F0BEF928469FED670A01F019FD05F684
:10571000687341F27842012400266349AC5428465C
:1057200085F86D6F22461960B3EE040A314601F028
:105730009FFB9FED5E0A324638EE000A214628465E
:1057400001F096FB9FED5A0A224638EE000A2146E8
:10575000284601F08DFB9FED570A324638EE000ACD
:105760002146284601F084FB9FED530A224638EE7D
:10577000000A2146284601F07BFB9FED500A324685
:1057800038EE000A2146284601F072FB9FED4C0AD4
:10579000224638EE000A2146284601F069FB9FEDBB
:1057A000490A324638EE000A2146284601F060FBDD
:1057B0009FED450A224638EE000A2146284601F0B0
:1057C00057FB3246314628469FED400A01F050FB18
:1057D0002246314628469FED3E0A01F049FB3246FB
:1057E000314628469FED3B0A01F042FB22463146F6
:1057F00028469FED390A01F03BFB9FED380A3246FF
:1058000038EE000A2146284601F032FB9FED340AAB
:10581000224638EE000A2146284601F029FB9FED7A
:10582000310A324638EE000A2146284601F020FBB4
:105830009FED2D0A224638EE000A2146284601F047
:1058400017FB9FED2A0A324638EE000A2146284609
:1058500001F00EFB9FED260A224638EE000A214693
:10586000284601F005FB9FED230A324638EE000A78
:105870002146284601F0FCFA9FED1F0A224638EE29
:10588000000A2146284601F0F3FA324631462846FE
:105890009FED1A0A01F0ECFABDEC028B85F86C4F13
:1058A00070BD00BFAE47E13D00008A430000844266
:1058B00000008C420000084300000C4300007643C7
:1058C00000007A4300009E430000A0430000AA436A
:1058D0000000B4430000BE430000C8430000D543AD
:1058E0000000D7430000F8430000FA43008017444B
:1058F000008018440000294400002A440000344479
:1059000070B501220446022101F0BAF8DFED330A36
:105910009FED330A204601F01BFB04F66873012556
:10592000002630499FED300A84F86D6F2A461960D1
:1059300020462946257001F09BFA3246294620462A
:105940009FED2A0A01F094FA2A46314620469FED3F
:10595000280A01F08DFA2A46294620469FED250A9D
:1059600001F086FA3246314620469FED230A01F0C7
:105970007FFA3246294620469FED200A01F078FA48
:105980002A46294620469FED1E0A01F071FA32464A
:10599000294620469FED1B0A01F06AFA2A46314645
:1059A00020469FED190A01F063FA2A46294620464F
:1059B0009FED160A01F05CFA3246294620469FED1B
:1059C000140A01F055FA3246314620469FED110A7D
:1059D00001F04EFA84F86C5F70BD00BF696FF83F4C
:1059E0002753653F0000934374D753429C45F542CB
:1059F000A4E55843DBA36843EC689043BB5297434C
:105A00005A39CE438A68F14346421044333814442D
:105A100095B9254400003444000000000000000057
:105A200038B502210546002201F02AF805F6687310
:105A30000024002285F86D4F28461A609FED1E0A4B
:105A400001F07EFB2246214628469FED1C0A01F00C
:105A50000FFA2146284601229FED190A01F008FAA3
:105A60002246214628469FED170A01F001FA2146F9
:105A7000284601229FED140A01F0FAF92246214638
:105A800028469FED120A01F0F3F92146284601222B
:105A90009FED0F0A01F0ECF92246214628469FEDC2
:105AA0000D0A01F0E5F92146284601229FED0A0A78
:105AB000BDE8384001F0DCB93333333F00007042B9
:105AC00000003443000070430000B4430000D243A0
:105AD0000000074400801A44000034440000000025
:105AE00010B504210446002200F0CAFF04F66873D2
:105AF000134A1A60DFED130A9FED130A204601F0E6
:105B000027FA0022204611469FED100A01F0B0F955
:105B10002046012200219FED0E0A01F0A9F9002282
:105B2000204611469FED0B0A01F0A2F92046012202
:105B300000219FED090ABDE8104001F099B900BFAE
:105B400000C0324448E17A3F3333B33E0000C043E3
:105B50000000C8430000304400003444000000004E
:105B60009FED010AFFF7C4BD000000000000000027
:105B7000BBEE060AFFF7BCBD0000000000000000FD
:105B800010B500220446022100F07AFF20460122CF
:105B900000219FED1C0A01F06BF9002211462046FE
:105BA0009FED190A01F064F92046012200219FEDC2
:105BB000170A01F05DF90022114620469FED140AF4
:105BC00001F056F92046012200219FED120A01F052
:105BD0004FF90022114620469FED0F0A01F048F9C7
:105BE0002046012200219FED0D0A01F041F900221B
:105BF000204611469FED0A0A01F03AF9002323706E
:105C000010BD00BF7B14E242000034431F85924365
:105C10000000B4431F85EC43000007448F42234437
:105C200000003444000000000000000000000000FC
:105C300038B5012205461446022100F021FF224614
:105C4000284600219FED250A85F86C4F01F010F9D8
:105C50002246214628469FED220A01F009F92146F5
:105C6000284600229FED1F0A01F002F9002211468A
:105C700028469FED1D0A01F0FBF8224621462846E2
:105C80009FED1A0A01F0F4F82146284600229FED04
:105C9000180A01F0EDF82246214628469FED150A24
:105CA00001F0E6F82146284600229FED130A01F094
:105CB000DFF82246214628469FED100A01F0D8F869
:105CC0002146002228469FED0E0A01F0D1F805F684
:105CD00068720C49116000232B7038BD94A8BE4235
:105CE0007269DC42D7053243CB72684391DA8F4345
:105CF0005E71B243E731EA4347B5064475AB2244CF
:105D000000003444811E0943000000000000000030
:105D100038B500F1720300EE103A012204460D4638
:105D20000846B8EEC00A114601F0A2F804F1740367
:105D300000EE103A2846B8EEC00A0022012101F018
:105D400097F804F1860300EE103A01222846114626
:105D5000B8EEC00A01F08CF804F1880300EE103AA6
:105D60002846B8EEC00A0022012101F081F804F1B2
:105D70009A0300EE103A012228461146B8EEC00AF6
:105D800001F076F804F19C0300EE103A2846B8EED4
:105D9000C00A0022012101F06BF804F1AE0300EE0D
:105DA000103A012228461146B8EEC00A01F060F808
:105DB00004F1B00300EE103A2846B8EEC00A002203
:105DC0000121BDE8384001F053B800BF00000000D9
:105DD00070B501222DED048B04469FED218ADFED85
:105DE000218ADFED219A9FED219A15460026022196
:105DF00000F046FEB0EE482AF0EE691AB0EE681ADE
:105E00003346B0EE490AFBEE090A2146284608222D
:105E100084F86D5F267003F063FCB0EE680A2A46D2
:105E20003146204601F024F8B0EE482AF0EE691A17
:105E3000B0EE681AB0EE490A334621462846DFED37
:105E40000C0A082203F04CFCB0EE480A32463146F8
:105E5000204601F00DF8BDEC048B84F86C5F70BD3A
:105E6000000034440000B443000000008FC2753DC0
:105E70000080A743000000000000000000000000B8
:105E800038B502210446002200F0FAFD04F66873DA
:105E900001253C4A84F86D5F20461A60F7EE080A37
:105EA000B6EE080A01F054F8F7EE040A2946204637
:105EB0009FED350A01F05CF82A46204684F86C5FB5
:105EC00000219FED320A00F0D3FF00222046114648
:105ED0009FED2F0A00F0CCFF2A46204600219FEDBF
:105EE0002D0A00F0C5FF0022204611469FED2A0A28
:105EF00000F0BEFF2A46204600219FED280A00F050
:105F0000B7FF0022204611469FED250A00F0B0FFA2
:105F10002A46204600219FED230A00F0A9FF002217
:105F2000204611469FED200A00F0A2FF2A46204697
:105F300000219FED1E0A00F09BFF00222046114623
:105F40009FED1B0A00F094FF2A46204600219FED9A
:105F5000190A00F08DFF0022204611469FED160A17
:105F600000F086FF2A46204600219FED140A00F02B
:105F70007FFF0022204611469FED110ABDE8384000
:105F800000F076BF0000F8436666263F000010432D
:105F9000000034430000584300007C43000090435D
:105FA0000000A2430000B4430000FC43000007448B
:105FB00000001044000019440000224400002B445B
:105FC0000000344400000000000000000000000059
:105FD00038B502210446002200F052FD04F6687331
:105FE00001255A4ADFED5A0A257020461A60B7EE9D
:105FF000040A00F0ADFF2A46204600219FED550A15
:1060000000F036FF0022204611469FED530A00F0B3
:106010002FFF2A46204600219FED500A00F028FF5E
:106020000022204611469FED4E0A00F021FF2A462D
:10603000204600219FED4B0A00F01AFF0022204667
:1060400011469FED490A00F013FF2A462046002121
:106050009FED460A00F00CFF0022204611469FEDFE
:10606000440A00F005FF2A46204600219FED410A20
:1060700000F0FEFE0022204611469FED3F0A00F090
:10608000F7FE2A46204600219FED3C0A00F0F0FE74
:106090000022204611469FED3A0A00F0E9FE2A460A
:1060A000204600219FED370A00F0E2FE0022204644
:1060B00011469FED350A00F0DBFE2A4620460021FE
:1060C0009FED320A00F0D4FE0022204611469FEDDB
